 instrument

 Timestamp is 6710e055 (Thu Oct 17 10:00:53 2024)

 Preferred load address is 10000000

 Start         Length     Name                   Class
 0001:00000000 0001d19fH .text$mn                CODE
 0001:0001d19f 000000bbH .text$x                 CODE
 0002:00000000 00000134H .idata$5                DATA
 0002:00000134 00000008H .00cfg                  DATA
 0002:0000013c 00000004H .CRT$XCA                DATA
 0002:00000140 00000004H .CRT$XCZ                DATA
 0002:00000144 00000004H .CRT$XIA                DATA
 0002:00000148 00000010H .CRT$XIC                DATA
 0002:00000158 00000004H .CRT$XIZ                DATA
 0002:0000015c 00000004H .CRT$XPA                DATA
 0002:00000160 00000008H .CRT$XPX                DATA
 0002:00000168 00000004H .CRT$XPXA               DATA
 0002:0000016c 00000004H .CRT$XPZ                DATA
 0002:00000170 00000004H .CRT$XTA                DATA
 0002:00000174 0000000cH .CRT$XTZ                DATA
 0002:00000178 00000000H .gfids$y                DATA
 0002:00000180 00009f80H .rdata                  DATA
 0002:0000a100 00000000H .rdata$CastGuardVftablesA DATA
 0002:0000a100 00000000H .rdata$CastGuardVftablesC DATA
 0002:0000a100 000000dcH .rdata$r                DATA
 0002:0000a1dc 00000028H .rdata$sxdata           DATA
 0002:0000a204 000001d8H .rdata$voltmd           DATA
 0002:0000a3dc 00000378H .rdata$zzzdbg           DATA
 0002:0000a754 00000004H .rtc$IAA                DATA
 0002:0000a758 00000004H .rtc$IZZ                DATA
 0002:0000a75c 00000004H .rtc$TAA                DATA
 0002:0000a760 00000008H .rtc$TZZ                DATA
 0002:0000a768 00000678H .xdata$x                DATA
 0002:0000ade0 00000388H .edata                  DATA
 0002:0000b168 00000014H .idata$2                DATA
 0002:0000b17c 00000014H .idata$3                DATA
 0002:0000b190 00000134H .idata$4                DATA
 0002:0000b2c4 00000588H .idata$6                DATA
 0003:00000000 000008e0H .data                   DATA
 0003:000008e0 0000003cH .data$r                 DATA
 0003:0000091c 0000001cH .data$rs                DATA
 0003:00000938 00000a78H .bss                    DATA
 0004:00000000 00000060H .rsrc$01                DATA
 0004:00000060 00000328H .rsrc$02                DATA

  Address         Publics by Value              Rva+Base       Lib:Object

 0000:00000000       ___AbsoluteZero            00000000     <absolute>
 0000:00000000       ___arm64x_extra_rfe_table  00000000     <absolute>
 0000:00000000       ___arm64x_extra_rfe_table_size 00000000     <absolute>
 0000:00000000       ___arm64x_native_entrypoint 00000000     <absolute>
 0000:00000000       ___arm64x_redirection_metadata 00000000     <absolute>
 0000:00000000       ___arm64x_redirection_metadata_count 00000000     <absolute>
 0000:00000000       ___dynamic_value_reloc_table 00000000     <absolute>
 0000:00000000       ___enclave_config          00000000     <absolute>
 0000:00000000       ___guard_check_icall_a64n_fptr 00000000     <absolute>
 0000:00000000       ___guard_eh_cont_count     00000000     <absolute>
 0000:00000000       ___guard_eh_cont_table     00000000     <absolute>
 0000:00000000       ___guard_fids_count        00000000     <absolute>
 0000:00000000       ___guard_fids_table        00000000     <absolute>
 0000:00000000       ___guard_iat_count         00000000     <absolute>
 0000:00000000       ___guard_iat_table         00000000     <absolute>
 0000:00000000       ___guard_longjmp_count     00000000     <absolute>
 0000:00000000       ___guard_longjmp_table     00000000     <absolute>
 0000:00000000       ___hybrid_auxiliary_delayload_iat 00000000     <absolute>
 0000:00000000       ___hybrid_auxiliary_delayload_iat_copy 00000000     <absolute>
 0000:00000000       ___hybrid_auxiliary_iat    00000000     <absolute>
 0000:00000000       ___hybrid_auxiliary_iat_copy 00000000     <absolute>
 0000:00000000       ___hybrid_code_map         00000000     <absolute>
 0000:00000000       ___hybrid_code_map_count   00000000     <absolute>
 0000:00000000       ___hybrid_image_info_bitfield 00000000     <absolute>
 0000:00000000       ___x64_code_ranges_to_entry_points 00000000     <absolute>
 0000:00000000       ___x64_code_ranges_to_entry_points_count 00000000     <absolute>
 0000:00000000       __except_list              00000000     <absolute>
 0000:0000000a       ___safe_se_handler_count   0000000a     <absolute>
 0000:00000100       ___guard_flags             00000100     <absolute>
 0000:00000000       ___ImageBase               10000000     <linker-defined>
 0001:00000000       _convertUtf8ToModifiedUtf8 10001000 f   EncodingSupport.obj
 0001:00000101       _modifiedUtf8LengthOfUtf8  10001101 f   EncodingSupport.obj
 0001:000001c9       _convertUft8ToPlatformString 100011c9 f   EncodingSupport_md.obj
 0001:000002a9       ___local_stdio_printf_options 100012a9 f i FileSystemSupport_md.obj
 0001:000002af       __vfprintf_l               100012af f i FileSystemSupport_md.obj
 0001:000002d2       _basePath                  100012d2 f   FileSystemSupport_md.obj
 0001:00000348       _fprintf                   10001348 f i FileSystemSupport_md.obj
 0001:00000360       _fromURIPath               10001360 f   FileSystemSupport_md.obj
 0001:000003ea       _isAbsolute                100013ea f   FileSystemSupport_md.obj
 0001:00000452       _normalize                 10001452 f   FileSystemSupport_md.obj
 0001:00000664       _resolve                   10001664 f   FileSystemSupport_md.obj
 0001:00000787       _Java_sun_instrument_InstrumentationImpl_appendToClassLoaderSearch0@24 10001787 f   InstrumentationImplNativeMethods.obj
 0001:000007a2       _Java_sun_instrument_InstrumentationImpl_getAllLoadedClasses0@16 100017a2 f   InstrumentationImplNativeMethods.obj
 0001:000007b4       _Java_sun_instrument_InstrumentationImpl_getInitiatedClasses0@20 100017b4 f   InstrumentationImplNativeMethods.obj
 0001:000007cb       _Java_sun_instrument_InstrumentationImpl_getObjectSize0@20 100017cb f   InstrumentationImplNativeMethods.obj
 0001:000007e2       _Java_sun_instrument_InstrumentationImpl_isModifiableClass0@20 100017e2 f   InstrumentationImplNativeMethods.obj
 0001:000007f9       _Java_sun_instrument_InstrumentationImpl_isRetransformClassesSupported0@16 100017f9 f   InstrumentationImplNativeMethods.obj
 0001:0000080b       _Java_sun_instrument_InstrumentationImpl_redefineClasses0@20 1000180b f   InstrumentationImplNativeMethods.obj
 0001:00000822       _Java_sun_instrument_InstrumentationImpl_retransformClasses0@20 10001822 f   InstrumentationImplNativeMethods.obj
 0001:00000839       _Java_sun_instrument_InstrumentationImpl_setHasRetransformableTransformers@20 10001839 f   InstrumentationImplNativeMethods.obj
 0001:00000850       _Java_sun_instrument_InstrumentationImpl_setNativeMethodPrefixes@24 10001850 f   InstrumentationImplNativeMethods.obj
 0001:0000086b       _Agent_OnAttach@12         1000186b f   InvocationAdapter.obj
 0001:00000b57       _Agent_OnLoad@12           10001b57 f   InvocationAdapter.obj
 0001:00000d9f       _Agent_OnUnload@4          10001d9f f   InvocationAdapter.obj
 0001:00001170       _convertCapabilityAtrributes 10002170 f   InvocationAdapter.obj
 0001:00001310       _eventHandlerClassFileLoadHook@40 10002310 f   InvocationAdapter.obj
 0001:00001368       _eventHandlerVMInit@12     10002368 f   InvocationAdapter.obj
 0001:000013b8       _getBooleanAttribute       100023b8 f   InvocationAdapter.obj
 0001:000014fe       _addNativeMethodPrefixCapability 100024fe f   JPLISAgent.obj
 0001:0000152d       _addOriginalMethodOrderCapability 1000252d f   JPLISAgent.obj
 0001:000015b5       _addRedefineClassesCapability 100025b5 f   JPLISAgent.obj
 0001:00001661       _allocateJPLISAgent        10002661 f   JPLISAgent.obj
 0001:0000166f       _appendToClassLoaderSearch 1000266f f   JPLISAgent.obj
 0001:0000176d       _checkCapabilities         1000276d f   JPLISAgent.obj
 0001:000017f2       _commandStringIntoJavaStrings 100027f2 f   JPLISAgent.obj
 0001:0000189c       _commonGetClassList        1000289c f   JPLISAgent.obj
 0001:0000195f       _createInstrumentationImpl 1000295f f   JPLISAgent.obj
 0001:00001bf7       _createNewJPLISAgent       10002bf7 f   JPLISAgent.obj
 0001:00001c8c       _deallocateCommandLineData 10002c8c f   JPLISAgent.obj
 0001:00001cb4       _enableNativeMethodPrefixCapability 10002cb4 f   JPLISAgent.obj
 0001:00001d36       _getAllLoadedClasses       10002d36 f   JPLISAgent.obj
 0001:00001d4e       _getAllLoadedClassesClassListFetcher 10002d4e f   JPLISAgent.obj
 0001:00001d64       _getInitiatedClasses       10002d64 f   JPLISAgent.obj
 0001:00001d7e       _getInitiatedClassesClassListFetcher 10002d7e f   JPLISAgent.obj
 0001:00001d98       _getJPLISEnvironment       10002d98 f   JPLISAgent.obj
 0001:00001e23       _getObjectArrayFromClasses 10002e23 f   JPLISAgent.obj
 0001:00001ee3       _getObjectSize             10002ee3 f   JPLISAgent.obj
 0001:00001f5b       _initializeJPLISAgent      10002f5b f   JPLISAgent.obj
 0001:000020c1       _invokeJavaAgentMainMethod 100030c1 f   JPLISAgent.obj
 0001:0000212d       _isModifiableClass         1000312d f   JPLISAgent.obj
 0001:00002178       _isRetransformClassesSupported 10003178 f   JPLISAgent.obj
 0001:00002180       _processJavaStart          10003180 f   JPLISAgent.obj
 0001:00002232       _recordCommandLineData     10003232 f   JPLISAgent.obj
 0001:000022d6       _redefineClassMapper       100032d6 f   JPLISAgent.obj
 0001:00002383       _redefineClasses           10003383 f   JPLISAgent.obj
 0001:0000280c       _retransformClasses        1000380c f   JPLISAgent.obj
 0001:000029d3       _retransformableEnvironment 100039d3 f   JPLISAgent.obj
 0001:00002b67       _setHasRetransformableTransformers 10003b67 f   JPLISAgent.obj
 0001:00002bc7       _setLivePhaseEventHandlers 10003bc7 f   JPLISAgent.obj
 0001:00002ca9       _setNativeMethodPrefixes   10003ca9 f   JPLISAgent.obj
 0001:00002f45       _startJavaAgent            10003f45 f   JPLISAgent.obj
 0001:00002f8b       _transformClassFile        10003f8b f   JPLISAgent.obj
 0001:0000323a       _JPLISAssertCondition      1000423a f   JPLISAssert.obj
 0001:00003264       _JPLISAssertConditionWithMessage 10004264 f   JPLISAssert.obj
 0001:0000333d       _freeAttributes            1000433d f   JarFacade.obj
 0001:0000336b       _getAttribute              1000436b f   JarFacade.obj
 0001:00003393       _readAttributes            10004393 f   JarFacade.obj
 0001:000033ed       _checkForAndClearThrowable 100043ed f   JavaExceptions.obj
 0001:0000340d       _checkForThrowable         1000440d f   JavaExceptions.obj
 0001:0000341b       _createAndThrowInternalError 1000441b f   JavaExceptions.obj
 0001:0000343d       _createAndThrowThrowableFromJVMTIErrorCode 1000443d f   JavaExceptions.obj
 0001:00003461       _createInternalError       10004461 f   JavaExceptions.obj
 0001:00003477       _createThrowable           10004477 f   JavaExceptions.obj
 0001:0000359e       _createThrowableFromJVMTIErrorCode 1000459e f   JavaExceptions.obj
 0001:000036f8       _getMessageFromThrowable   100046f8 f   JavaExceptions.obj
 0001:00003801       _initializeFallbackError   10004801 f   JavaExceptions.obj
 0001:0000385e       _isSafeForJNICalls         1000485e f   JavaExceptions.obj
 0001:00003872       _isUnchecked               10004872 f   JavaExceptions.obj
 0001:000038ff       _logThrowable              100048ff f   JavaExceptions.obj
 0001:00003917       _mapAllCheckedToInternalErrorMapper 10004917 f   JavaExceptions.obj
 0001:000039ae       _mapThrownThrowableIfNecessary 100049ae f   JavaExceptions.obj
 0001:000039ed       _preserveThrowable         100049ed f   JavaExceptions.obj
 0001:00003a0a       _restoreThrowable          10004a0a f   JavaExceptions.obj
 0001:00003a0f       _throwThrowable            10004a0f f   JavaExceptions.obj
 0001:00003d0e       _validatePathChars         10004d0e f   PathCharsValidator.obj
 0001:00003dfe       _assertTLSValue            10004dfe f   Reentrancy.obj
 0001:00003e5d       _confirmingTLSSet          10004e5d f   Reentrancy.obj
 0001:00003e92       _releaseReentrancyToken    10004e92 f   Reentrancy.obj
 0001:00003edc       _tryToAcquireReentrancyToken 10004edc f   Reentrancy.obj
 0001:00003f7e       _abortJVM                  10004f7e f   Utilities.obj
 0001:00003f8d       _allocate                  10004f8d f   Utilities.obj
 0001:00003fda       _deallocate                10004fda f   Utilities.obj
 0001:0000400e       _isInstanceofClassName     1000500e f   Utilities.obj
 0001:000040ba       _canonicalize              100050ba f   canonicalize_md.obj
 0001:000043ed       _lastErrorReportable       100053ed f   canonicalize_md.obj
 0001:0000445c       _JLI_ManifestIterate       1000545c f   jli_static:parse_manifest.obj
 0001:000050b5       _inflate                   100060b5 f   jli_static:inflate.obj
 0001:000065e1       _inflateEnd                100075e1 f   jli_static:inflate.obj
 0001:00006621       _inflateInit2_             10007621 f   jli_static:inflate.obj
 0001:000066c7       _inflateReset              100076c7 f   jli_static:inflate.obj
 0001:000066f0       _inflateReset2             100076f0 f   jli_static:inflate.obj
 0001:00006768       _inflateResetKeep          10007768 f   jli_static:inflate.obj
 0001:000068e1       _adler32                   100078e1 f   jli_static:zadler32.obj
 0001:000068e6       _adler32_z                 100078e6 f   jli_static:zadler32.obj
 0001:00006b23       _crc32                     10007b23 f   jli_static:zcrc32.obj
 0001:00006b28       _crc32_z                   10007b28 f   jli_static:zcrc32.obj
 0001:00006e11       _zcalloc                   10007e11 f   jli_static:zutil.obj
 0001:00006e22       _zcfree                    10007e22 f   jli_static:zutil.obj
 0001:00006e2d       _inflate_table             10007e2d f   jli_static:inftrees.obj
 0001:00007266       _inflate_fast              10008266 f   jli_static:inffast.obj
 0001:0000766e       @__security_check_cookie@4 1000866e f   LIBCMT:secchk.obj
 0001:000079bc       __DllMainCRTStartup@12     100089bc f   LIBCMT:dll_dllmain.obj
 0001:000079e0       __allrem                   100089e0 f   LIBCMT:llrem.obj
 0001:00007a92       ___raise_securityfailure   10008a92 f   LIBCMT:gs_report.obj
 0001:00007aba       ___report_gsfailure        10008aba f   LIBCMT:gs_report.obj
 0001:00007c01       ___security_init_cookie    10008c01 f   LIBCMT:gs_support.obj
 0001:00007c4c       _DllMain@12                10008c4c f   LIBCMT:dll_dllmain_stub.obj
 0001:00007c52       ?__scrt_initialize_type_info@@YAXXZ 10008c52 f   LIBCMT:tncleanup.obj
 0001:00007c5e       ?__scrt_uninitialize_type_info@@YAXXZ 10008c5e f   LIBCMT:tncleanup.obj
 0001:00007c6a       ___local_stdio_scanf_options 10008c6a f i LIBCMT:default_local_stdio_options.obj
 0001:00007c70       ___scrt_initialize_default_local_stdio_options 10008c70 f   LIBCMT:default_local_stdio_options.obj
 0001:00007cd1       ___scrt_acquire_startup_lock 10008cd1 f   LIBCMT:utility.obj
 0001:00007d03       ___scrt_dllmain_after_initialize_c 10008d03 f   LIBCMT:utility.obj
 0001:00007d2e       ___scrt_dllmain_before_initialize_c 10008d2e f   LIBCMT:utility.obj
 0001:00007d3c       ___scrt_dllmain_crt_thread_attach 10008d3c f   LIBCMT:utility.obj
 0001:00007d5b       ___scrt_dllmain_crt_thread_detach 10008d5b f   LIBCMT:utility.obj
 0001:00007d68       ___scrt_dllmain_exception_filter 10008d68 f   LIBCMT:utility.obj
 0001:00007d9c       ___scrt_dllmain_uninitialize_c 10008d9c f   LIBCMT:utility.obj
 0001:00007dbf       ___scrt_dllmain_uninitialize_critical 10008dbf f   LIBCMT:utility.obj
 0001:00007dcc       ___scrt_initialize_crt     10008dcc f   LIBCMT:utility.obj
 0001:00007e05       ___scrt_initialize_onexit_tables 10008e05 f   LIBCMT:utility.obj
 0001:00007e8c       ___scrt_is_nonwritable_in_current_image 10008e8c f   LIBCMT:utility.obj
 0001:00007f20       ___scrt_release_startup_lock 10008f20 f   LIBCMT:utility.obj
 0001:00007f3d       ___scrt_uninitialize_crt   10008f3d f   LIBCMT:utility.obj
 0001:00007f65       ___scrt_get_dyn_tls_init_callback 10008f65 f   LIBCMT:dyn_tls_init.obj
 0001:00007f6b       ___scrt_fastfail           10008f6b f   LIBCMT:utility_desktop.obj
 0001:00008086       __crt_debugger_hook        10009086 f   LIBCMT:utility_desktop.obj
 0001:0000808e       __RTC_Initialize           1000908e f   LIBCMT:initsect.obj
 0001:000080ba       __RTC_Terminate            100090ba f   LIBCMT:initsect.obj
 0001:000080f0       __SEH_prolog4              100090f0 f   LIBCMT:sehprolg4.obj
 0001:00008135       @_guard_check_icall_nop@4  10009135 f i LIBCMT:guard_support.obj
 0001:00008138       ___isa_available_init      10009138 f   LIBCMT:cpu_disp.obj
 0001:0000830c       __get_startup_argv_mode    1000930c f   LIBCMT:argv_mode.obj
 0001:00008310       ___scrt_is_ucrt_dll_in_use 10009310 f   LIBCMT:ucrt_detection.obj
 0001:00008320       _memcpy                    10009320 f   libvcruntime:memcpy.obj
 0001:00008320       _memmove                   10009320 f   libvcruntime:memmove.obj
 0001:000088a0       _strchr                    100098a0 f   libvcruntime:strchr.obj
 0001:0000890e       ___from_strstr_to_strchr   1000990e     libvcruntime:strchr.obj
 0001:000089d0       _memset                    100099d0 f   libvcruntime:memset.obj
 0001:00008b2a       _memcmp                    10009b2a f   libvcruntime:memcmp.obj
 0001:0000a1f0       __except_handler4          1000b1f0 f   libvcruntime:chandler4.obj
 0001:0000a34e       ___std_type_info_compare   1000b34e f   libvcruntime:std_type_info.obj
 0001:0000a38a       ___std_type_info_destroy_list 1000b38a f   libvcruntime:std_type_info.obj
 0001:0000a3ad       ___vcrt_initialize         1000b3ad f   libvcruntime:initialization.obj
 0001:0000a3cc       ___vcrt_thread_attach      1000b3cc f   libvcruntime:initialization.obj
 0001:0000a3d7       ___vcrt_thread_detach      1000b3d7 f   libvcruntime:initialization.obj
 0001:0000a3df       ___vcrt_uninitialize       1000b3df f   libvcruntime:initialization.obj
 0001:0000a3f6       ___vcrt_uninitialize_critical 1000b3f6 f   libvcruntime:initialization.obj
 0001:0000a3fe       ___DestructExceptionObject 1000b3fe f   libvcruntime:ehhelpers.obj
 0001:0000a49f       ?_CallMemberFunction0@@YGXQAX0@Z 1000b49f f i libvcruntime:ehhelpers.obj
 0001:0000a504       __IsExceptionObjectToBeDestroyed 1000b504 f   libvcruntime:ehhelpers.obj
 0001:0000a52a       ___AdjustPointer           1000b52a f   libvcruntime:ehhelpers.obj
 0001:0000a54f       ___FrameUnwindFilter       1000b54f f   libvcruntime:ehhelpers.obj
 0001:0000a5a5       ___std_terminate           1000b5a5 f   libvcruntime:ehhelpers.obj
 0001:0000a5b0       __local_unwind4            1000b5b0 f   libvcruntime:exsup4.obj
 0001:0000a6a0       @_EH4_CallFilterFunc@8     1000b6a0 f   libvcruntime:exsup4.obj
 0001:0000a6c0       @_EH4_TransferToHandler@8  1000b6c0 f   libvcruntime:exsup4.obj
 0001:0000a6e0       @_EH4_GlobalUnwind2@8      1000b6e0 f   libvcruntime:exsup4.obj
 0001:0000a700       @_EH4_LocalUnwind@16       1000b700 f   libvcruntime:exsup4.obj
 0001:0000a717       ___except_validate_context_record 1000b717 f   libvcruntime:jbcxrval.obj
 0001:0000a747       ___vcrt_freefls@4          1000b747 f   libvcruntime:per_thread_data.obj
 0001:0000a763       ___vcrt_freeptd_for_this_thread 1000b763 f   libvcruntime:per_thread_data.obj
 0001:0000a78e       ___vcrt_getptd             1000b78e f   libvcruntime:per_thread_data.obj
 0001:0000a79c       ___vcrt_getptd_noexit      1000b79c f   libvcruntime:per_thread_data.obj
 0001:0000a82e       ___vcrt_initialize_ptd     1000b82e f   libvcruntime:per_thread_data.obj
 0001:0000a861       ___vcrt_uninitialize_ptd   1000b861 f   libvcruntime:per_thread_data.obj
 0001:0000a87c       ___vcrt_initialize_locks   1000b87c f   libvcruntime:locks.obj
 0001:0000a8b8       ___vcrt_uninitialize_locks 1000b8b8 f   libvcruntime:locks.obj
 0001:0000a8f0       __NLG_Notify1              1000b8f0 f   libvcruntime:exsup.obj
 0001:0000a900       __NLG_Notify               1000b900 f   libvcruntime:exsup.obj
 0001:0000a917       __NLG_Dispatch             1000b917     libvcruntime:exsup.obj
 0001:0000a917       __NLG_Dispatch2            1000b917     libvcruntime:exsup.obj
 0001:0000a920       __NLG_Call                 1000b920 f   libvcruntime:exsup.obj
 0001:0000a922       __NLG_Return2              1000b922     libvcruntime:exsup.obj
 0001:0000a923       ?GetRangeOfTrysToCheck@__FrameHandler3@@SA?AU?$pair@Viterator@TryBlockMap@__FrameHandler3@@V123@@std@@AAVTryBlockMap@1@HPAXPBU_s_FuncInfo@@H@Z 1000b923 f   libvcruntime:trnsctrl.obj
 0001:0000a993       ?_CallCatchBlock2@@YAPAXPAUEHRegistrationNode@@PBU_s_FuncInfo@@PAXHK@Z 1000b993 f   libvcruntime:trnsctrl.obj
 0001:0000a9f0       ?_CallSETranslator@@YAHPAUEHExceptionRecord@@PAUEHRegistrationNode@@PAX2PBU_s_FuncInfo@@H1@Z 1000b9f0 f   libvcruntime:trnsctrl.obj
 0001:0000aae6       ?_JumpToContinuation@@YGXPAXPAUEHRegistrationNode@@@Z 1000bae6 f   libvcruntime:trnsctrl.obj
 0001:0000ab16       ?_UnwindNestedFrames@@YGXPAUEHRegistrationNode@@PAUEHExceptionRecord@@@Z 1000bb16 f   libvcruntime:trnsctrl.obj
 0001:0000ab69       __CatchGuardHandler        1000bb69 f   libvcruntime:trnsctrl.obj
 0001:0000ab9a       __CreateFrameInfo          1000bb9a f   libvcruntime:trnsctrl.obj
 0001:0000abbe       __FindAndUnlinkFrame       1000bbbe f   libvcruntime:trnsctrl.obj
 0001:0000ac06       __TranslatorGuardHandler   1000bc06 f   libvcruntime:trnsctrl.obj
 0001:0000aca3       ___CxxFrameHandler3        1000bca3 f   libvcruntime:trnsctrl.obj
 0001:0000adc4       ___vcrt_FlsAlloc           1000bdc4 f   libvcruntime:winapi_downlevel.obj
 0001:0000adff       ___vcrt_FlsFree            1000bdff f   libvcruntime:winapi_downlevel.obj
 0001:0000ae3a       ___vcrt_FlsGetValue        1000be3a f   libvcruntime:winapi_downlevel.obj
 0001:0000ae75       ___vcrt_FlsSetValue        1000be75 f   libvcruntime:winapi_downlevel.obj
 0001:0000aeb3       ___vcrt_InitializeCriticalSectionEx 1000beb3 f   libvcruntime:winapi_downlevel.obj
 0001:0000b62c       ??$TypeMatchHelper@V__FrameHandler3@@@@YAHPBU_s_HandlerType@@PBU_s_CatchableType@@PBU_s_ThrowInfo@@@Z 1000c62c f i libvcruntime:frame.obj
 0001:0000b6ba       ??$__InternalCxxFrameHandler@V__FrameHandler3@@@@YA?AW4_EXCEPTION_DISPOSITION@@PAUEHExceptionRecord@@PAUEHRegistrationNode@@PAU_CONTEXT@@PAXPBU_s_FuncInfo@@H1E@Z 1000c6ba f i libvcruntime:frame.obj
 0001:0000b7bc       ??$__InternalCxxFrameHandlerWrapper@V__FrameHandler3@@@@YA?AW4_EXCEPTION_DISPOSITION@@PAUEHExceptionRecord@@PAUEHRegistrationNode@@PAU_CONTEXT@@PAXPBU_s_FuncInfo@@H1E@Z 1000c7bc f i libvcruntime:frame.obj
 0001:0000b7c5       ??0bad_exception@std@@QAE@ABV01@@Z 1000c7c5 f i libvcruntime:frame.obj
 0001:0000b7e0       ??0bad_exception@std@@QAE@XZ 1000c7e0 f i libvcruntime:frame.obj
 0001:0000b7f8       ??0exception@std@@QAE@ABV01@@Z 1000c7f8 f i libvcruntime:frame.obj
 0001:0000b824       ??1bad_exception@std@@UAE@XZ 1000c824 f i libvcruntime:frame.obj
 0001:0000b835       ??8type_info@@QBE_NABV0@@Z 1000c835 f i libvcruntime:frame.obj
 0001:0000b854       ??_Ebad_exception@std@@UAEPAXI@Z 1000c854 f i libvcruntime:frame.obj
 0001:0000b854       ??_Eexception@std@@UAEPAXI@Z 1000c854 f i libvcruntime:frame.obj
 0001:0000b854       ??_Gbad_exception@std@@UAEPAXI@Z 1000c854 f i libvcruntime:frame.obj
 0001:0000b854       ??_Gexception@std@@UAEPAXI@Z 1000c854 f i libvcruntime:frame.obj
 0001:0000bad9       ?FrameUnwindToEmptyState@__FrameHandler3@@SAXPAUEHRegistrationNode@@PAXPBU_s_FuncInfo@@@Z 1000cad9 f   libvcruntime:frame.obj
 0001:0000baf1       ?FrameUnwindToState@__FrameHandler3@@SAXPAUEHRegistrationNode@@PAXPBU_s_FuncInfo@@H@Z 1000caf1 f   libvcruntime:frame.obj
 0001:0000bc73       ?_CallMemberFunction1@@YGXQAX00@Z 1000cc73 f i libvcruntime:frame.obj
 0001:0000bc83       ?_CallMemberFunction2@@YGXQAX00H@Z 1000cc83 f i libvcruntime:frame.obj
 0001:0000bc96       ?getESTypes@__FrameHandler3@@SAPBU_s_ESTypeList@@PBU_s_FuncInfo@@@Z 1000cc96 f i libvcruntime:frame.obj
 0001:0000bca1       ?what@exception@std@@UBEPBDXZ 1000cca1 f i libvcruntime:frame.obj
 0001:0000bcb0       __CallSettingFrame@12      1000ccb0 f   libvcruntime:lowhelpr.obj
 0001:0000bcd7       __NLG_Return               1000ccd7     libvcruntime:lowhelpr.obj
 0001:0000bcfc       _unexpected                1000ccfc f   libvcruntime:unexpected.obj
 0001:0000bd19       ?GetCurrentState@__FrameHandler3@@SAHPAUEHRegistrationNode@@PAXPBU_s_FuncInfo@@@Z 1000cd19 f   libvcruntime:ehstate.obj
 0001:0000bd36       ?SetState@__FrameHandler3@@SAXPAUEHRegistrationNode@@PBU_s_FuncInfo@@H@Z 1000cd36 f   libvcruntime:ehstate.obj
 0001:0000bd44       ___std_exception_copy      1000cd44 f   libvcruntime:std_exception.obj
 0001:0000bda7       ___std_exception_destroy   1000cda7 f   libvcruntime:std_exception.obj
 0001:0000bdc6       __CxxThrowException@8      1000cdc6 f   libvcruntime:throw.obj
 0001:0000be32       _free                      1000ce32 f   libucrt:free.obj
 0001:0000be4d       _malloc                    1000ce4d f   libucrt:malloc.obj
 0001:0000be58       ??$is_overflow_condition@K@__crt_strtox@@YA_NIK@Z 1000ce58 f i libucrt:atox.obj
 0001:0000be8c       ??$parse_integer@KV?$c_string_character_source@D@__crt_strtox@@$00@__crt_strtox@@YAKAAV__crt_cached_ptd_host@@V?$c_string_character_source@D@0@H_N@Z 1000ce8c f i libucrt:atox.obj
 0001:0000c0e0       ??0__crt_cached_ptd_host@@QAE@QAU__crt_locale_pointers@@@Z 1000d0e0 f i libucrt:atox.obj
 0001:0000c140       ??1__crt_cached_ptd_host@@QAE@XZ 1000d140 f i libucrt:atox.obj
 0001:0000c180       ?force_synchronize_per_thread_data@__crt_cached_ptd_host@@AAEPAU__acrt_ptd@@XZ 1000d180 f i libucrt:atox.obj
 0001:0000c1d0       ?get_raw_ptd@__crt_cached_ptd_host@@QAEPAU__acrt_ptd@@XZ 1000d1d0 f i libucrt:atox.obj
 0001:0000c22c       ?unget@?$c_string_character_source@D@__crt_strtox@@QAEXD@Z 1000d22c f i libucrt:atox.obj
 0001:0000c260       ?update_locale_slow@__crt_cached_ptd_host@@AAEXXZ 1000d260 f i libucrt:atox.obj
 0001:0000c2bb       ?validate@?$c_string_character_source@D@__crt_strtox@@QBE_NXZ 1000d2bb f i libucrt:atox.obj
 0001:0000c2d6       ___acrt_locale_get_ctype_array_value 1000d2d6 f i libucrt:atox.obj
 0001:0000c2f8       __ischartype_l             1000d2f8 f i libucrt:atox.obj
 0001:0000c34f       _atoi                      1000d34f f   libucrt:atox.obj
 0001:0000c38e       ___acrt_initialize_stdio   1000d38e f   libucrt:_file.obj
 0001:0000c456       ___acrt_iob_func           1000d456 f   libucrt:_file.obj
 0001:0000c466       ___acrt_uninitialize_stdio 1000d466 f   libucrt:_file.obj
 0001:0000c4b2       __lock_file                1000d4b2 f   libucrt:_file.obj
 0001:0000c4c6       __unlock_file              1000d4c6 f   libucrt:_file.obj
 0001:0000c535       ??$count@D@formatting_buffer@__crt_stdio_output@@QBEIXZ 1000d535 f i libucrt:output.obj
 0001:0000c54d       ??$ensure_buffer_is_big_enough@D@formatting_buffer@__crt_stdio_output@@QAE_NIAAV__crt_cached_ptd_host@@@Z 1000d54d f i libucrt:output.obj
 0001:0000c5ce       ??$is_wide_character_specifier@D@__crt_stdio_output@@YA_N_KDW4length_modifier@0@@Z 1000d5ce f i libucrt:output.obj
 0001:0000c5ff       ??$parse_integer@KV?$c_string_character_source@D@__crt_strtox@@$0A@@__crt_strtox@@YAKAAV__crt_cached_ptd_host@@V?$c_string_character_source@D@0@H_N@Z 1000d5ff f i libucrt:output.obj
 0001:0000c80e       ??$scratch_data@D@formatting_buffer@__crt_stdio_output@@QAEPADXZ 1000d80e f i libucrt:output.obj
 0001:0000c82c       ??$type_case_integer@$07@?$output_processor@DV?$stream_output_adapter@D@__crt_stdio_output@@V?$standard_base@DV?$stream_output_adapter@D@__crt_stdio_output@@@2@@__crt_stdio_output@@AAE_N_N@Z 1000d82c f i libucrt:output.obj
 0001:0000c9b9       ??$type_case_integer@$09@?$output_processor@DV?$stream_output_adapter@D@__crt_stdio_output@@V?$standard_base@DV?$stream_output_adapter@D@__crt_stdio_output@@@2@@__crt_stdio_output@@AAE_N_N@Z 1000d9b9 f i libucrt:output.obj
 0001:0000cb46       ??$type_case_integer@$0BA@@?$output_processor@DV?$stream_output_adapter@D@__crt_stdio_output@@V?$standard_base@DV?$stream_output_adapter@D@__crt_stdio_output@@@2@@__crt_stdio_output@@AAE_N_N@Z 1000db46 f i libucrt:output.obj
 0001:0000ccd3       ??$type_case_integer_parse_into_buffer@I$07@?$output_processor@DV?$stream_output_adapter@D@__crt_stdio_output@@V?$standard_base@DV?$stream_output_adapter@D@__crt_stdio_output@@@2@@__crt_stdio_output@@AAEXI_N@Z 1000dcd3 f i libucrt:output.obj
 0001:0000cd36       ??$type_case_integer_parse_into_buffer@I$09@?$output_processor@DV?$stream_output_adapter@D@__crt_stdio_output@@V?$standard_base@DV?$stream_output_adapter@D@__crt_stdio_output@@@2@@__crt_stdio_output@@AAEXI_N@Z 1000dd36 f i libucrt:output.obj
 0001:0000cdbd       ??$type_case_integer_parse_into_buffer@I$0BA@@?$output_processor@DV?$stream_output_adapter@D@__crt_stdio_output@@V?$standard_base@DV?$stream_output_adapter@D@__crt_stdio_output@@@2@@__crt_stdio_output@@AAEXI_N@Z 1000ddbd f i libucrt:output.obj
 0001:0000ce3a       ??$type_case_integer_parse_into_buffer@_K$07@?$output_processor@DV?$stream_output_adapter@D@__crt_stdio_output@@V?$standard_base@DV?$stream_output_adapter@D@__crt_stdio_output@@@2@@__crt_stdio_output@@AAEX_K_N@Z 1000de3a f i libucrt:output.obj
 0001:0000ceb2       ??$type_case_integer_parse_into_buffer@_K$09@?$output_processor@DV?$stream_output_adapter@D@__crt_stdio_output@@V?$standard_base@DV?$stream_output_adapter@D@__crt_stdio_output@@@2@@__crt_stdio_output@@AAEX_K_N@Z 1000deb2 f i libucrt:output.obj
 0001:0000cf59       ??$type_case_integer_parse_into_buffer@_K$0BA@@?$output_processor@DV?$stream_output_adapter@D@__crt_stdio_output@@V?$standard_base@DV?$stream_output_adapter@D@__crt_stdio_output@@@2@@__crt_stdio_output@@AAEX_K_N@Z 1000df59 f i libucrt:output.obj
 0001:0000cfe3       ??0?$output_adapter_data@DV?$stream_output_adapter@D@__crt_stdio_output@@@__crt_stdio_output@@IAE@ABV?$stream_output_adapter@D@1@_KQBDAAV__crt_cached_ptd_host@@QAD@Z 1000dfe3 f i libucrt:output.obj
 0001:0000d04a       ??1formatting_buffer@__crt_stdio_output@@QAE@XZ 1000e04a f i libucrt:output.obj
 0001:0000d064       ??4?$__crt_unique_heap_ptr@DU__crt_internal_free_policy@@@@QAEAAV0@$$QAV0@@Z 1000e064 f i libucrt:output.obj
 0001:0000d124       ?crop_zeroes@__crt_stdio_output@@YAXPADQAU__crt_locale_pointers@@@Z 1000e124 f i libucrt:output.obj
 0001:0000d184       ?find_next_state@?$output_processor@DV?$stream_output_adapter@D@__crt_stdio_output@@V?$standard_base@DV?$stream_output_adapter@D@__crt_stdio_output@@@2@@__crt_stdio_output@@ABE?AW4state@2@DW432@@Z 1000e184 f i libucrt:output.obj
 0001:0000d1bf       ?force_decimal_point@__crt_stdio_output@@YAXPADQAU__crt_locale_pointers@@@Z 1000e1bf f i libucrt:output.obj
 0001:0000d21b       ?parse_int_from_format_string@?$output_processor@DV?$stream_output_adapter@D@__crt_stdio_output@@V?$standard_base@DV?$stream_output_adapter@D@__crt_stdio_output@@@2@@__crt_stdio_output@@AAE_NQAH@Z 1000e21b f i libucrt:output.obj
 0001:0000d293       ?process@?$output_processor@DV?$stream_output_adapter@D@__crt_stdio_output@@V?$standard_base@DV?$stream_output_adapter@D@__crt_stdio_output@@@2@@__crt_stdio_output@@QAEHXZ 1000e293 f i libucrt:output.obj
 0001:0000d543       ?state_case_size@?$output_processor@DV?$stream_output_adapter@D@__crt_stdio_output@@V?$standard_base@DV?$stream_output_adapter@D@__crt_stdio_output@@@2@@__crt_stdio_output@@AAE_NXZ 1000e543 f i libucrt:output.obj
 0001:0000d69c       ?state_case_type@?$output_processor@DV?$stream_output_adapter@D@__crt_stdio_output@@V?$standard_base@DV?$stream_output_adapter@D@__crt_stdio_output@@@2@@__crt_stdio_output@@AAE_NXZ 1000e69c f i libucrt:output.obj
 0001:0000d9de       ?to_integer_size@__crt_stdio_output@@YAIW4length_modifier@1@@Z 1000e9de f i libucrt:output.obj
 0001:0000da32       ?type_case_Z@?$output_processor@DV?$stream_output_adapter@D@__crt_stdio_output@@V?$standard_base@DV?$stream_output_adapter@D@__crt_stdio_output@@@2@@__crt_stdio_output@@AAE_NXZ 1000ea32 f i libucrt:output.obj
 0001:0000da95       ?type_case_a@?$output_processor@DV?$stream_output_adapter@D@__crt_stdio_output@@V?$standard_base@DV?$stream_output_adapter@D@__crt_stdio_output@@@2@@__crt_stdio_output@@AAE_NXZ 1000ea95 f i libucrt:output.obj
 0001:0000dc26       ?type_case_c_tchar@?$output_processor@DV?$stream_output_adapter@D@__crt_stdio_output@@V?$standard_base@DV?$stream_output_adapter@D@__crt_stdio_output@@@2@@__crt_stdio_output@@AAE_ND@Z 1000ec26 f i libucrt:output.obj
 0001:0000dcbb       ?type_case_n@?$output_processor@DV?$stream_output_adapter@D@__crt_stdio_output@@V?$standard_base@DV?$stream_output_adapter@D@__crt_stdio_output@@@2@@__crt_stdio_output@@AAE_NXZ 1000ecbb f i libucrt:output.obj
 0001:0000dd40       ?type_case_o@?$output_processor@DV?$stream_output_adapter@D@__crt_stdio_output@@V?$standard_base@DV?$stream_output_adapter@D@__crt_stdio_output@@@2@@__crt_stdio_output@@AAE_NXZ 1000ed40 f i libucrt:output.obj
 0001:0000dd5d       ?type_case_p@?$output_processor@DV?$stream_output_adapter@D@__crt_stdio_output@@V?$standard_base@DV?$stream_output_adapter@D@__crt_stdio_output@@@2@@__crt_stdio_output@@AAE_NXZ 1000ed5d f i libucrt:output.obj
 0001:0000dd73       ?type_case_s@?$output_processor@DV?$stream_output_adapter@D@__crt_stdio_output@@V?$standard_base@DV?$stream_output_adapter@D@__crt_stdio_output@@@2@@__crt_stdio_output@@AAE_NXZ 1000ed73 f i libucrt:output.obj
 0001:0000dde5       ?validate@?$stream_output_adapter@D@__crt_stdio_output@@QBE_NAAV__crt_cached_ptd_host@@@Z 1000ede5 f i libucrt:output.obj
 0001:0000de1d       ?validate_stream_is_ansi_if_required@?$__acrt_stdio_char_traits@D@@SA_NQAU_iobuf@@@Z 1000ee1d f i libucrt:output.obj
 0001:0000dea4       ?write_character@?$output_adapter_common@DV?$stream_output_adapter@D@__crt_stdio_output@@@__crt_stdio_output@@QBEXDQAHAAV__crt_cached_ptd_host@@@Z 1000eea4 f i libucrt:output.obj
 0001:0000dec6       ?write_character_without_count_update@?$stream_output_adapter@D@__crt_stdio_output@@QBE_NDAAV__crt_cached_ptd_host@@@Z 1000eec6 f i libucrt:output.obj
 0001:0000df00       ?write_string@?$stream_output_adapter@D@__crt_stdio_output@@QBEXQBDHQAHAAV__crt_cached_ptd_host@@@Z 1000ef00 f i libucrt:output.obj
 0001:0000df2c       ?write_string_impl@?$output_adapter_common@DV?$stream_output_adapter@D@__crt_stdio_output@@@__crt_stdio_output@@IBEXQBDHQAHAAV__crt_cached_ptd_host@@@Z 1000ef2c f i libucrt:output.obj
 0001:0000dfab       ___stdio_common_vfprintf   1000efab f   libucrt:output.obj
 0001:0000e050       _strlen                    1000f050 f   libucrt:strlen.obj
 0001:0000e0e0       _strcpy                    1000f0e0 f   libucrt:strcat.obj
 0001:0000e0f0       _strcat                    1000f0f0 f   libucrt:strcat.obj
 0001:0000e1d8       _calloc                    1000f1d8 f   libucrt:calloc.obj
 0001:0000e1e3       _realloc                   1000f1e3 f   libucrt:realloc.obj
 0001:0000e1f0       _strncpy                   1000f1f0 f   libucrt:strncpy.obj
 0001:0000e314       ___acrt_errno_from_os_error 1000f314 f   libucrt:errno.obj
 0001:0000e357       ___acrt_errno_map_os_error 1000f357 f   libucrt:errno.obj
 0001:0000e37a       ___acrt_errno_map_os_error_ptd 1000f37a f   libucrt:errno.obj
 0001:0000e39e       ___doserrno                1000f39e f   libucrt:errno.obj
 0001:0000e3b1       __errno                    1000f3b1 f   libucrt:errno.obj
 0001:0000e3c4       ??$__acrt_convert_wcs_mbs_cp@D_WV<lambda_62f6974d9771e494a5ea317cc32e971c>@@U__crt_win32_buffer_internal_dynamic_resizing@@@@YAHQBDAAV?$__crt_win32_buffer@_WU__crt_win32_buffer_internal_dynamic_resizing@@@@ABV<lambda_62f6974d9771e494a5ea317cc32e971c>@@I@Z 1000f3c4 f i libucrt:fullpath.obj
 0001:0000e476       ??$__acrt_convert_wcs_mbs_cp@_WDV<lambda_0fec1a7b3f42a53036604e18c2d5e07e>@@U__crt_win32_buffer_no_resizing@@@@YAHQB_WAAV?$__crt_win32_buffer@DU__crt_win32_buffer_no_resizing@@@@ABV<lambda_0fec1a7b3f42a53036604e18c2d5e07e>@@I@Z 1000f476 f i libucrt:fullpath.obj
 0001:0000e538       ??$__acrt_convert_wcs_mbs_cp@_WDV<lambda_fecc33a432ccb74a901dff60d61ca385>@@U__crt_win32_buffer_public_dynamic_resizing@@@@YAHQB_WAAV?$__crt_win32_buffer@DU__crt_win32_buffer_public_dynamic_resizing@@@@ABV<lambda_fecc33a432ccb74a901dff60d61ca385>@@I@Z 1000f538 f i libucrt:fullpath.obj
 0001:0000e5fe       ??$__acrt_get_full_path_name_narrow_acp_or_utf8@U__crt_win32_buffer_no_resizing@@@@YAHQBDAAV?$__crt_win32_buffer@DU__crt_win32_buffer_no_resizing@@@@@Z 1000f5fe f i libucrt:fullpath.obj
 0001:0000e705       ??$__acrt_get_full_path_name_narrow_acp_or_utf8@U__crt_win32_buffer_public_dynamic_resizing@@@@YAHQBDAAV?$__crt_win32_buffer@DU__crt_win32_buffer_public_dynamic_resizing@@@@@Z 1000f705 f i libucrt:fullpath.obj
 0001:0000e80c       ??$__acrt_get_full_path_name_wide@U__crt_win32_buffer_internal_dynamic_resizing@@@@YAHQB_WAAV?$__crt_win32_buffer@_WU__crt_win32_buffer_internal_dynamic_resizing@@@@@Z 1000f80c f i libucrt:fullpath.obj
 0001:0000e826       ??$__acrt_mbs_to_wcs_cp@U__crt_win32_buffer_internal_dynamic_resizing@@@@YAHQBDAAV?$__crt_win32_buffer@_WU__crt_win32_buffer_internal_dynamic_resizing@@@@I@Z 1000f826 f i libucrt:fullpath.obj
 0001:0000e843       ??$__acrt_wcs_to_mbs_cp@U__crt_win32_buffer_no_resizing@@@@YAHQB_WAAV?$__crt_win32_buffer@DU__crt_win32_buffer_no_resizing@@@@I@Z 1000f843 f i libucrt:fullpath.obj
 0001:0000e860       ??$__acrt_wcs_to_mbs_cp@U__crt_win32_buffer_public_dynamic_resizing@@@@YAHQB_WAAV?$__crt_win32_buffer@DU__crt_win32_buffer_public_dynamic_resizing@@@@I@Z 1000f860 f i libucrt:fullpath.obj
 0001:0000e87d       ??$call_win32_function@V<lambda_44f1df80ccead0226c26eac3423fba1d>@@@?$__crt_win32_buffer@_WU__crt_win32_buffer_internal_dynamic_resizing@@@@QAEHABV<lambda_44f1df80ccead0226c26eac3423fba1d>@@@Z 1000f87d f i libucrt:fullpath.obj
 0001:0000e983       ??0_LocaleUpdate@@QAE@QAU__crt_locale_pointers@@@Z 1000f983 f i libucrt:fullpath.obj
 0001:0000ea05       ??R<lambda_0fec1a7b3f42a53036604e18c2d5e07e>@@QBE@IQB_WQADI@Z 1000fa05 f i libucrt:fullpath.obj
 0001:0000ea05       ??R<lambda_28bda7af82a03b66c1cb3803a755f95d>@@QBE@IQB_WQADI@Z 1000fa05 f i libucrt:argv_wildcards.obj
 0001:0000ea05       ??R<lambda_fecc33a432ccb74a901dff60d61ca385>@@QBE@IQB_WQADI@Z 1000fa05 f i libucrt:fullpath.obj
 0001:0000ea29       ?__acrt_get_utf8_acp_compatibility_codepage@@YAIXZ 1000fa29 f i libucrt:fullpath.obj
 0001:0000ea68       ?_deallocate@?$__crt_win32_buffer@DU__crt_win32_buffer_public_dynamic_resizing@@@@AAEXXZ 1000fa68 f i libucrt:fullpath.obj
 0001:0000ea82       ?_deallocate@?$__crt_win32_buffer@DU__crt_win32_buffer_internal_dynamic_resizing@@@@AAEXXZ 1000fa82 f i libucrt:argv_wildcards.obj
 0001:0000ea82       ?_deallocate@?$__crt_win32_buffer@_WU__crt_win32_buffer_internal_dynamic_resizing@@@@AAEXXZ 1000fa82 f i libucrt:fullpath.obj
 0001:0000ea9c       ?allocate@?$__crt_win32_buffer@DU__crt_win32_buffer_no_resizing@@@@QAEHI@Z 1000fa9c f i libucrt:fullpath.obj
 0001:0000eac3       ?allocate@?$__crt_win32_buffer@DU__crt_win32_buffer_public_dynamic_resizing@@@@QAEHI@Z 1000fac3 f i libucrt:fullpath.obj
 0001:0000eaff       ?allocate@?$__crt_win32_buffer@_WU__crt_win32_buffer_internal_dynamic_resizing@@@@QAEHI@Z 1000faff f i libucrt:fullpath.obj
 0001:0000eb3e       ?allocate@__crt_win32_buffer_internal_dynamic_resizing@@SAHQAPAXIABV__crt_win32_buffer_empty_debug_info@@@Z 1000fb3e f i libucrt:fullpath.obj
 0001:0000eb5d       ?allocate@__crt_win32_buffer_public_dynamic_resizing@@SAHQAPAXIABV__crt_win32_buffer_debug_info@@@Z 1000fb5d f i libucrt:fullpath.obj
 0001:0000eb7c       ?detach@?$__crt_win32_buffer@DU__crt_win32_buffer_public_dynamic_resizing@@@@QAEPADXZ 1000fb7c f i libucrt:fullpath.obj
 0001:0000ebc9       ?set_to_nullptr@?$__crt_win32_buffer@DU__crt_win32_buffer_no_resizing@@@@QAEXXZ 1000fbc9 f i libucrt:fullpath.obj
 0001:0000ebdd       __fullpath                 1000fbdd f   libucrt:fullpath.obj
 0001:0000ec7c       _strnlen                   1000fc7c f   libucrt:strnlen.obj
 0001:0000ed9e       _wcsnlen                   1000fd9e f   libucrt:strnlen.obj
 0001:0000ef4e       _wcsncmp                   1000ff4e f   libucrt:wcsncmp.obj
 0001:0000ef90       _isalpha                   1000ff90 f   libucrt:_ctype.obj
 0001:0000f01b       __toupper_l                1001001b f   libucrt:tolower_toupper.obj
 0001:0000f119       _toupper                   10010119 f   libucrt:tolower_toupper.obj
 0001:0000f150       _strpbrk                   10010150 f   libucrt:strpbrk.obj
 0001:0000f338       __lseeki64                 10010338 f   libucrt:lseek.obj
 0001:0000f378       __lseeki64_nolock          10010378 f   libucrt:lseek.obj
 0001:0000f3b8       __lseeki64_nolock_internal 100103b8 f   libucrt:lseek.obj
 0001:0000f3d6       __initterm                 100103d6 f   libucrt:initterm.obj
 0001:0000f401       __initterm_e               10010401 f   libucrt:initterm.obj
 0001:0000f42f       __seh_filter_dll           1001042f f   libucrt:exception_filter.obj
 0001:0000f44f       __seh_filter_exe           1001044f f   libucrt:exception_filter.obj
 0001:0000f5e2       ??$__crt_fast_decode_pointer@P6AHI@Z@@YAP6AHI@ZQ6AHI@Z@Z 100105e2 f i libucrt:new_handler.obj
 0001:0000f5e2       ??$__crt_fast_decode_pointer@P6AXH@Z@@YAP6AXH@ZQ6AXH@Z@Z 100105e2 f i libucrt:signal.obj
 0001:0000f5e2       ??$__crt_fast_decode_pointer@P6GXPAXK0@Z@@YAP6GXPAXK0@ZQ6GX0K0@Z@Z 100105e2 f i libucrt:exit.obj
 0001:0000f88a       ___acrt_initialize_thread_local_exit_callback 1001088a f   libucrt:exit.obj
 0001:0000f899       __cexit                    10010899 f   libucrt:exit.obj
 0001:0000f8a8       __exit                     100108a8 f   libucrt:exit.obj
 0001:0000f8be       __is_c_termination_complete 100108be f   libucrt:exit.obj
 0001:0000fb76       ___acrt_allocate_buffer_for_argv 10010b76 f   libucrt:argv_parsing.obj
 0001:0000fbc5       __configure_narrow_argv    10010bc5 f   libucrt:argv_parsing.obj
 0001:0000fd71       ___dcrt_uninitialize_environments_nolock 10010d71 f   libucrt:environment_initialization.obj
 0001:0000fdc2       __initialize_narrow_environment 10010dc2 f   libucrt:environment_initialization.obj
 0001:0000fefc       __execute_onexit_table     10010efc f   libucrt:onexit.obj
 0001:0000ff3a       __initialize_onexit_table  10010f3a f   libucrt:onexit.obj
 0001:0000ff8a       ___acrt_uninitialize_command_line 10010f8a f   libucrt:argv_data.obj
 0001:00010033       ??$__crt_fast_encode_pointer@PAX@@YAPAXQAX@Z 10011033 f i libucrt:initialization.obj
 0001:00010080       ___acrt_initialize         10011080 f   libucrt:initialization.obj
 0001:00010092       ___acrt_thread_attach      10011092 f   libucrt:initialization.obj
 0001:0001009d       ___acrt_thread_detach      1001109d f   libucrt:initialization.obj
 0001:000100a5       ___acrt_uninitialize       100110a5 f   libucrt:initialization.obj
 0001:000100d5       ___acrt_uninitialize_critical 100110d5 f   libucrt:initialization.obj
 0001:000100e7       _terminate                 100110e7 f   libucrt:terminate.obj
 0001:00010123       __strdup                   10011123 f   libucrt:strdup.obj
 0001:00010123       _strdup                    10011123 f   libucrt:strdup.obj
 0001:00010177       ___ascii_stricmp           10011177 f   libucrt:stricmp.obj
 0001:000101b0       __stricmp                  100111b0 f   libucrt:stricmp.obj
 0001:000101b0       _stricmp                   100111b0 f   libucrt:stricmp.obj
 0001:000101f9       __stricmp_l                100111f9 f   libucrt:stricmp.obj
 0001:0001031a       __close                    1001131a f   libucrt:close.obj
 0001:0001031a       _close                     1001131a f   libucrt:close.obj
 0001:0001034a       __close_internal           1001134a f   libucrt:close.obj
 0001:000103ed       __close_nolock             100113ed f   libucrt:close.obj
 0001:0001041d       __close_nolock_internal    1001141d f   libucrt:close.obj
 0001:00010a9d       __open                     10011a9d f   libucrt:open.obj
 0001:00010a9d       _open                      10011a9d f   libucrt:open.obj
 0001:00010ab5       __sopen_nolock             10011ab5 f   libucrt:open.obj
 0001:00010b23       __wsopen_nolock            10011b23 f   libucrt:open.obj
 0001:00011329       __read                     10012329 f   libucrt:read.obj
 0001:00011329       _read                      10012329 f   libucrt:read.obj
 0001:00011442       __read_nolock              10012442 f   libucrt:read.obj
 0001:000117cd       _strcpy_s                  100127cd f   libucrt:strcpy_s.obj
 0001:00011827       _abort                     10012827 f   libucrt:abort.obj
 0001:00011870       _strncmp                   10012870 f   libucrt:strncmp.obj
 0001:000118e8       __free_base                100128e8 f   libucrt:free_base.obj
 0001:00011922       __malloc_base              10012922 f   libucrt:malloc_base.obj
 0001:00011970       ?check_synchronize_global_state_index@__crt_cached_ptd_host@@AAEIXZ 10012970 f i libucrt:invalid_parameter.obj
 0001:00011999       ___acrt_call_reportfault   10012999 f   libucrt:invalid_parameter.obj
 0001:00011ad2       ___acrt_initialize_invalid_parameter_handler 10012ad2 f   libucrt:invalid_parameter.obj
 0001:00011ae1       __invalid_parameter        10012ae1 f   libucrt:invalid_parameter.obj
 0001:00011b18       __invalid_parameter_internal 10012b18 f   libucrt:invalid_parameter.obj
 0001:00011b95       __invalid_parameter_noinfo 10012b95 f   libucrt:invalid_parameter.obj
 0001:00011ba5       __invoke_watson            10012ba5 f   libucrt:invalid_parameter.obj
 0001:00011bd9       ___pctype_func             10012bd9 f   libucrt:ctype.obj
 0001:00011bfd       __isctype_l                10012bfd f   libucrt:isctype.obj
 0001:00011cc8       ___acrt_update_locale_info 10012cc8 f   libucrt:locale_update.obj
 0001:00011cf5       ___acrt_update_locale_info_explicit 10012cf5 f   libucrt:locale_update.obj
 0001:00011d26       ___acrt_update_multibyte_info 10012d26 f   libucrt:locale_update.obj
 0001:00011d53       ___acrt_update_multibyte_info_explicit 10012d53 f   libucrt:locale_update.obj
 0001:000120c2       ___acrt_freeptd            100130c2 f   libucrt:per_thread_data.obj
 0001:000120ee       ___acrt_getptd             100130ee f   libucrt:per_thread_data.obj
 0001:000121a9       ___acrt_getptd_head        100131a9 f   libucrt:per_thread_data.obj
 0001:0001223f       ___acrt_getptd_noexit      1001323f f   libucrt:per_thread_data.obj
 0001:000122f0       ___acrt_getptd_noexit_explicit 100132f0 f   libucrt:per_thread_data.obj
 0001:00012393       ___acrt_initialize_ptd     10013393 f   libucrt:per_thread_data.obj
 0001:000123bf       ___acrt_uninitialize_ptd   100133bf f   libucrt:per_thread_data.obj
 0001:00012447       ___acrt_set_locale_changed 10013447 f   libucrt:wsetlocale.obj
 0001:00012452       ___acrt_uninitialize_locale 10013452 f   libucrt:wsetlocale.obj
 0001:00012479       __calloc_base              10013479 f   libucrt:calloc_base.obj
 0001:00012674       ___acrt_AppPolicyGetProcessTerminationMethodInternal@4 10013674 f   libucrt:winapi_thunks.obj
 0001:000126b4       ___acrt_AreFileApisANSI@0  100136b4 f   libucrt:winapi_thunks.obj
 0001:000126d3       ___acrt_FlsAlloc@4         100136d3 f   libucrt:winapi_thunks.obj
 0001:00012712       ___acrt_FlsFree@4          10013712 f   libucrt:winapi_thunks.obj
 0001:00012751       ___acrt_FlsGetValue@4      10013751 f   libucrt:winapi_thunks.obj
 0001:00012790       ___acrt_FlsSetValue@8      10013790 f   libucrt:winapi_thunks.obj
 0001:000127d2       ___acrt_InitializeCriticalSectionEx@12 100137d2 f   libucrt:winapi_thunks.obj
 0001:0001281d       ___acrt_LCMapStringEx@36   1001381d f   libucrt:winapi_thunks.obj
 0001:0001287a       ___acrt_LocaleNameToLCID@8 1001387a f   libucrt:winapi_thunks.obj
 0001:000128ab       ___acrt_initialize_winapi_thunks 100138ab f   libucrt:winapi_thunks.obj
 0001:000128bf       ___acrt_uninitialize_winapi_thunks 100138bf f   libucrt:winapi_thunks.obj
 0001:000128f5       __fcloseall                100138f5 f   libucrt:closeall.obj
 0001:00012b79       ___acrt_stdio_flush_nolock 10013b79 f   libucrt:fflush.obj
 0001:00012be2       __fflush_nolock            10013be2 f   libucrt:fflush.obj
 0001:00012c47       __flushall                 10013c47 f   libucrt:fflush.obj
 0001:00012c50       ___acrt_stdio_free_buffer_nolock 10013c50 f   libucrt:_freebuf.obj
 0001:00012df6       ___acrt_initialize_lowio   10013df6 f   libucrt:ioinit.obj
 0001:00012e56       ___acrt_uninitialize_lowio 10013e56 f   libucrt:ioinit.obj
 0001:00012e82       ?__acrt_fp_classify@@YA?AW4__acrt_fp_class@@ABN@Z 10013e82 f i libucrt:cvt.obj
 0001:0001385a       ___acrt_fp_format          1001485a f   libucrt:cvt.obj
 0001:000139db       __wctomb_internal          100149db f   libucrt:wctomb.obj
 0001:00013b45       __mbtowc_internal          10014b45 f   libucrt:mbtowc.obj
 0001:00013c78       __fileno                   10014c78 f   libucrt:fileno.obj
 0001:00013c9f       __get_printf_count_output  10014c9f f   libucrt:printf_count_output.obj
 0001:00013cb4       __fputc_nolock_internal    10014cb4 f   libucrt:fputc.obj
 0001:00013ce1       ___acrt_should_use_temporary_buffer 10014ce1 f   libucrt:_sftbuf.obj
 0001:00013d1f       ___acrt_stdio_begin_temporary_buffering_nolock 10014d1f f   libucrt:_sftbuf.obj
 0001:00013dca       ___acrt_stdio_end_temporary_buffering_nolock 10014dca f   libucrt:_sftbuf.obj
 0001:00013e08       __realloc_base             10014e08 f   libucrt:realloc_base.obj
 0001:0001401e       __getcwd                   1001501e f   libucrt:getcwd.obj
 0001:000140d2       ___acrt_MultiByteToWideChar 100150d2 f   libucrt:multibytetowidechar.obj
 0001:0001418c       ___acrt_WideCharToMultiByte 1001518c f   libucrt:widechartomultibyte.obj
 0001:000143e7       ___acrt_LCMapStringA       100153e7 f   libucrt:lcmapstringa.obj
 0001:00014430       __freea_crt                10015430 f i libucrt:lcmapstringa.obj
 0001:00014450       ___acrt_lowio_create_handle_array 10015450 f   libucrt:osfinfo.obj
 0001:000144cb       ___acrt_lowio_destroy_handle_array 100154cb f   libucrt:osfinfo.obj
 0001:00014500       ___acrt_lowio_ensure_fh_exists 10015500 f   libucrt:osfinfo.obj
 0001:0001459e       ___acrt_lowio_lock_fh      1001559e f   libucrt:osfinfo.obj
 0001:000145c1       ___acrt_lowio_set_os_handle 100155c1 f   libucrt:osfinfo.obj
 0001:00014653       ___acrt_lowio_unlock_fh    10015653 f   libucrt:osfinfo.obj
 0001:00014676       __alloc_osfhnd             10015676 f   libucrt:osfinfo.obj
 0001:00014789       __free_osfhnd              10015789 f   libucrt:osfinfo.obj
 0001:0001481a       __get_osfhandle            1001581a f   libucrt:osfinfo.obj
 0001:00014884       ___acrt_initialize_locks   10015884 f   libucrt:locks.obj
 0001:000148c5       ___acrt_lock               100158c5 f   libucrt:locks.obj
 0001:000148dc       ___acrt_uninitialize_locks 100158dc f   libucrt:locks.obj
 0001:0001490d       ___acrt_unlock             1001590d f   libucrt:locks.obj
 0001:00014924       ___acrt_app_verifier_enabled 10015924 f   libucrt:peb_access.obj
 0001:00014936       ___acrt_is_secure_process  10015936 f   libucrt:peb_access.obj
 0001:00014949       ___acrt_get_process_end_policy 10015949 f   libucrt:win_policies.obj
 0001:00014988       ??$__acrt_convert_wcs_mbs_cp@_WDV<lambda_28bda7af82a03b66c1cb3803a755f95d>@@U__crt_win32_buffer_internal_dynamic_resizing@@@@YAHQB_WAAV?$__crt_win32_buffer@DU__crt_win32_buffer_internal_dynamic_resizing@@@@ABV<lambda_28bda7af82a03b66c1cb3803a755f95d>@@I@Z 10015988 f i libucrt:argv_wildcards.obj
 0001:00014f26       ?allocate@?$__crt_win32_buffer@DU__crt_win32_buffer_internal_dynamic_resizing@@@@QAEHI@Z 10015f26 f i libucrt:argv_wildcards.obj
 0001:00014fe9       ___acrt_expand_narrow_argv_wildcards 10015fe9 f   libucrt:argv_wildcards.obj
 0001:00014ff4       ___acrt_GetModuleFileNameA 10015ff4 f   libucrt:getmodulefilenamea.obj
 0001:00015611       ___acrt_initialize_multibyte 10016611 f   libucrt:mbctype.obj
 0001:00015659       ___acrt_update_thread_multibyte_data 10016659 f   libucrt:mbctype.obj
 0001:0001566c       __setmbcp_nolock           1001666c f   libucrt:mbctype.obj
 0001:000158c1       __ismbblead                100168c1 f   libucrt:ismbbyte.obj
 0001:000158d9       ___acrt_initialize_command_line 100168d9 f   libucrt:argv_data.obj
 0001:00015929       ___dcrt_get_narrow_environment_from_os 10016929 f   libucrt:get_environment_from_os.obj
 0001:000159c9       __recalloc_base            100169c9 f   libucrt:recalloc.obj
 0001:00015a36       ___acrt_initialize_heap    10016a36 f   libucrt:heap_handle.obj
 0001:00015a47       ___acrt_uninitialize_heap  10016a47 f   libucrt:heap_handle.obj
 0001:00015a51       ___acrt_execute_initializers 10016a51 f   libucrt:shared_initialization.obj
 0001:00015ab9       ___acrt_execute_uninitializers 10016ab9 f   libucrt:shared_initialization.obj
 0001:00015aea       ___acrt_initialize_new_handler 10016aea f   libucrt:new_handler.obj
 0001:00015af9       __callnewh                 10016af9 f   libucrt:new_handler.obj
 0001:00015b25       __query_new_handler        10016b25 f   libucrt:new_handler.obj
 0001:00015c4e       ___acrt_get_sigabrt_handler 10016c4e f   libucrt:signal.obj
 0001:00015c75       ___acrt_initialize_signal_handlers 10016c75 f   libucrt:signal.obj
 0001:00015c93       _raise                     10016c93 f   libucrt:signal.obj
 0001:00015e85       ___acrt_has_user_matherr   10016e85 f   libucrt:matherr.obj
 0001:00015ea2       ___acrt_initialize_user_matherr 10016ea2 f   libucrt:matherr.obj
 0001:00015eb1       ___acrt_invoke_user_matherr 10016eb1 f   libucrt:matherr.obj
 0001:00016689       __write                    10017689 f   libucrt:write.obj
 0001:000166c0       __write_internal           100176c0 f   libucrt:write.obj
 0001:000167d1       __write_nolock             100177d1 f   libucrt:write.obj
 0001:000169ed       __get_fmode                100179ed f   libucrt:setmode.obj
 0001:00016a1a       __setmode_nolock           10017a1a f   libucrt:setmode.obj
 0001:00016ae9       ??0__crt_seek_guard@@QAE@H_J@Z 10017ae9 f i libucrt:chsize.obj
 0001:00016b36       __chsize_nolock            10017b36 f   libucrt:chsize.obj
 0001:00016b6d       __chsize_nolock_internal   10017b6d f   libucrt:chsize.obj
 0001:00016d04       __isatty                   10017d04 f   libucrt:isatty.obj
 0001:00016d5a       __query_new_mode           10017d5a f   libucrt:new_mode.obj
 0001:00016d61       ___acrt_GetStringTypeA     10017d61 f   libucrt:getstringtypea.obj
 0001:00016e62       ___acrt_add_locale_ref     10017e62 f   libucrt:locale_refcounting.obj
 0001:00016edf       ___acrt_free_locale        10017edf f   libucrt:locale_refcounting.obj
 0001:00017027       ___acrt_locale_add_lc_time_reference 10018027 f   libucrt:locale_refcounting.obj
 0001:00017050       ___acrt_locale_free_lc_time_if_unreferenced 10018050 f   libucrt:locale_refcounting.obj
 0001:00017081       ___acrt_locale_release_lc_time_reference 10018081 f   libucrt:locale_refcounting.obj
 0001:000170aa       ___acrt_release_locale_ref 100180aa f   libucrt:locale_refcounting.obj
 0001:0001712b       ___acrt_update_thread_locale_data 1001812b f   libucrt:locale_refcounting.obj
 0001:000171ac       __updatetlocinfoEx_nolock  100181ac f   libucrt:locale_refcounting.obj
 0001:000171fc       ___acrt_locale_free_monetary 100181fc f   libucrt:initmon.obj
 0001:000172fa       ___acrt_locale_free_numeric 100182fa f   libucrt:initnum.obj
 0001:00017388       ___acrt_locale_free_time   10018388 f   libucrt:inittime.obj
 0001:000174bc       ___acrt_DownlevelLocaleNameToLCID 100184bc f   libucrt:lcidtoname_downlevel.obj
 0001:0001760d       _fclose                    1001860d f   libucrt:fclose.obj
 0001:000176df       __commit                   100186df f   libucrt:commit.obj
 0001:0001780d       ___acrt_fp_strflt_to_string 1001880d f   libucrt:_fptostr.obj
 0001:00017910       ?divide@__crt_strtox@@YA_KAAUbig_integer@1@ABU21@@Z 10018910 f i libucrt:cfout.obj
 0001:00017dbb       ___acrt_fltout             10018dbb f   libucrt:cfout.obj
 0001:000193a3       _fegetround                1001a3a3 f   libucrt:fegetround.obj
 0001:000193b0       ?__c32rtomb_utf8@__crt_mbstring@@YAIPAD_UPAU_Mbstatet@@AAV__crt_cached_ptd_host@@@Z 1001a3b0 f   libucrt:c32rtomb.obj
 0001:0001948c       ?__mbrtowc_utf8@__crt_mbstring@@YAIPA_WPBDIPAU_Mbstatet@@AAV__crt_cached_ptd_host@@@Z 1001a48c f   libucrt:mbrtowc.obj
 0001:000194cf       ?__mbsrtowcs_utf8@__crt_mbstring@@YAIPA_WPAPBDIPAU_Mbstatet@@AAV__crt_cached_ptd_host@@@Z 1001a4cf f   libucrt:mbrtowc.obj
 0001:00019824       ___acrt_stdio_flush_and_write_narrow_nolock 1001a824 f   libucrt:_flsbuf.obj
 0001:0001985a       __getdrive                 1001a85a f   libucrt:drive.obj
 0001:000198fe       ___strncnt                 1001a8fe f   libucrt:strncnt.obj
 0001:0001991a       __query_app_type           1001a91a f   libucrt:report_runtime_error.obj
 0001:00019920       _qsort                     1001a920 f   libucrt:qsort.obj
 0001:00019ec5       _strncpy_s                 1001aec5 f   libucrt:strncpy_s.obj
 0001:00019ed0       __mbsdec                   1001aed0 f   libucrt:mbsdec.obj
 0001:00019ee7       __mbsdec_l                 1001aee7 f   libucrt:mbsdec.obj
 0001:00019f83       __msize_base               1001af83 f   libucrt:msize.obj
 0001:00019fb6       __putwch_nolock            1001afb6 f   libucrt:putwch.obj
 0001:00019fe8       ___acrt_initialize_fmode   1001afe8 f   libucrt:txtmode.obj
 0001:00019ffe       ___ascii_wcsnicmp          1001affe f   libucrt:wcsnicmp.obj
 0001:0001a04d       ?__acrt_stdio_free_stream@@YAXV__crt_stdio_stream@@@Z 1001b04d f   libucrt:stream.obj
 0001:0001a088       __controlfp_s              1001b088 f   libucrt:contrlfp.obj
 0001:0001a0e7       _fegetenv                  1001b0e7 f   libucrt:fegetenv.obj
 0001:0001a104       _fesetenv                  1001b104 f   libucrt:fesetenv.obj
 0001:0001a150       _feholdexcept              1001b150 f   libucrt:feholdexcept.obj
 0001:0001a1a0       __CIlog10                  1001b1a0 f   libucrt:log10_impl.obj
 0001:0001a1db       __CIlog10_default          1001b1db f   libucrt:log10_impl.obj
 0001:0001a1ef       __log10_default            1001b1ef     libucrt:log10_impl.obj
 0001:0001a2b0       _ceil                      1001b2b0 f   libucrt:ceil_pentium4.obj
 0001:0001a2f0       __ceil_pentium4            1001b2f0 f   libucrt:ceil_pentium4.obj
 0001:0001a696       ___acrt_fenv_get_common_round_control 1001b696 f   libucrt:_fenvutils.obj
 0001:0001a6b8       ___acrt_fenv_get_control   1001b6b8 f   libucrt:_fenvutils.obj
 0001:0001a738       ___acrt_fenv_get_status    1001b738 f   libucrt:_fenvutils.obj
 0001:0001a7e2       ___acrt_fenv_set_control   1001b7e2 f   libucrt:_fenvutils.obj
 0001:0001a85d       ___acrt_fenv_set_status    1001b85d f   libucrt:_fenvutils.obj
 0001:0001a959       ?reset_and_return@__crt_mbstring@@YAIIPAU_Mbstatet@@@Z 1001b959 f   libucrt:common_utf8.obj
 0001:0001a96d       ?return_illegal_sequence@__crt_mbstring@@YAIPAU_Mbstatet@@AAV__crt_cached_ptd_host@@@Z 1001b96d f   libucrt:common_utf8.obj
 0001:0001a98f       ?__mbrtoc32_utf8@__crt_mbstring@@YAIPA_UPBDIPAU_Mbstatet@@AAV__crt_cached_ptd_host@@@Z 1001b98f f   libucrt:mbrtoc32.obj
 0001:0001ab40       ___acrt_stdio_allocate_buffer_nolock 1001bb40 f   libucrt:_getbuf.obj
 0001:0001abbb       ___dcrt_lowio_ensure_console_output_initialized 1001bbbb f   libucrt:initcon.obj
 0001:0001abda       ___dcrt_terminate_console_output 1001bbda f   libucrt:initcon.obj
 0001:0001abf1       ___dcrt_write_console      1001bbf1 f   libucrt:initcon.obj
 0001:0001aced       __clearfp                  1001bced f   libucrt:ieee87.obj
 0001:0001adcb       __control87                1001bdcb f   libucrt:ieee87.obj
 0001:0001b16a       ___acrt_initialize_sse2    1001c16a f   libucrt:mathfcns.obj
 0001:0001b180       __CIlog10_pentium4         1001c180 f   libucrt:log10_pentium4.obj
 0001:0001b198       __log10_pentium4           1001c198     libucrt:log10_pentium4.obj
 0001:0001b430       __fFEXP                    1001c430 f   libucrt:87tran.obj
 0001:0001b487       __rtinfpopse               1001c487     libucrt:87tran.obj
 0001:0001b489       __rtinfnpopse              1001c489     libucrt:87tran.obj
 0001:0001b499       __fFLN                     1001c499     libucrt:87tran.obj
 0001:0001b54e       __rtinfpop                 1001c54e     libucrt:87tran.obj
 0001:0001b550       __rtinfnpop                1001c550     libucrt:87tran.obj
 0001:0001b560       __rtforexpinf              1001c560 f   libucrt:87tran.obj
 0001:0001b56d       __ffexpm1                  1001c56d     libucrt:87tran.obj
 0001:0001b620       __trandisp1                1001c620 f   libucrt:87disp.obj
 0001:0001b695       __trandisp2                1001c695 f   libucrt:87disp.obj
 0001:0001b72f       __rttospopde               1001c72f     libucrt:87disp.obj
 0001:0001b734       __rttospop                 1001c734     libucrt:87disp.obj
 0001:0001b740       __rtnospop                 1001c740 f   libucrt:87disp.obj
 0001:0001b750       __rttosnpop                1001c750 f   libucrt:87disp.obj
 0001:0001b751       __rtnospopde               1001c751     libucrt:87disp.obj
 0001:0001b758       __rtzeropop                1001c758     libucrt:87disp.obj
 0001:0001b75a       __rtzeronpop               1001c75a     libucrt:87disp.obj
 0001:0001b760       __rtzerospop               1001c760 f   libucrt:87disp.obj
 0001:0001b76d       __rtonepop                 1001c76d     libucrt:87disp.obj
 0001:0001b770       __rtonenpop                1001c770 f   libucrt:87disp.obj
 0001:0001b780       __tosnan1                  1001c780 f   libucrt:87disp.obj
 0001:0001b7b0       __nosnan2                  1001c7b0 f   libucrt:87disp.obj
 0001:0001b7c0       __tosnan2                  1001c7c0 f   libucrt:87disp.obj
 0001:0001b7f0       __nan2                     1001c7f0 f   libucrt:87disp.obj
 0001:0001b830       __rtindfpop                1001c830 f   libucrt:87disp.obj
 0001:0001b832       __rtindfnpop               1001c832     libucrt:87disp.obj
 0001:0001b843       __rttosnpopde              1001c843     libucrt:87disp.obj
 0001:0001b850       __rtatan2inf               1001c850 f   libucrt:87disp.obj
 0001:0001b86d       __rtchsifneg               1001c86d     libucrt:87disp.obj
 0001:0001b880       __twoToTOS                 1001c880 f   libucrt:common.obj
 0001:0001b895       __load_CW                  1001c895 f   libucrt:common.obj
 0001:0001b8ac       __convertTOStoQNaN         1001c8ac f   libucrt:common.obj
 0001:0001b8c5       __fload_withFB             1001c8c5 f   libucrt:common.obj
 0001:0001b908       __checkTOS_withFB          1001c908 f   libucrt:common.obj
 0001:0001b91e       __fast_exit                1001c91e f   libucrt:common.obj
 0001:0001b92b       __math_exit                1001c92b f   libucrt:common.obj
 0001:0001b955       __check_overflow_exit      1001c955 f   libucrt:common.obj
 0001:0001b969       __check_range_exit         1001c969 f   libucrt:common.obj
 0001:0001ba10       __startTwoArgErrorHandling 1001ca10 f   libucrt:genexcep.obj
 0001:0001ba27       __startOneArgErrorHandling 1001ca27 f   libucrt:genexcep.obj
 0001:0001ba63       ___libm_error_support      1001ca63 f   libucrt:libm_error.obj
 0001:0001bc57       __ceil_default             1001cc57 f   libucrt:ceil.obj
 0001:0001bd20       ___ascii_strnicmp          1001cd20 f   libucrt:_strnicm.obj
 0001:0001bd81       ___set_fpsr_sse2           1001cd81 f   libucrt:fpctrl.obj
 0001:0001be01       __clrfp                    1001ce01 f   libucrt:fpctrl.obj
 0001:0001be12       __ctrlfp                   1001ce12 f   libucrt:fpctrl.obj
 0001:0001be3c       __set_statfp               1001ce3c f   libucrt:fpctrl.obj
 0001:0001be95       __statfp                   1001ce95 f   libucrt:fpctrl.obj
 0001:0001bea5       __d_inttype                1001cea5 f   libucrt:powhlp.obj
 0001:0001bf0d       __powhlp                   1001cf0d f   libucrt:powhlp.obj
 0001:0001c038       __87except                 1001d038 f   libucrt:87except.obj
 0001:0001c148       __frnd                     1001d148 f   libucrt:frnd.obj
 0001:0001c15c       __errcode                  1001d15c f   libucrt:fpexcept.obj
 0001:0001c190       __except1                  1001d190 f   libucrt:fpexcept.obj
 0001:0001c25e       __handle_exc               1001d25e f   libucrt:fpexcept.obj
 0001:0001c4de       __raise_exc                1001d4de f   libucrt:fpexcept.obj
 0001:0001c501       __raise_exc_ex             1001d501 f   libucrt:fpexcept.obj
 0001:0001c7f2       __set_errno_from_matherr   1001d7f2 f   libucrt:fpexcept.obj
 0001:0001c823       __umatherr                 1001d823 f   libucrt:fpexcept.obj
 0001:0001c8c3       __decomp                   1001d8c3 f   libucrt:util.obj
 0001:0001c995       __set_exp                  1001d995 f   libucrt:util.obj
 0001:0001c9c2       __sptype                   1001d9c2 f   libucrt:util.obj
 0001:0001ca25       __fpclass                  1001da25 f   libucrt:ieeemisc.obj
 0001:0001cad0       __FindPESection            1001dad0 f   LIBCMT:pesect.obj
 0001:0001cb20       __IsNonwritableInCurrentImage 1001db20 f   LIBCMT:pesect.obj
 0001:0001cbe0       __ValidateImageBase        1001dbe0 f   LIBCMT:pesect.obj
 0001:0001cc11       ??_Etype_info@@UAEPAXI@Z   1001dc11 f i LIBCMT:std_type_info_static.obj
 0001:0001cc11       ??_Gtype_info@@UAEPAXI@Z   1001dc11 f i LIBCMT:std_type_info_static.obj
 0001:0001cc34       __EH_epilog3               1001dc34 f   LIBCMT:ehprolg3.obj
 0001:0001cc48       __EH_prolog3               1001dc48 f   LIBCMT:ehprolg3.obj
 0001:0001cc7b       __EH_prolog3_catch         1001dc7b f   LIBCMT:ehprolg3.obj
 0001:0001ccc0       ??3@YAXPAXI@Z              1001dcc0 f   LIBCMT:delete_scalar_size.obj
 0001:0001ccd0       __allmul                   1001dcd0 f   LIBCMT:llmul.obj
 0001:0001cd10       __aulldiv                  1001dd10 f   LIBCMT:ulldiv.obj
 0001:0001cd80       __aullrem                  1001dd80 f   LIBCMT:ullrem.obj
 0001:0001ce00       __alldiv                   1001de00 f   LIBCMT:lldiv.obj
 0001:0001ceb0       __allshl                   1001deb0 f   LIBCMT:llshl.obj
 0001:0001ced0       __aullshr                  1001ded0 f   LIBCMT:ullshr.obj
 0001:0001cef0       __alloca_probe_16          1001def0 f   LIBCMT:alloca16.obj
 0001:0001cf06       __alloca_probe_8           1001df06     LIBCMT:alloca16.obj
 0001:0001cf20       __alloca_probe             1001df20 f   LIBCMT:chkstk.obj
 0001:0001cf20       __chkstk                   1001df20 f   LIBCMT:chkstk.obj
 0001:0001cf50       __ftol2_sse                1001df50 f   LIBCMT:ftol2.obj
 0001:0001cf60       __ftoi2                    1001df60 f   LIBCMT:ftol2.obj
 0001:0001cfdc       ??3@YAXPAX@Z               1001dfdc f   LIBCMT:delete_scalar.obj
 0001:0001cff0       _strrchr                   1001dff0 f   libvcruntime:strrchr.obj
 0001:0001d127       __filter_x86_sse2_floating_point_exception 1001e127 f   LIBCMT:x86_exception_filter.obj
 0001:0001d127       __filter_x86_sse2_floating_point_exception_default 1001e127 f   LIBCMT:x86_exception_filter.obj
 0002:00000000       __imp__MultiByteToWideChar@24 1001f000     kernel32:KERNEL32.dll
 0002:00000004       __imp__WideCharToMultiByte@32 1001f004     kernel32:KERNEL32.dll
 0002:00000008       __imp__GetACP@0            1001f008     kernel32:KERNEL32.dll
 0002:0000000c       __imp__GetLocaleInfoA@16   1001f00c     kernel32:KERNEL32.dll
 0002:00000010       __imp__GetUserDefaultLCID@0 1001f010     kernel32:KERNEL32.dll
 0002:00000014       __imp__FindClose@4         1001f014     kernel32:KERNEL32.dll
 0002:00000018       __imp__FindFirstFileA@8    1001f018     kernel32:KERNEL32.dll
 0002:0000001c       __imp__GetLastError@0      1001f01c     kernel32:KERNEL32.dll
 0002:00000020       __imp__IsDBCSLeadByte@4    1001f020     kernel32:KERNEL32.dll
 0002:00000024       __imp__UnhandledExceptionFilter@4 1001f024     kernel32:KERNEL32.dll
 0002:00000028       __imp__SetUnhandledExceptionFilter@4 1001f028     kernel32:KERNEL32.dll
 0002:0000002c       __imp__GetCurrentProcess@0 1001f02c     kernel32:KERNEL32.dll
 0002:00000030       __imp__TerminateProcess@8  1001f030     kernel32:KERNEL32.dll
 0002:00000034       __imp__IsProcessorFeaturePresent@4 1001f034     kernel32:KERNEL32.dll
 0002:00000038       __imp__QueryPerformanceCounter@4 1001f038     kernel32:KERNEL32.dll
 0002:0000003c       __imp__GetCurrentProcessId@0 1001f03c     kernel32:KERNEL32.dll
 0002:00000040       __imp__GetCurrentThreadId@0 1001f040     kernel32:KERNEL32.dll
 0002:00000044       __imp__GetSystemTimeAsFileTime@4 1001f044     kernel32:KERNEL32.dll
 0002:00000048       __imp__InitializeSListHead@4 1001f048     kernel32:KERNEL32.dll
 0002:0000004c       __imp__IsDebuggerPresent@0 1001f04c     kernel32:KERNEL32.dll
 0002:00000050       __imp__GetStartupInfoW@4   1001f050     kernel32:KERNEL32.dll
 0002:00000054       __imp__GetModuleHandleW@4  1001f054     kernel32:KERNEL32.dll
 0002:00000058       __imp__WriteConsoleW@20    1001f058     kernel32:KERNEL32.dll
 0002:0000005c       __imp__InterlockedFlushSList@4 1001f05c     kernel32:KERNEL32.dll
 0002:00000060       __imp__RtlUnwind@16        1001f060     kernel32:KERNEL32.dll
 0002:00000064       __imp__SetLastError@4      1001f064     kernel32:KERNEL32.dll
 0002:00000068       __imp__EnterCriticalSection@4 1001f068     kernel32:KERNEL32.dll
 0002:0000006c       __imp__LeaveCriticalSection@4 1001f06c     kernel32:KERNEL32.dll
 0002:00000070       __imp__DeleteCriticalSection@4 1001f070     kernel32:KERNEL32.dll
 0002:00000074       __imp__InitializeCriticalSectionAndSpinCount@8 1001f074     kernel32:KERNEL32.dll
 0002:00000078       __imp__TlsAlloc@0          1001f078     kernel32:KERNEL32.dll
 0002:0000007c       __imp__TlsGetValue@4       1001f07c     kernel32:KERNEL32.dll
 0002:00000080       __imp__TlsSetValue@8       1001f080     kernel32:KERNEL32.dll
 0002:00000084       __imp__TlsFree@4           1001f084     kernel32:KERNEL32.dll
 0002:00000088       __imp__FreeLibrary@4       1001f088     kernel32:KERNEL32.dll
 0002:0000008c       __imp__GetProcAddress@8    1001f08c     kernel32:KERNEL32.dll
 0002:00000090       __imp__LoadLibraryExW@12   1001f090     kernel32:KERNEL32.dll
 0002:00000094       __imp__EncodePointer@4     1001f094     kernel32:KERNEL32.dll
 0002:00000098       __imp__RaiseException@16   1001f098     kernel32:KERNEL32.dll
 0002:0000009c       __imp__GetFullPathNameW@16 1001f09c     kernel32:KERNEL32.dll
 0002:000000a0       __imp__SetFilePointerEx@20 1001f0a0     kernel32:KERNEL32.dll
 0002:000000a4       __imp__ExitProcess@4       1001f0a4     kernel32:KERNEL32.dll
 0002:000000a8       __imp__GetModuleHandleExW@12 1001f0a8     kernel32:KERNEL32.dll
 0002:000000ac       __imp__GetModuleFileNameW@12 1001f0ac     kernel32:KERNEL32.dll
 0002:000000b0       __imp__CloseHandle@4       1001f0b0     kernel32:KERNEL32.dll
 0002:000000b4       __imp__CreateFileW@28      1001f0b4     kernel32:KERNEL32.dll
 0002:000000b8       __imp__GetFileType@4       1001f0b8     kernel32:KERNEL32.dll
 0002:000000bc       __imp__ReadFile@20         1001f0bc     kernel32:KERNEL32.dll
 0002:000000c0       __imp__GetConsoleMode@8    1001f0c0     kernel32:KERNEL32.dll
 0002:000000c4       __imp__ReadConsoleW@20     1001f0c4     kernel32:KERNEL32.dll
 0002:000000c8       __imp__HeapFree@12         1001f0c8     kernel32:KERNEL32.dll
 0002:000000cc       __imp__HeapAlloc@12        1001f0cc     kernel32:KERNEL32.dll
 0002:000000d0       __imp__LCMapStringW@24     1001f0d0     kernel32:KERNEL32.dll
 0002:000000d4       __imp__GetStdHandle@4      1001f0d4     kernel32:KERNEL32.dll
 0002:000000d8       __imp__HeapReAlloc@16      1001f0d8     kernel32:KERNEL32.dll
 0002:000000dc       __imp__GetDriveTypeW@4     1001f0dc     kernel32:KERNEL32.dll
 0002:000000e0       __imp__SetStdHandle@8      1001f0e0     kernel32:KERNEL32.dll
 0002:000000e4       __imp__FindFirstFileExW@24 1001f0e4     kernel32:KERNEL32.dll
 0002:000000e8       __imp__FindNextFileW@8     1001f0e8     kernel32:KERNEL32.dll
 0002:000000ec       __imp__IsValidCodePage@4   1001f0ec     kernel32:KERNEL32.dll
 0002:000000f0       __imp__GetOEMCP@0          1001f0f0     kernel32:KERNEL32.dll
 0002:000000f4       __imp__GetCPInfo@8         1001f0f4     kernel32:KERNEL32.dll
 0002:000000f8       __imp__GetCommandLineA@0   1001f0f8     kernel32:KERNEL32.dll
 0002:000000fc       __imp__GetCommandLineW@0   1001f0fc     kernel32:KERNEL32.dll
 0002:00000100       __imp__GetEnvironmentStringsW@0 1001f100     kernel32:KERNEL32.dll
 0002:00000104       __imp__FreeEnvironmentStringsW@4 1001f104     kernel32:KERNEL32.dll
 0002:00000108       __imp__GetProcessHeap@0    1001f108     kernel32:KERNEL32.dll
 0002:0000010c       __imp__WriteFile@20        1001f10c     kernel32:KERNEL32.dll
 0002:00000110       __imp__GetConsoleOutputCP@0 1001f110     kernel32:KERNEL32.dll
 0002:00000114       __imp__SetEndOfFile@4      1001f114     kernel32:KERNEL32.dll
 0002:00000118       __imp__GetStringTypeW@16   1001f118     kernel32:KERNEL32.dll
 0002:0000011c       __imp__FlushFileBuffers@4  1001f11c     kernel32:KERNEL32.dll
 0002:00000120       __imp__GetFileSizeEx@8     1001f120     kernel32:KERNEL32.dll
 0002:00000124       __imp__GetCurrentDirectoryW@8 1001f124     kernel32:KERNEL32.dll
 0002:00000128       __imp__HeapSize@12         1001f128     kernel32:KERNEL32.dll
 0002:0000012c       __imp__DecodePointer@4     1001f12c     kernel32:KERNEL32.dll
 0002:00000130       \177KERNEL32_NULL_THUNK_DATA 1001f130     kernel32:KERNEL32.dll
 0002:00000134       ___guard_check_icall_fptr  1001f134     LIBCMT:guard_support.obj
 0002:00000138       ___castguard_check_failure_os_handled_fptr 1001f138     LIBCMT:guard_support.obj
 0002:0000013c       ___xc_a                    1001f13c     LIBCMT:initializers.obj
 0002:00000140       ___xc_z                    1001f140     LIBCMT:initializers.obj
 0002:00000144       ___xi_a                    1001f144     LIBCMT:initializers.obj
 0002:00000148       ___acrt_stdio_initializer  1001f148     libucrt:stdio_initializer.obj
 0002:0000014c       ___acrt_multibyte_initializer 1001f14c     libucrt:multibyte_initializer.obj
 0002:00000150       ___acrt_fmode_initializer  1001f150     libucrt:fmode_initializer.obj
 0002:00000154       ___acrt_tran_sse2_initializer 1001f154     libucrt:sse2_initializer.obj
 0002:00000158       ___xi_z                    1001f158     LIBCMT:initializers.obj
 0002:0000015c       ___xp_a                    1001f15c     LIBCMT:initializers.obj
 0002:00000160       ___acrt_locale_terminator  1001f160     libucrt:locale_initializer.obj
 0002:00000164       ___dcrt_console_output_terminator 1001f164     libucrt:console_output_initializer.obj
 0002:00000168       ___acrt_stdio_terminator   1001f168     libucrt:stdio_initializer.obj
 0002:0000016c       ___xp_z                    1001f16c     LIBCMT:initializers.obj
 0002:00000170       ___xt_a                    1001f170     LIBCMT:initializers.obj
 0002:00000174       ___xt_z                    1001f174     LIBCMT:initializers.obj
 0002:00000180       ??_C@_0CK@PECNJIMP@OOM?5error?5in?5native?5tmp?5buffer?5@ 1001f180     FileSystemSupport_md.obj
 0002:000001ac       ??_C@_04LOAJBDKD@true@     1001f1ac     InvocationAdapter.obj
 0002:000001b4       ??_C@_0BF@MPBBPFEA@Can?9Redefine?9Classes@ 1001f1b4     InvocationAdapter.obj
 0002:000001cc       ??_C@_0BI@DOGNCBOD@Can?9Retransform?9Classes@ 1001f1cc     InvocationAdapter.obj
 0002:000001e4       ??_C@_0BN@GGMNHHCI@Can?9Set?9Native?9Method?9Prefix@ 1001f1e4     InvocationAdapter.obj
 0002:00000204       ??_C@_0CD@ONCIGEJ@Can?9Maintain?9Original?9Method?9Or@ 1001f204     InvocationAdapter.obj
 0002:00000228       ??_C@_0CI@HNHEPCMG@?9javaagent?3?5memory?5allocation?5f@ 1001f228     InvocationAdapter.obj
 0002:00000250       ??_C@_0DF@GEAEBGFM@Error?5opening?5zip?5file?5or?5JAR?5m@ 1001f250     InvocationAdapter.obj
 0002:00000288       ??_C@_0O@FJIJHIPN@Premain?9Class@ 1001f288     InvocationAdapter.obj
 0002:00000298       ??_C@_0DH@NNDEJOON@Failed?5to?5find?5Premain?9Class?5ma@ 1001f298     InvocationAdapter.obj
 0002:000002d0       ??_C@_0CM@BAFHELIF@?9javaagent?3?5Premain?9Class?5value@ 1001f2d0     InvocationAdapter.obj
 0002:000002fc       ??_C@_0CG@MGGAPOHH@?9javaagent?3?5memory?5allocation?5f@ 1001f2fc     InvocationAdapter.obj
 0002:00000324       ??_C@_0BA@EEOHCMMC@Boot?9Class?9Path@ 1001f324     InvocationAdapter.obj
 0002:00000334       ??_C@_0DO@FCLCEKPM@java?4lang?4instrument?1?9javaagent@ 1001f334     InvocationAdapter.obj
 0002:00000378       ??_C@_0EJ@MNINEPDM@java?4lang?4instrument?1?9javaagent@ 1001f378     InvocationAdapter.obj
 0002:000003c4       ??_C@_0DG@GEFLELM@java?4lang?4instrument?1?9javaagent@ 1001f3c4     InvocationAdapter.obj
 0002:000003fc       ??_C@_0CI@DPANPEKD@?9javaagent?3?5agent?5class?5not?5spe@ 1001f3fc     InvocationAdapter.obj
 0002:00000424       ??_C@_0DA@KPCNALNC@java?4lang?4instrument?1?9javaagent@ 1001f424     InvocationAdapter.obj
 0002:00000454       ??_C@_0BE@IFOLKMLG@InvocationAdapter?4c@ 1001f454     InvocationAdapter.obj
 0002:00000468       ??_C@_0P@CKGKOICP@result?$DN?$DNJNI_OK@ 1001f468     InvocationAdapter.obj
 0002:00000478       ??_C@_0DE@KGGELLFG@Error?5opening?5zip?5file?5or?5JAR?5m@ 1001f478     InvocationAdapter.obj
 0002:000004ac       ??_C@_0M@HHCNJNFE@Agent?9Class@ 1001f4ac     InvocationAdapter.obj
 0002:000004b8       ??_C@_0DH@DADPHJGN@Failed?5to?5find?5Agent?9Class?5mani@ 1001f4b8     InvocationAdapter.obj
 0002:000004f0       ??_C@_0GG@HGIJBLPF@Unable?5to?5add?5?$CFs?5to?5system?5clas@ 1001f4f0     InvocationAdapter.obj
 0002:00000558       ??_C@_0BO@PHLNGFOC@Agent?9Class?5value?5is?5too?5big?6@ 1001f558     InvocationAdapter.obj
 0002:00000578       ??_C@_07IPNMCAN@success@   1001f578     InvocationAdapter.obj
 0002:00000580       ??_C@_0BI@FNNMMHD@Agent?5failed?5to?5start?$CB?6@ 1001f580     InvocationAdapter.obj
 0002:00000598       ??_C@_0CA@BILEKGHH@processing?5of?5?9javaagent?5failed@ 1001f598     InvocationAdapter.obj
 0002:000005b8       ??_C@_0BJ@CALIJBCB@segments?5?$CB?$DN?5?$CIchar?$CK?$CK?$CJNULL@ 1001f5b8     InvocationAdapter.obj
 0002:000005d4       ??_C@_0BI@GCGOKABC@err?5?$DN?$DN?5JVMTI_ERROR_NONE@ 1001f5d4     InvocationAdapter.obj
 0002:000005f0       ??_C@_0GC@LFNBLJED@System?5class?5loader?5does?5not?5su@ 1001f5f0     InvocationAdapter.obj
 0002:00000658       ??_C@_0EA@GNNEHPOG@Unexpected?5error?5?$CI?$CFd?$CJ?5returned?5@ 1001f658     InvocationAdapter.obj
 0002:00000698       ??_C@_01GBGANLPD@0@        1001f698     InvocationAdapter.obj
 0002:0000069c       ??_C@_0BE@JIIENKGJ@path?5?$CB?$DN?5?$CIchar?$CK?$CJNULL@ 1001f69c     InvocationAdapter.obj
 0002:000006b0       ??_C@_0DJ@KAMKBHCJ@WARNING?3?5illegal?5character?5in?5B@ 1001f6b0     InvocationAdapter.obj
 0002:000006ec       ??_C@_0BL@EGNHKKEM@?$CIvoid?$CK?$CJpath?5?$CB?$DN?5?$CIvoid?$CK?$CJNULL@ 1001f6ec     InvocationAdapter.obj
 0002:00000708       ??_C@_0CE@BMNGMKPL@WARNING?3?5unable?5to?5canonicalize@ 1001f708     InvocationAdapter.obj
 0002:0000072c       ??_C@_0BG@LFGEPDCD@parent?5?$CB?$DN?5?$CIchar?$CK?$CJNULL@ 1001f72c     InvocationAdapter.obj
 0002:00000744       ??_C@_0DJ@BINIAAK@WARNING?3?5?$CFs?5not?5added?5to?5bootst@ 1001f744     InvocationAdapter.obj
 0002:00000780       ??_C@_0CC@HMBHOALF@Illegal?5argument?5or?5not?5JAR?5fil@ 1001f780     InvocationAdapter.obj
 0002:000007a4       ??_C@_0BG@IPMFCDFJ@Unexpected?5error?3?5?$CFd?6@ 1001f7a4     InvocationAdapter.obj
 0002:000007bc       ??_C@_0N@PDEDENJF@JPLISAgent?4c@ 1001f7bc     JPLISAgent.obj
 0002:000007cc       ??_C@_0BP@JFPONFCF@jvmtierror?5?$DN?$DN?5JVMTI_ERROR_NONE@ 1001f7cc     JPLISAgent.obj
 0002:000007ec       ??_C@_0BE@JEGDIMFH@environment?5?$CB?$DN?5NULL@ 1001f7ec     JPLISAgent.obj
 0002:00000800       ??_C@_0CD@EAGMGAOH@environment?9?$DOmJVMTIEnv?5?$DN?$DN?5jvmti@ 1001f800     JPLISAgent.obj
 0002:00000824       ??_C@_06KJFADLGN@result@   1001f824     JPLISAgent.obj
 0002:0000082c       ??_C@_0CD@FJABNFOF@sun?1instrument?1InstrumentationI@ 1001f82c     JPLISAgent.obj
 0002:00000850       ??_C@_0CJ@HOIGMIGF@find?5class?5on?5InstrumentationIm@ 1001f850     JPLISAgent.obj
 0002:0000087c       ??_C@_0BC@NFAEECCL@?$CBerrorOutstanding@ 1001f87c     JPLISAgent.obj
 0002:00000890       ??_C@_06DNGMMBGB@?$CIJZZ?$CJV@ 1001f890     JPLISAgent.obj
 0002:00000898       ??_C@_06FALKBLGB@?$DMinit?$DO@ 1001f898     JPLISAgent.obj
 0002:000008a0       ??_C@_0CP@DNJEEBBF@find?5constructor?5on?5Instrumenta@ 1001f8a0     JPLISAgent.obj
 0002:000008d0       ??_C@_0CP@HELLCCDH@call?5constructor?5on?5Instrumenta@ 1001f8d0     JPLISAgent.obj
 0002:00000900       ??_C@_0BN@KICHEFJM@copy?5local?5ref?5to?5global?5ref@ 1001f900     JPLISAgent.obj
 0002:00000920       ??_C@_0CI@HEGLGDKJ@?$CILjava?1lang?1String?$DLLjava?1lang?1S@ 1001f920     JPLISAgent.obj
 0002:00000948       ??_C@_0BI@MHLLCGNO@loadClassAndCallPremain@ 1001f948     JPLISAgent.obj
 0002:00000960       ??_C@_0CE@KECKFJKE@can?8t?5find?5premain?5invoker?5meth@ 1001f960     JPLISAgent.obj
 0002:00000984       ??_C@_0BK@JAOFMOJK@loadClassAndCallAgentmain@ 1001f984     JPLISAgent.obj
 0002:000009a0       ??_C@_0CG@DOGNAPEF@can?8t?5find?5agentmain?5invoker?5me@ 1001f9a0     JPLISAgent.obj
 0002:000009c8       ??_C@_0GC@CPEKEAKP@?$CILjava?1lang?1ClassLoader?$DLLjava?1l@ 1001f9c8     JPLISAgent.obj
 0002:00000a2c       ??_C@_09IFONHNKG@transform@ 1001fa2c     JPLISAgent.obj
 0002:00000a38       ??_C@_0BO@LKBEMJID@can?8t?5find?5transform?5methodID@ 1001fa38     JPLISAgent.obj
 0002:00000a58       ??_C@_0CE@NNNMFAHP@can?8t?5create?5class?5name?5java?5st@ 1001fa58     JPLISAgent.obj
 0002:00000a7c       ??_C@_0CB@GCBHBCEC@can?8t?5create?5options?5java?5strin@ 1001fa7c     JPLISAgent.obj
 0002:00000aa0       ??_C@_0BK@OLJIPBJG@mainCallingMethod?5?$CB?$DN?5NULL@ 1001faa0     JPLISAgent.obj
 0002:00000ac0       ??_C@_0EK@NBNNLAGF@jvmtierror?5?$DN?$DN?5JVMTI_ERROR_NONE?5@ 1001fac0     JPLISAgent.obj
 0002:00000b0c       ??_C@_0BJ@OFPEOMG@can?8t?5create?5name?5string@ 1001fb0c     JPLISAgent.obj
 0002:00000b28       ??_C@_0BI@PGLGLBA@can?8t?5create?5byte?5arrau@ 1001fb28     JPLISAgent.obj
 0002:00000b40       ??_C@_0BM@NODFBCMB@can?8t?5set?5byte?5array?5region@ 1001fb40     JPLISAgent.obj
 0002:00000b5c       ??_C@_0CE@NCFBINFF@agent?9?$DOmInstrumentationImpl?5?$CB?$DN?5@ 1001fb5c     JPLISAgent.obj
 0002:00000b80       ??_C@_0BK@GEFGBHIE@agent?9?$DOmTransform?5?$CB?$DN?5NULL@ 1001fb80     JPLISAgent.obj
 0002:00000b9c       ??_C@_0BN@JDJGIEH@transform?5method?5call?5failed@ 1001fb9c     JPLISAgent.obj
 0002:00000bbc       ??_C@_0BH@DDPAAIBF@can?8t?5get?5array?5length@ 1001fbbc     JPLISAgent.obj
 0002:00000bd4       ??_C@_0BN@KNPJDEBO@can?8t?5allocate?5result?5buffer@ 1001fbd4     JPLISAgent.obj
 0002:00000bf4       ??_C@_0BM@CLGDMLIA@can?8t?5get?5byte?5array?5region@ 1001fbf4     JPLISAgent.obj
 0002:00000c10       ??_C@_0BK@JCFBFKNG@isSafeForJNICalls?$CIjnienv?$CJ@ 1001fc10     JPLISAgent.obj
 0002:00000c2c       ??_C@_0CF@PBJJFPHF@?$CBisUnchecked?$CIjnienv?0?5throwableT@ 1001fc2c     JPLISAgent.obj
 0002:00000c54       ??_C@_0CB@KCPANAMN@java?1lang?1ClassNotFoundExceptio@ 1001fc54     JPLISAgent.obj
 0002:00000c78       ??_C@_0DA@MJOAEAPC@java?1lang?1instrument?1Unmodifiab@ 1001fc78     JPLISAgent.obj
 0002:00000ca8       ??_C@_0BA@JJLOPNCP@java?1lang?1Class@ 1001fca8     JPLISAgent.obj
 0002:00000cb8       ??_C@_0BO@GBLMHFAI@FindClass?5returned?5null?5class@ 1001fcb8     JPLISAgent.obj
 0002:00000cd8       ??_C@_0BI@JLMJJPLE@classArrayClass?5?$CB?$DN?5NULL@ 1001fcd8     JPLISAgent.obj
 0002:00000cf0       ??_C@_0CD@NMCFBNHK@NewObjectArray?5returned?5null?5ar@ 1001fcf0     JPLISAgent.obj
 0002:00000d14       ??_C@_0BD@BNJLEHDL@localArray?5?$CB?$DN?5NULL@ 1001fd14     JPLISAgent.obj
 0002:00000d28       ??_C@_0CI@MJAJKCDF@jvmtierror?5?$DN?$DN?5JVMTI_ERROR_NOT_A@ 1001fd28     JPLISAgent.obj
 0002:00000d50       ??_C@_0BJ@EJCHPAPK@retransformerEnv?5?$CB?$DN?5NULL@ 1001fd50     JPLISAgent.obj
 0002:00000d6c       ??_C@_0BA@DKKKAEPC@classes?5?$CB?$DN?5NULL@ 1001fd6c     JPLISAgent.obj
 0002:00000d7c       ??_C@_0P@IBHCMEIB@?$CBerrorOccurred@ 1001fd7c     JPLISAgent.obj
 0002:00000d8c       ??_C@_0BA@DHKCDHMI@numClasses?5?$CB?$DN?50@ 1001fd8c     JPLISAgent.obj
 0002:00000d9c       ??_C@_0BK@HBLAKIEB@classArray?$FLindex?$FN?5?$CB?$DN?5NULL@ 1001fd9c     JPLISAgent.obj
 0002:00000db8       ??_C@_0BJ@NGKAGHPG@classDefinitions?5?$CB?$DN?5NULL@ 1001fdb8     JPLISAgent.obj
 0002:00000dd4       ??_C@_0M@KGLONNBG@numDefs?5?$DO?50@ 1001fdd4     JPLISAgent.obj
 0002:00000de0       ??_C@_0CF@BGAIILOJ@java?1lang?1instrument?1ClassDefin@ 1001fde0     JPLISAgent.obj
 0002:00000e08       ??_C@_0BE@IIFEGCLG@?$CI?$CJLjava?1lang?1Class?$DL@ 1001fe08     JPLISAgent.obj
 0002:00000e1c       ??_C@_0BD@FFKMDMBN@getDefinitionClass@ 1001fe1c     JPLISAgent.obj
 0002:00000e30       ??_C@_04LHPAGAEF@?$CI?$CJ?$FLB@ 1001fe30     JPLISAgent.obj
 0002:00000e38       ??_C@_0BH@FOGLHNOO@getDefinitionClassFile@ 1001fe38     JPLISAgent.obj
 0002:00000e50       ??_C@_0BE@NLJNCPBN@prefixArray?5?$CB?$DN?5NULL@ 1001fe50     JPLISAgent.obj
 0002:00000e68       ??_C@_0EE@FPMMKFJK@?$CK?$CK?$CK?5java?4lang?4instrument?5ASSERT@ 1001fe68     JPLISAssert.obj
 0002:00000eb0       ??_C@_0FE@HCMNEDKA@?$CK?$CK?$CK?5java?4lang?4instrument?5ASSERT@ 1001feb0     JPLISAssert.obj
 0002:00000f04       ??_C@_0BB@JLIFFPJB@JavaExceptions?4c@ 1001ff04     JavaExceptions.obj
 0002:00000f18       ??_C@_0BH@EKGMOCH@throwableToMap?5?$CB?$DN?5NULL@ 1001ff18     JavaExceptions.obj
 0002:00000f30       ??_C@_0BC@HKCJMFCP@className?5?$CB?$DN?5NULL@ 1001ff30     JavaExceptions.obj
 0002:00000f44       ??_C@_0BG@IKDDPPGD@?$CILjava?1lang?1String?$DL?$CJV@ 1001ff44     JavaExceptions.obj
 0002:00000f5c       ??_C@_0BI@NBLNIHIB@java?1lang?1InternalError@ 1001ff5c     JavaExceptions.obj
 0002:00000f74       ??_C@_0BP@GJLHLAKJ@java?1lang?1NullPointerException@ 1001ff74     JavaExceptions.obj
 0002:00000f94       ??_C@_0CD@MOHADDFA@java?1lang?1IllegalArgumentExcept@ 1001ff94     JavaExceptions.obj
 0002:00000fb8       ??_C@_0BL@ENCPOIKC@java?1lang?1OutOfMemoryError@ 1001ffb8     JavaExceptions.obj
 0002:00000fd4       ??_C@_0CA@OCDKFHGJ@java?1lang?1ClassCircularityError@ 1001ffd4     JavaExceptions.obj
 0002:00000ff4       ??_C@_0BG@FNCILCAN@java?1lang?1VerifyError@ 1001fff4     JavaExceptions.obj
 0002:0000100c       ??_C@_0CI@LDDEGNGM@java?1lang?1UnsupportedOperationE@ 1002000c     JavaExceptions.obj
 0002:00001034       ??_C@_0DF@IFGMNJBO@class?5redefinition?5failed?3?5atte@ 10020034     JavaExceptions.obj
 0002:00001070       ??_C@_0EO@LOHFEPOO@class?5redefinition?5failed?3?5atte@ 10020070     JavaExceptions.obj
 0002:000010c0       ??_C@_0EI@PJGIIEAK@class?5redefinition?5failed?3?5atte@ 100200c0     JavaExceptions.obj
 0002:00001108       ??_C@_0DI@KJLEIONK@class?5redefinition?5failed?3?5atte@ 10020108     JavaExceptions.obj
 0002:00001140       ??_C@_0ED@PPHPPFFE@class?5redefinition?5failed?3?5atte@ 10020140     JavaExceptions.obj
 0002:00001188       ??_C@_0EA@INKOHMMN@class?5redefinition?5failed?3?5atte@ 10020188     JavaExceptions.obj
 0002:000011c8       ??_C@_0CH@DNCLOIOF@java?1lang?1UnsupportedClassVersi@ 100201c8     JavaExceptions.obj
 0002:000011f0       ??_C@_0BP@NAHGIHIH@java?1lang?1NoClassDefFoundError@ 100201f0     JavaExceptions.obj
 0002:00001210       ??_C@_0BI@MAPDCENK@class?5names?5don?8t?5match@ 10020210     JavaExceptions.obj
 0002:00001228       ??_C@_0BL@EEAIAIEG@java?1lang?1ClassFormatError@ 10020228     JavaExceptions.obj
 0002:00001244       ??_C@_0CJ@DNCKJBBE@class?5redefinition?5failed?3?5inva@ 10020244     JavaExceptions.obj
 0002:00001270       ??_C@_0BG@JKFIFBMN@unsupported?5operation@ 10020270     JavaExceptions.obj
 0002:00001288       ??_C@_0CD@LAOKENHO@can?8t?5create?5exception?5java?5str@ 10020288     JavaExceptions.obj
 0002:000012ac       ??_C@_0BF@FOHFOJOB@?$CI?$CJLjava?1lang?1String?$DL@ 100202ac     JavaExceptions.obj
 0002:000012c4       ??_C@_08JCDFGHAO@toString@ 100202c4     JavaExceptions.obj
 0002:000012d0       ??_C@_0BA@NOLMKEPF@java?1lang?1Error@ 100202d0     JavaExceptions.obj
 0002:000012e0       ??_C@_0BL@IONOAEOO@java?1lang?1RuntimeException@ 100202e0     JavaExceptions.obj
 0002:000012fc       ??_C@_0CC@GKBBLNKJ@throwThrowable?5failed?5to?5re?9thr@ 100202fc     JavaExceptions.obj
 0002:00001320       ??_C@_0BB@EJBOEPOM@result?5?$DN?$DN?5JNI_OK@ 10020320     JavaExceptions.obj
 0002:00001334       ??_C@_09HLKPJHCC@?9_?4?$CB?$HO?$CK?8?$CI?$CJ@ 10020334     PathCharsValidator.obj
 0002:00001340       ??_C@_07DDNJCNOL@?3?$EA?$CG?$DN?$CL$?0@ 10020340     PathCharsValidator.obj
 0002:00001348       ??_C@_02DKJMBEPB@?$DL?1@   10020348     PathCharsValidator.obj
 0002:0000134c       ??_C@_0N@CPKCLCKM@Reentrancy?4c@ 1002034c     Reentrancy.obj
 0002:0000135c       ??_C@_0BK@PPCACBKK@error?5?$DN?$DN?5JVMTI_ERROR_NONE@ 1002035c     Reentrancy.obj
 0002:00001378       ??_C@_0BB@LLFPNPAC@test?5?$DN?$DN?5expected@ 10020378     Reentrancy.obj
 0002:0000138c       ??_C@_0M@FFIPNNAM@Utilities?4c@ 1002038c     Utilities.obj
 0002:00001398       ??_C@_0BI@NNKHJJFO@Can?8t?5deallocate?5memory@ 10020398     Utilities.obj
 0002:000013b0       ??_C@_0BF@LACNODFI@META?9INF?1MANIFEST?4MF@ 100203b0     jli_static:parse_manifest.obj
 0002:000013c8       ??_C@_05OJPKCACG@1?43?41@  100203c8     jli_static:parse_manifest.obj
 0002:000013d0       ??_C@_02LIIHNNHG@?6?$AN@   100203d0     jli_static:parse_manifest.obj
 0002:00001c80       ??_C@_0BH@LIBMMIGA@incorrect?5header?5check@ 10020c80     jli_static:inflate.obj
 0002:00001c98       ??_C@_0BL@IHKGDAEE@unknown?5compression?5method@ 10020c98     jli_static:inflate.obj
 0002:00001cb4       ??_C@_0BE@EMOGCLGO@invalid?5window?5size@ 10020cb4     jli_static:inflate.obj
 0002:00001cc8       ??_C@_0BJ@BLBBCOMO@unknown?5header?5flags?5set@ 10020cc8     jli_static:inflate.obj
 0002:00001ce4       ??_C@_0BE@GONKLEPM@header?5crc?5mismatch@ 10020ce4     jli_static:inflate.obj
 0002:00001cf8       ??_C@_0BD@PJCBIDD@invalid?5block?5type@ 10020cf8     jli_static:inflate.obj
 0002:00001d0c       ??_C@_0BN@LGAADGOK@invalid?5stored?5block?5lengths@ 10020d0c     jli_static:inflate.obj
 0002:00001d2c       ??_C@_0CE@GMIGFPBB@too?5many?5length?5or?5distance?5sym@ 10020d2c     jli_static:inflate.obj
 0002:00001d50       ??_C@_0BJ@HDEPPGOH@invalid?5code?5lengths?5set@ 10020d50     jli_static:inflate.obj
 0002:00001d6c       ??_C@_0BK@BMMPFBBH@invalid?5bit?5length?5repeat@ 10020d6c     jli_static:inflate.obj
 0002:00001d88       ??_C@_0CF@DGDMADCD@invalid?5code?5?9?9?5missing?5end?9of?9@ 10020d88     jli_static:inflate.obj
 0002:00001db0       ??_C@_0BM@IIMGAINC@invalid?5literal?1lengths?5set@ 10020db0     jli_static:inflate.obj
 0002:00001dcc       ??_C@_0BG@GMDFCBGP@invalid?5distances?5set@ 10020dcc     jli_static:inflate.obj
 0002:00001de4       ??_C@_0BM@FFFLPBBC@invalid?5literal?1length?5code@ 10020de4     jli_static:inflate.obj
 0002:00001e00       ??_C@_0BG@LBKINIKP@invalid?5distance?5code@ 10020e00     jli_static:inflate.obj
 0002:00001e18       ??_C@_0BO@ECPMAOGG@invalid?5distance?5too?5far?5back@ 10020e18     jli_static:inflate.obj
 0002:00001e38       ??_C@_0BF@MEIGEHBE@incorrect?5data?5check@ 10020e38     jli_static:inflate.obj
 0002:00001e50       ??_C@_0BH@FGKKJGOC@incorrect?5length?5check@ 10020e50     jli_static:inflate.obj
 0002:000046e8       _z_errmsg                  100236e8     jli_static:zutil.obj
 0002:00004710       ??_C@_0BA@MOKMMFOD@need?5dictionary@ 10023710     jli_static:zutil.obj
 0002:00004720       ??_C@_0L@FNAOCBOG@stream?5end@ 10023720     jli_static:zutil.obj
 0002:0000472b       ??_C@_00CNPNBAHC@@         1002372b     jli_static:zutil.obj
 0002:0000472c       ??_C@_0L@KIJFAKBJ@file?5error@ 1002372c     jli_static:zutil.obj
 0002:00004738       ??_C@_0N@MKKNPMJD@stream?5error@ 10023738     jli_static:zutil.obj
 0002:00004748       ??_C@_0L@HAHMBNLP@data?5error@ 10023748     jli_static:zutil.obj
 0002:00004754       ??_C@_0BE@OGGJBMCE@insufficient?5memory@ 10023754     jli_static:zutil.obj
 0002:00004768       ??_C@_0N@DFPGLBGC@buffer?5error@ 10023768     jli_static:zutil.obj
 0002:00004778       ??_C@_0BF@CJFPCCEG@incompatible?5version@ 10023778     jli_static:zutil.obj
 0002:00004790       _inflate_copyright         10023790     jli_static:inftrees.obj
 0002:000048c0       __pDefaultRawDllMain       100238c0     LIBCMT:dll_dllmain.obj
 0002:000048c0       __pRawDllMain              100238c0     LIBCMT:dll_dllmain.obj
 0002:000048cc       __pDestructExceptionObject 100238cc     libvcruntime:ehhelpers.obj
 0002:00004c58       ??_C@_08EHJDFFNH@__based?$CI@ 10023c58     libvcruntime:undname.obj
 0002:00004c64       ??_C@_07KOLFKCDI@__cdecl@  10023c64     libvcruntime:undname.obj
 0002:00004c6c       ??_C@_08GHMPAG@__pascal@   10023c6c     libvcruntime:undname.obj
 0002:00004c78       ??_C@_09IFJBGAPI@__stdcall@ 10023c78     libvcruntime:undname.obj
 0002:00004c84       ??_C@_0L@NPHFGOKO@__thiscall@ 10023c84     libvcruntime:undname.obj
 0002:00004c90       ??_C@_0L@JMKHOMEK@__fastcall@ 10023c90     libvcruntime:undname.obj
 0002:00004c9c       ??_C@_0N@BCKKPABJ@__vectorcall@ 10023c9c     libvcruntime:undname.obj
 0002:00004cac       ??_C@_09HIJEGCPM@__clrcall@ 10023cac     libvcruntime:undname.obj
 0002:00004cb8       ??_C@_06GHPCKEAG@__eabi@   10023cb8     libvcruntime:undname.obj
 0002:00004cc0       ??_C@_09IOPIDJLG@__swift_1@ 10023cc0     libvcruntime:undname.obj
 0002:00004ccc       ??_C@_09KFNFGKHF@__swift_2@ 10023ccc     libvcruntime:undname.obj
 0002:00004cd8       ??_C@_09LMMOFLDE@__swift_3@ 10023cd8     libvcruntime:undname.obj
 0002:00004ce4       ??_C@_07JOMMBBKO@__ptr64@  10023ce4     libvcruntime:undname.obj
 0002:00004cec       ??_C@_0L@PILCLIHE@__restrict@ 10023cec     libvcruntime:undname.obj
 0002:00004cf8       ??_C@_0M@GFIIJFMG@__unaligned@ 10023cf8     libvcruntime:undname.obj
 0002:00004d04       ??_C@_09DHDLOLLB@restrict?$CI@ 10023d04     libvcruntime:undname.obj
 0002:00004d10       ??_C@_04NIHEBCM@?5new@     10023d10     libvcruntime:undname.obj
 0002:00004d18       ??_C@_07FPCDHGMM@?5delete@ 10023d18     libvcruntime:undname.obj
 0002:00004d20       ??_C@_01NEMOKFLO@?$DN@     10023d20     libvcruntime:undname.obj
 0002:00004d24       ??_C@_02GPIOPFAK@?$DO?$DO@ 10023d24     libvcruntime:undname.obj
 0002:00004d28       ??_C@_02FODMEDOG@?$DM?$DM@ 10023d28     libvcruntime:undname.obj
 0002:00004d2c       ??_C@_01DCLJPIOD@?$CB@     10023d2c     libvcruntime:undname.obj
 0002:00004d30       ??_C@_02EGOFBIJA@?$DN?$DN@ 10023d30     libvcruntime:undname.obj
 0002:00004d34       ??_C@_02FDNJECIE@?$CB?$DN@ 10023d34     libvcruntime:undname.obj
 0002:00004d38       ??_C@_02GPECMEKF@?$FL?$FN@ 10023d38     libvcruntime:undname.obj
 0002:00004d3c       ??_C@_08LHJFAFGD@operator@ 10023d3c     libvcruntime:undname.obj
 0002:00004d48       ??_C@_02HBOOOICD@?9?$DO@   10023d48     libvcruntime:undname.obj
 0002:00004d4c       ??_C@_01NBENCBCI@?$CK@     10023d4c     libvcruntime:undname.obj
 0002:00004d50       ??_C@_02ECNGHCIF@?$CL?$CL@ 10023d50     libvcruntime:undname.obj
 0002:00004d54       ??_C@_02BAABKJLB@?9?9@     10023d54     libvcruntime:undname.obj
 0002:00004d58       ??_C@_01JOAMLHOP@?9@       10023d58     libvcruntime:undname.obj
 0002:00004d5c       ??_C@_01MIFGBAGJ@?$CL@     10023d5c     libvcruntime:undname.obj
 0002:00004d60       ??_C@_01HNPIGOCE@?$CG@     10023d60     libvcruntime:undname.obj
 0002:00004d64       ??_C@_03MNHNFDLC@?9?$DO?$CK@ 10023d64     libvcruntime:undname.obj
 0002:00004d68       ??_C@_01KMDKNFGN@?1@       10023d68     libvcruntime:undname.obj
 0002:00004d6c       ??_C@_01FGNFDNOH@?$CF@     10023d6c     libvcruntime:undname.obj
 0002:00004d70       ??_C@_01MNNFJEPP@?$DM@     10023d70     libvcruntime:undname.obj
 0002:00004d74       ??_C@_02EHCHHCKH@?$DM?$DN@ 10023d74     libvcruntime:undname.obj
 0002:00004d78       ??_C@_01PPODPGHN@?$DO@     10023d78     libvcruntime:undname.obj
 0002:00004d7c       ??_C@_02EEKDKGMJ@?$DO?$DN@ 10023d7c     libvcruntime:undname.obj
 0002:00004d80       ??_C@_01IHBHIGKO@?0@       10023d80     libvcruntime:undname.obj
 0002:00004d84       ??_C@_02HCKGKOFO@?$CI?$CJ@ 10023d84     libvcruntime:undname.obj
 0002:00004d88       ??_C@_01PJKLJHI@?$HO@      10023d88     libvcruntime:undname.obj
 0002:00004d8c       ??_C@_01JKBOJNNK@?$FO@     10023d8c     libvcruntime:undname.obj
 0002:00004d90       ??_C@_01DNKMNLPK@?$HM@     10023d90     libvcruntime:undname.obj
 0002:00004d94       ??_C@_02PPKAJPJL@?$CG?$CG@ 10023d94     libvcruntime:undname.obj
 0002:00004d98       ??_C@_02NONPIBCD@?$HM?$HM@ 10023d98     libvcruntime:undname.obj
 0002:00004d9c       ??_C@_02FPIMKNGF@?$CK?$DN@ 10023d9c     libvcruntime:undname.obj
 0002:00004da0       ??_C@_02FOEOMHFC@?$CL?$DN@ 10023da0     libvcruntime:undname.obj
 0002:00004da4       ??_C@_02FKMDLLOA@?9?$DN@   10023da4     libvcruntime:undname.obj
 0002:00004da8       ??_C@_02FJEHGPIO@?1?$DN@   10023da8     libvcruntime:undname.obj
 0002:00004dac       ??_C@_02FENAOKFI@?$CF?$DN@ 10023dac     libvcruntime:undname.obj
 0002:00004db0       ??_C@_03IKFCCPFF@?$DO?$DO?$DN@ 10023db0     libvcruntime:undname.obj
 0002:00004db4       ??_C@_03CDNPDDLA@?$DM?$DM?$DN@ 10023db4     libvcruntime:undname.obj
 0002:00004db8       ??_C@_02FGJGFEAB@?$CG?$DN@ 10023db8     libvcruntime:undname.obj
 0002:00004dbc       ??_C@_02DHLNPPGH@?$HM?$DN@ 10023dbc     libvcruntime:undname.obj
 0002:00004dc0       ??_C@_02MHEGNOJ@?$FO?$DN@  10023dc0     libvcruntime:undname.obj
 0002:00004dc4       ??_C@_09IFPLHPGF@?$GAvftable?8@ 10023dc4     libvcruntime:undname.obj
 0002:00004dd0       ??_C@_09BLBHBJP@?$GAvbtable?8@ 10023dd0     libvcruntime:undname.obj
 0002:00004ddc       ??_C@_07FEEIOKP@?$GAvcall?8@ 10023ddc     libvcruntime:undname.obj
 0002:00004de4       ??_C@_08LLFFHHDJ@?$GAtypeof?8@ 10023de4     libvcruntime:undname.obj
 0002:00004df0       ??_C@_0BF@KDPPACIK@?$GAlocal?5static?5guard?8@ 10023df0     libvcruntime:undname.obj
 0002:00004e08       ??_C@_08OBABFOLI@?$GAstring?8@ 10023e08     libvcruntime:undname.obj
 0002:00004e14       ??_C@_0BD@JDLKDPAB@?$GAvbase?5destructor?8@ 10023e14     libvcruntime:undname.obj
 0002:00004e28       ??_C@_0BN@DEGPLNFK@?$GAvector?5deleting?5destructor?8@ 10023e28     libvcruntime:undname.obj
 0002:00004e48       ??_C@_0BO@OBMKPJIG@?$GAdefault?5constructor?5closure?8@ 10023e48     libvcruntime:undname.obj
 0002:00004e68       ??_C@_0BN@IMDCHIKM@?$GAscalar?5deleting?5destructor?8@ 10023e68     libvcruntime:undname.obj
 0002:00004e88       ??_C@_0BO@PFGOCPJJ@?$GAvector?5constructor?5iterator?8@ 10023e88     libvcruntime:undname.obj
 0002:00004ea8       ??_C@_0BN@LFPFMEDL@?$GAvector?5destructor?5iterator?8@ 10023ea8     libvcruntime:undname.obj
 0002:00004ec8       ??_C@_0CE@IKBNEHA@?$GAvector?5vbase?5constructor?5itera@ 10023ec8     libvcruntime:undname.obj
 0002:00004eec       ??_C@_0BL@NILFHHPC@?$GAvirtual?5displacement?5map?8@ 10023eec     libvcruntime:undname.obj
 0002:00004f08       ??_C@_0CB@JONCMFFK@?$GAeh?5vector?5constructor?5iterator@ 10023f08     libvcruntime:undname.obj
 0002:00004f2c       ??_C@_0CA@GCEOPDGL@?$GAeh?5vector?5destructor?5iterator?8@ 10023f2c     libvcruntime:undname.obj
 0002:00004f4c       ??_C@_0CH@OOJPLCPH@?$GAeh?5vector?5vbase?5constructor?5it@ 10023f4c     libvcruntime:undname.obj
 0002:00004f74       ??_C@_0BL@LLKPOHJI@?$GAcopy?5constructor?5closure?8@ 10023f74     libvcruntime:undname.obj
 0002:00004f90       ??_C@_0BA@KBCDOMBN@?$GAudt?5returning?8@ 10023f90     libvcruntime:undname.obj
 0002:00004fa0       ??_C@_03KLGMFNMG@?$GAEH@   10023fa0     libvcruntime:undname.obj
 0002:00004fa4       ??_C@_05KHLCHHI@?$GARTTI@  10023fa4     libvcruntime:undname.obj
 0002:00004fac       ??_C@_0BA@KKLDJDLB@?$GAlocal?5vftable?8@ 10023fac     libvcruntime:undname.obj
 0002:00004fbc       ??_C@_0CE@IIHCMGGL@?$GAlocal?5vftable?5constructor?5clos@ 10023fbc     libvcruntime:undname.obj
 0002:00004fe0       ??_C@_06FHBGPFGH@?5new?$FL?$FN@ 10023fe0     libvcruntime:undname.obj
 0002:00004fe8       ??_C@_09LBNFPBCA@?5delete?$FL?$FN@ 10023fe8     libvcruntime:undname.obj
 0002:00004ff4       ??_C@_0P@HJKNJFNN@?$GAomni?5callsig?8@ 10023ff4     libvcruntime:undname.obj
 0002:00005004       ??_C@_0BL@CNOONJFP@?$GAplacement?5delete?5closure?8@ 10024004     libvcruntime:undname.obj
 0002:00005020       ??_C@_0BN@CKNJLHMB@?$GAplacement?5delete?$FL?$FN?5closure?8@ 10024020     libvcruntime:undname.obj
 0002:00005040       ??_C@_0CG@CFDHKGGD@?$GAmanaged?5vector?5constructor?5ite@ 10024040     libvcruntime:undname.obj
 0002:00005068       ??_C@_0CF@IMGKMJNO@?$GAmanaged?5vector?5destructor?5iter@ 10024068     libvcruntime:undname.obj
 0002:00005090       ??_C@_0CG@HLDDJMAG@?$GAeh?5vector?5copy?5constructor?5ite@ 10024090     libvcruntime:undname.obj
 0002:000050b8       ??_C@_0CM@FCBBDIGB@?$GAeh?5vector?5vbase?5copy?5construct@ 100240b8     libvcruntime:undname.obj
 0002:000050e4       ??_C@_0BL@CLIPGLGB@?$GAdynamic?5initializer?5for?5?8@ 100240e4     libvcruntime:undname.obj
 0002:00005100       ??_C@_0CB@PDBIFEP@?$GAdynamic?5atexit?5destructor?5for?5@ 10024100     libvcruntime:undname.obj
 0002:00005124       ??_C@_0CD@CGAJBKEJ@?$GAvector?5copy?5constructor?5iterat@ 10024124     libvcruntime:undname.obj
 0002:00005148       ??_C@_0CJ@GJELGAMM@?$GAvector?5vbase?5copy?5constructor?5@ 10024148     libvcruntime:undname.obj
 0002:00005174       ??_C@_0CL@FGIJHLCE@?$GAmanaged?5vector?5copy?5constructo@ 10024174     libvcruntime:undname.obj
 0002:000051a0       ??_C@_0BM@PMGGMLDN@?$GAlocal?5static?5thread?5guard?8@ 100241a0     libvcruntime:undname.obj
 0002:000051bc       ??_C@_0N@BDNMDMOL@operator?5?$CC?$CC?5@ 100241bc     libvcruntime:undname.obj
 0002:000051cc       ??_C@_0BC@GGEBGALA@operator?5co_await@ 100241cc     libvcruntime:undname.obj
 0002:000051e0       ??_C@_0M@GAAIMMOH@operator?$DM?$DN?$DO@ 100241e0     libvcruntime:undname.obj
 0002:000051ec       ??_C@_0BC@DAFEJGAK@?5Type?5Descriptor?8@ 100241ec     libvcruntime:undname.obj
 0002:00005200       ??_C@_0BM@LDKODKLH@?5Base?5Class?5Descriptor?5at?5?$CI@ 10024200     libvcruntime:undname.obj
 0002:0000521c       ??_C@_0BD@LGICGFMM@?5Base?5Class?5Array?8@ 1002421c     libvcruntime:undname.obj
 0002:00005230       ??_C@_0BN@MECKDCOJ@?5Class?5Hierarchy?5Descriptor?8@ 10024230     libvcruntime:undname.obj
 0002:00005250       ??_C@_0BK@CFCOFLF@?5Complete?5Object?5Locator?8@ 10024250     libvcruntime:undname.obj
 0002:0000526c       ??_C@_0BG@JNJLAMPM@?$GAanonymous?5namespace?8@ 1002426c     libvcruntime:undname.obj
 0002:00005290       ??_C@_1DM@KHCHBNEB@?$AAa?$AAp?$AAi?$AA?9?$AAm?$AAs?$AA?9?$AAw?$AAi?$AAn?$AA?9?$AAc?$AAo?$AAr?$AAe@ 10024290     libvcruntime:winapi_downlevel.obj
 0002:000052cc       ??_C@_1DK@LPPGFMPP@?$AAa?$AAp?$AAi?$AA?9?$AAm?$AAs?$AA?9?$AAw?$AAi?$AAn?$AA?9?$AAc?$AAo?$AAr?$AAe@ 100242cc     libvcruntime:winapi_downlevel.obj
 0002:00005308       ??_C@_1BC@GDMECMAK@?$AAk?$AAe?$AAr?$AAn?$AAe?$AAl?$AA3?$AA2@ 10024308     libvcruntime:winapi_downlevel.obj
 0002:0000531c       ??_C@_1BA@PFFKHIOG@?$AAa?$AAp?$AAi?$AA?9?$AAm?$AAs?$AA?9@ 1002431c     libvcruntime:winapi_downlevel.obj
 0002:00005334       ??_C@_08KNHFBNJ@FlsAlloc@  10024334     libvcruntime:winapi_downlevel.obj
 0002:00005348       ??_C@_07PEJMOBNF@FlsFree@  10024348     libvcruntime:winapi_downlevel.obj
 0002:00005358       ??_C@_0M@GDNOONDI@FlsGetValue@ 10024358     libvcruntime:winapi_downlevel.obj
 0002:0000536c       ??_C@_0M@JCPCPOEF@FlsSetValue@ 1002436c     libvcruntime:winapi_downlevel.obj
 0002:00005380       ??_C@_0BM@HCFOFFN@InitializeCriticalSectionEx@ 10024380     libvcruntime:winapi_downlevel.obj
 0002:000053a0       ??_7exception@std@@6B@     100243a0     libvcruntime:frame.obj
 0002:000053a8       ??_C@_0BC@EOODALEL@Unknown?5exception@ 100243a8     libvcruntime:frame.obj
 0002:000053c0       ??_7bad_exception@std@@6B@ 100243c0     libvcruntime:frame.obj
 0002:000053c8       ??_C@_0O@DPKOEFFH@bad?5exception@ 100243c8     libvcruntime:frame.obj
 0002:000053d8       ?standard_lookup_table_spectre@__crt_stdio_output@@3V?$spectre_mitigated_lookup_table@Ustate_transition_pair@__crt_stdio_output@@$0IA@@1@B 100243d8     libucrt:output.obj
 0002:000054d8       ??_C@_1O@CEDCILHN@?$AA?$CI?$AAn?$AAu?$AAl?$AAl?$AA?$CJ@ 100244d8     libucrt:output.obj
 0002:000054e8       ??_C@_06OJHGLDPL@?$CInull?$CJ@ 100244e8     libucrt:output.obj
 0002:00005658       ___acrt_exception_action_table 10024658     libucrt:exception_filter.obj
 0002:000056e8       ___acrt_signal_action_table_count 100246e8     libucrt:exception_filter.obj
 0002:000056ec       ___acrt_signal_action_first_fpe_index 100246ec     libucrt:exception_filter.obj
 0002:000056f0       ___acrt_signal_action_fpe_count 100246f0     libucrt:exception_filter.obj
 0002:000056f4       ??_C@_1BI@BGOHAHKC@?$AAm?$AAs?$AAc?$AAo?$AAr?$AAe?$AAe?$AA?4?$AAd?$AAl?$AAl@ 100246f4     libucrt:exit.obj
 0002:0000570c       ??_C@_0P@MIGLKIOC@CorExitProcess@ 1002470c     libucrt:exit.obj
 0002:000057a0       ___newctype                100247a0     libucrt:ctype.obj
 0002:00005aa0       ___newclmap                10024aa0     libucrt:ctype.obj
 0002:00005c20       ___newcumap                10024c20     libucrt:ctype.obj
 0002:00005da0       ___lc_time_c               10024da0     libucrt:nlsdata.obj
 0002:00005f04       ??_C@_03KOEHGMDN@Sun@      10024f04     libucrt:nlsdata.obj
 0002:00005f08       ??_C@_03PDAGKDH@Mon@       10024f08     libucrt:nlsdata.obj
 0002:00005f0c       ??_C@_03NAGEINEP@Tue@      10024f0c     libucrt:nlsdata.obj
 0002:00005f10       ??_C@_03MHOMLAJA@Wed@      10024f10     libucrt:nlsdata.obj
 0002:00005f14       ??_C@_03IOFIKPDN@Thu@      10024f14     libucrt:nlsdata.obj
 0002:00005f18       ??_C@_03IDIOELNC@Fri@      10024f18     libucrt:nlsdata.obj
 0002:00005f1c       ??_C@_03FEFJNEK@Sat@       10024f1c     libucrt:nlsdata.obj
 0002:00005f20       ??_C@_06OOPIFAJ@Sunday@    10024f20     libucrt:nlsdata.obj
 0002:00005f28       ??_C@_06JLEDEDGH@Monday@   10024f28     libucrt:nlsdata.obj
 0002:00005f30       ??_C@_07BAAGCFCM@Tuesday@  10024f30     libucrt:nlsdata.obj
 0002:00005f38       ??_C@_09DLIGFAKA@Wednesday@ 10024f38     libucrt:nlsdata.obj
 0002:00005f44       ??_C@_08HACCIKIA@Thursday@ 10024f44     libucrt:nlsdata.obj
 0002:00005f50       ??_C@_06JECMNKMI@Friday@   10024f50     libucrt:nlsdata.obj
 0002:00005f58       ??_C@_08INBOOONO@Saturday@ 10024f58     libucrt:nlsdata.obj
 0002:00005f64       ??_C@_03JIHJHPIE@Jan@      10024f64     libucrt:nlsdata.obj
 0002:00005f68       ??_C@_03HJBDCHOM@Feb@      10024f68     libucrt:nlsdata.obj
 0002:00005f6c       ??_C@_03ODNJBKGA@Mar@      10024f6c     libucrt:nlsdata.obj
 0002:00005f70       ??_C@_03LEOLGMJP@Apr@      10024f70     libucrt:nlsdata.obj
 0002:00005f74       ??_C@_03CNMDKL@May@        10024f74     libucrt:nlsdata.obj
 0002:00005f78       ??_C@_03IDFGHECI@Jun@      10024f78     libucrt:nlsdata.obj
 0002:00005f7c       ??_C@_03LBGABGKK@Jul@      10024f7c     libucrt:nlsdata.obj
 0002:00005f80       ??_C@_03IFJFEIGA@Aug@      10024f80     libucrt:nlsdata.obj
 0002:00005f84       ??_C@_03GGCAPAJC@Sep@      10024f84     libucrt:nlsdata.obj
 0002:00005f88       ??_C@_03BMAOKBAD@Oct@      10024f88     libucrt:nlsdata.obj
 0002:00005f8c       ??_C@_03JPJOFNIA@Nov@      10024f8c     libucrt:nlsdata.obj
 0002:00005f90       ??_C@_03MKABNOCG@Dec@      10024f90     libucrt:nlsdata.obj
 0002:00005f94       ??_C@_07CGJPFGJA@January@  10024f94     libucrt:nlsdata.obj
 0002:00005f9c       ??_C@_08GNJGEPFN@February@ 10024f9c     libucrt:nlsdata.obj
 0002:00005fa8       ??_C@_05HPCKOFNC@March@    10024fa8     libucrt:nlsdata.obj
 0002:00005fb0       ??_C@_05DMJDNLEJ@April@    10024fb0     libucrt:nlsdata.obj
 0002:00005fb8       ??_C@_04CNLMGBGM@June@     10024fb8     libucrt:nlsdata.obj
 0002:00005fc0       ??_C@_04MIEPOIFP@July@     10024fc0     libucrt:nlsdata.obj
 0002:00005fc8       ??_C@_06LBBHFDDG@August@   10024fc8     libucrt:nlsdata.obj
 0002:00005fd0       ??_C@_09BHHEALKD@September@ 10024fd0     libucrt:nlsdata.obj
 0002:00005fdc       ??_C@_07JJNFCEND@October@  10024fdc     libucrt:nlsdata.obj
 0002:00005fe4       ??_C@_08HCHEGEOA@November@ 10024fe4     libucrt:nlsdata.obj
 0002:00005ff0       ??_C@_08EDHMEBNP@December@ 10024ff0     libucrt:nlsdata.obj
 0002:00005ffc       ??_C@_02DEDBPAFC@AM@       10024ffc     libucrt:nlsdata.obj
 0002:00006000       ??_C@_02CJNFDJBF@PM@       10025000     libucrt:nlsdata.obj
 0002:00006004       ??_C@_08BPBNCDIB@MM?1dd?1yy@ 10025004     libucrt:nlsdata.obj
 0002:00006010       ??_C@_0BE@CKGJFCPC@dddd?0?5MMMM?5dd?0?5yyyy@ 10025010     libucrt:nlsdata.obj
 0002:00006024       ??_C@_08JCCMCCIL@HH?3mm?3ss@ 10025024     libucrt:nlsdata.obj
 0002:00006030       ??_C@_17MBGCMIPB@?$AAS?$AAu?$AAn@ 10025030     libucrt:nlsdata.obj
 0002:00006038       ??_C@_17KBOMKBF@?$AAM?$AAo?$AAn@ 10025038     libucrt:nlsdata.obj
 0002:00006040       ??_C@_17BMKGEGOJ@?$AAT?$AAu?$AAe@ 10025040     libucrt:nlsdata.obj
 0002:00006048       ??_C@_17CJEDCEPE@?$AAW?$AAe?$AAd@ 10025048     libucrt:nlsdata.obj
 0002:00006050       ??_C@_17PDPHAADD@?$AAT?$AAh?$AAu@ 10025050     libucrt:nlsdata.obj
 0002:00006058       ??_C@_17HFOLPPLP@?$AAF?$AAr?$AAi@ 10025058     libucrt:nlsdata.obj
 0002:00006060       ??_C@_17GGIBDPIH@?$AAS?$AAa?$AAt@ 10025060     libucrt:nlsdata.obj
 0002:00006068       ??_C@_1O@IHNHDHPB@?$AAS?$AAu?$AAn?$AAd?$AAa?$AAy@ 10025068     libucrt:nlsdata.obj
 0002:00006078       ??_C@_1O@MMNBFLIA@?$AAM?$AAo?$AAn?$AAd?$AAa?$AAy@ 10025078     libucrt:nlsdata.obj
 0002:00006088       ??_C@_1BA@ENFBFFEK@?$AAT?$AAu?$AAe?$AAs?$AAd?$AAa?$AAy@ 10025088     libucrt:nlsdata.obj
 0002:00006098       ??_C@_1BE@EBOGMDOH@?$AAW?$AAe?$AAd?$AAn?$AAe?$AAs?$AAd?$AAa?$AAy@ 10025098     libucrt:nlsdata.obj
 0002:000060ac       ??_C@_1BC@HHMNLIHE@?$AAT?$AAh?$AAu?$AAr?$AAs?$AAd?$AAa?$AAy@ 100250ac     libucrt:nlsdata.obj
 0002:000060c0       ??_C@_1O@PDICJHAG@?$AAF?$AAr?$AAi?$AAd?$AAa?$AAy@ 100250c0     libucrt:nlsdata.obj
 0002:000060d0       ??_C@_1BC@ENMNNPAJ@?$AAS?$AAa?$AAt?$AAu?$AAr?$AAd?$AAa?$AAy@ 100250d0     libucrt:nlsdata.obj
 0002:000060e4       ??_C@_17DKNBKCHM@?$AAJ?$AAa?$AAn@ 100250e4     libucrt:nlsdata.obj
 0002:000060ec       ??_C@_17LMDJEKJN@?$AAF?$AAe?$AAb@ 100250ec     libucrt:nlsdata.obj
 0002:000060f4       ??_C@_17CKNLEDEC@?$AAM?$AAa?$AAr@ 100250f4     libucrt:nlsdata.obj
 0002:000060fc       ??_C@_17LFPOIHDD@?$AAA?$AAp?$AAr@ 100250fc     libucrt:nlsdata.obj
 0002:00006104       ??_C@_17PNNKMEED@?$AAM?$AAa?$AAy@ 10025104     libucrt:nlsdata.obj
 0002:0000610c       ??_C@_17KCJGOCPB@?$AAJ?$AAu?$AAn@ 1002510c     libucrt:nlsdata.obj
 0002:00006114       ??_C@_17IJPCKHK@?$AAJ?$AAu?$AAl@ 10025114     libucrt:nlsdata.obj
 0002:0000611c       ??_C@_17ICPELBCN@?$AAA?$AAu?$AAg@ 1002511c     libucrt:nlsdata.obj
 0002:00006124       ??_C@_17HCHCOKMG@?$AAS?$AAe?$AAp@ 10025124     libucrt:nlsdata.obj
 0002:0000612c       ??_C@_17FNLKOI@?$AAO?$AAc?$AAt@ 1002512c     libucrt:nlsdata.obj
 0002:00006134       ??_C@_17BBDMLCIG@?$AAN?$AAo?$AAv@ 10025134     libucrt:nlsdata.obj
 0002:0000613c       ??_C@_17EGKACKIF@?$AAD?$AAe?$AAc@ 1002513c     libucrt:nlsdata.obj
 0002:00006144       ??_C@_1BA@EFMEIEBA@?$AAJ?$AAa?$AAn?$AAu?$AAa?$AAr?$AAy@ 10025144     libucrt:nlsdata.obj
 0002:00006154       ??_C@_1BC@JGDDFFAM@?$AAF?$AAe?$AAb?$AAr?$AAu?$AAa?$AAr?$AAy@ 10025154     libucrt:nlsdata.obj
 0002:00006168       ??_C@_1M@IKEENEDF@?$AAM?$AAa?$AAr?$AAc?$AAh@ 10025168     libucrt:nlsdata.obj
 0002:00006174       ??_C@_1M@GJNLMHFD@?$AAA?$AAp?$AAr?$AAi?$AAl@ 10025174     libucrt:nlsdata.obj
 0002:00006180       ??_C@_19EPFLPGAP@?$AAJ?$AAu?$AAn?$AAe@ 10025180     libucrt:nlsdata.obj
 0002:0000618c       ??_C@_19BIFMLPCD@?$AAJ?$AAu?$AAl?$AAy@ 1002518c     libucrt:nlsdata.obj
 0002:00006198       ??_C@_1O@PAHLKOAC@?$AAA?$AAu?$AAg?$AAu?$AAs?$AAt@ 10025198     libucrt:nlsdata.obj
 0002:000061a8       ??_C@_1BE@DKAAMBJL@?$AAS?$AAe?$AAp?$AAt?$AAe?$AAm?$AAb?$AAe?$AAr@ 100251a8     libucrt:nlsdata.obj
 0002:000061bc       ??_C@_1BA@EPANDLNG@?$AAO?$AAc?$AAt?$AAo?$AAb?$AAe?$AAr@ 100251bc     libucrt:nlsdata.obj
 0002:000061cc       ??_C@_1BC@BGLIFPF@?$AAN?$AAo?$AAv?$AAe?$AAm?$AAb?$AAe?$AAr@ 100251cc     libucrt:nlsdata.obj
 0002:000061e0       ??_C@_1BC@FEMKIFH@?$AAD?$AAe?$AAc?$AAe?$AAm?$AAb?$AAe?$AAr@ 100251e0     libucrt:nlsdata.obj
 0002:000061f4       ??_C@_15ODEHAHHF@?$AAA?$AAM@ 100251f4     libucrt:nlsdata.obj
 0002:000061fc       ??_C@_15CLMNNGEL@?$AAP?$AAM@ 100251fc     libucrt:nlsdata.obj
 0002:00006204       ??_C@_1BC@IEBCMHCM@?$AAM?$AAM?$AA?1?$AAd?$AAd?$AA?1?$AAy?$AAy@ 10025204     libucrt:nlsdata.obj
 0002:00006218       ??_C@_1CI@KNAKOEBC@?$AAd?$AAd?$AAd?$AAd?$AA?0?$AA?5?$AAM?$AAM?$AAM?$AAM?$AA?5?$AAd?$AAd?$AA?0?$AA?5@ 10025218     libucrt:nlsdata.obj
 0002:00006240       ??_C@_1BC@GDGBMEMK@?$AAH?$AAH?$AA?3?$AAm?$AAm?$AA?3?$AAs?$AAs@ 10025240     libucrt:nlsdata.obj
 0002:00006254       ??_C@_1M@BMHNFIME@?$AAe?$AAn?$AA?9?$AAU?$AAS@ 10025254     libucrt:nlsdata.obj
 0002:000062b8       ??_C@_1EA@JGEFHKEI@?$AAa?$AAp?$AAi?$AA?9?$AAm?$AAs?$AA?9?$AAw?$AAi?$AAn?$AA?9?$AAc?$AAo?$AAr?$AAe@ 100252b8     libucrt:winapi_thunks.obj
 0002:000062f8       ??_C@_1DI@KMEPCBPN@?$AAa?$AAp?$AAi?$AA?9?$AAm?$AAs?$AA?9?$AAw?$AAi?$AAn?$AA?9?$AAc?$AAo?$AAr?$AAe@ 100252f8     libucrt:winapi_thunks.obj
 0002:00006330       ??_C@_1DI@IJCEHOCB@?$AAa?$AAp?$AAi?$AA?9?$AAm?$AAs?$AA?9?$AAw?$AAi?$AAn?$AA?9?$AAc?$AAo?$AAr?$AAe@ 10025330     libucrt:winapi_thunks.obj
 0002:00006368       ??_C@_1EI@MPIAOHOC@?$AAa?$AAp?$AAi?$AA?9?$AAm?$AAs?$AA?9?$AAw?$AAi?$AAn?$AA?9?$AAc?$AAo?$AAr?$AAe@ 10025368     libucrt:winapi_thunks.obj
 0002:000063b0       ??_C@_1FK@FPHCKFIE@?$AAa?$AAp?$AAi?$AA?9?$AAm?$AAs?$AA?9?$AAw?$AAi?$AAn?$AA?9?$AAc?$AAo?$AAr?$AAe@ 100253b0     libucrt:winapi_thunks.obj
 0002:00006410       ??_C@_1EM@DILCGIIO@?$AAa?$AAp?$AAi?$AA?9?$AAm?$AAs?$AA?9?$AAw?$AAi?$AAn?$AA?9?$AAc?$AAo?$AAr?$AAe@ 10025410     libucrt:winapi_thunks.obj
 0002:0000645c       ??_C@_1DM@LNCGDDPN@?$AAa?$AAp?$AAi?$AA?9?$AAm?$AAs?$AA?9?$AAw?$AAi?$AAn?$AA?9?$AAc?$AAo?$AAr?$AAe@ 1002545c     libucrt:winapi_thunks.obj
 0002:00006498       ??_C@_1DO@FPAPJEMD@?$AAa?$AAp?$AAi?$AA?9?$AAm?$AAs?$AA?9?$AAw?$AAi?$AAn?$AA?9?$AAc?$AAo?$AAr?$AAe@ 10025498     libucrt:winapi_thunks.obj
 0002:000064d8       ??_C@_1DK@NDHNAHIO@?$AAa?$AAp?$AAi?$AA?9?$AAm?$AAs?$AA?9?$AAw?$AAi?$AAn?$AA?9?$AAc?$AAo?$AAr?$AAe@ 100254d8     libucrt:winapi_thunks.obj
 0002:00006514       ??_C@_1DM@KGHDGBCM@?$AAa?$AAp?$AAi?$AA?9?$AAm?$AAs?$AA?9?$AAw?$AAi?$AAn?$AA?9?$AAc?$AAo?$AAr?$AAe@ 10025514     libucrt:winapi_thunks.obj
 0002:00006550       ??_C@_1EO@IJIOEFOH@?$AAa?$AAp?$AAi?$AA?9?$AAm?$AAs?$AA?9?$AAw?$AAi?$AAn?$AA?9?$AAr?$AAt?$AAc?$AAo@ 10025550     libucrt:winapi_thunks.obj
 0002:000065a0       ??_C@_1FG@HHGEKANL@?$AAa?$AAp?$AAi?$AA?9?$AAm?$AAs?$AA?9?$AAw?$AAi?$AAn?$AA?9?$AAs?$AAe?$AAc?$AAu@ 100255a0     libucrt:winapi_thunks.obj
 0002:000065f8       ??_C@_1EG@DBIOJECG@?$AAe?$AAx?$AAt?$AA?9?$AAm?$AAs?$AA?9?$AAw?$AAi?$AAn?$AA?9?$AAn?$AAt?$AAu?$AAs@ 100255f8     libucrt:winapi_thunks.obj
 0002:00006640       ??_C@_1EO@FIHMJCLF@?$AAe?$AAx?$AAt?$AA?9?$AAm?$AAs?$AA?9?$AAw?$AAi?$AAn?$AA?9?$AAn?$AAt?$AAu?$AAs@ 10025640     libucrt:winapi_thunks.obj
 0002:00006690       ??_C@_1BC@DNHGCMLG@?$AAa?$AAd?$AAv?$AAa?$AAp?$AAi?$AA3?$AA2@ 10025690     libucrt:winapi_thunks.obj
 0002:000066a4       ??_C@_1BG@CJPGBMEF@?$AAk?$AAe?$AAr?$AAn?$AAe?$AAl?$AAb?$AAa?$AAs?$AAe@ 100256a4     libucrt:winapi_thunks.obj
 0002:000066bc       ??_C@_1M@OAIMIKLP@?$AAn?$AAt?$AAd?$AAl?$AAl@ 100256bc     libucrt:winapi_thunks.obj
 0002:000066c8       ??_C@_1EG@DPGNFKGC@?$AAa?$AAp?$AAi?$AA?9?$AAm?$AAs?$AA?9?$AAw?$AAi?$AAn?$AA?9?$AAa?$AAp?$AAp?$AAm@ 100256c8     libucrt:winapi_thunks.obj
 0002:00006710       ??_C@_1O@BCCLBEOE@?$AAu?$AAs?$AAe?$AAr?$AA3?$AA2@ 10025710     libucrt:winapi_thunks.obj
 0002:00006720       ??_C@_1DM@BPJLHKCE@?$AAa?$AAp?$AAi?$AA?9?$AAm?$AAs?$AA?9?$AAw?$AAi?$AAn?$AA?9?$AAc?$AAo?$AAr?$AAe@ 10025720     libucrt:winapi_thunks.obj
 0002:0000675c       ??_C@_1BA@IAIFMGEF@?$AAe?$AAx?$AAt?$AA?9?$AAm?$AAs?$AA?9@ 1002575c     libucrt:winapi_thunks.obj
 0002:00006770       ??_C@_0BA@FHFNEAED@AreFileApisANSI@ 10025770     libucrt:winapi_thunks.obj
 0002:00006790       ??_C@_0O@KKBNKAPF@LCMapStringEx@ 10025790     libucrt:winapi_thunks.obj
 0002:000067a8       ??_C@_0BB@HBDEELFH@LocaleNameToLCID@ 100257a8     libucrt:winapi_thunks.obj
 0002:000067c0       ??_C@_0CF@OJOFEIGO@AppPolicyGetProcessTerminationM@ 100257c0     libucrt:winapi_thunks.obj
 0002:00006848       ??_C@_03OEIAHPBN@INF@      10025848     libucrt:cvt.obj
 0002:0000684c       ??_C@_03OJHLLCGB@inf@      1002584c     libucrt:cvt.obj
 0002:00006850       ??_C@_03LKNCIKJB@NAN@      10025850     libucrt:cvt.obj
 0002:00006854       ??_C@_03LHCJEHON@nan@      10025854     libucrt:cvt.obj
 0002:00006858       ??_C@_09OFJJIMPC@NAN?$CISNAN?$CJ@ 10025858     libucrt:cvt.obj
 0002:00006864       ??_C@_09IPFBKMDL@nan?$CIsnan?$CJ@ 10025864     libucrt:cvt.obj
 0002:00006870       ??_C@_08IKHNHAJ@NAN?$CIIND?$CJ@ 10025870     libucrt:cvt.obj
 0002:0000687c       ??_C@_08OFCDMILK@nan?$CIind?$CJ@ 1002587c     libucrt:cvt.obj
 0002:00006888       ??_C@_05KLBDPFGC@e?$CL000@ 10025888     libucrt:cvt.obj
 0002:000068a0       ??_C@_1M@HPNHIDJI@?$AAj?$AAa?$AA?9?$AAJ?$AAP@ 100258a0     libucrt:mbctype.obj
 0002:000068ac       ??_C@_1M@BIBDDEMK@?$AAz?$AAh?$AA?9?$AAC?$AAN@ 100258ac     libucrt:mbctype.obj
 0002:000068b8       ??_C@_1M@JLOOOEGK@?$AAk?$AAo?$AA?9?$AAK?$AAR@ 100258b8     libucrt:mbctype.obj
 0002:000068c4       ??_C@_1M@CLNBBOPM@?$AAz?$AAh?$AA?9?$AAT?$AAW@ 100258c4     libucrt:mbctype.obj
 0002:000068d0       ??_C@_15PJPFLCCM@?$AAu?$AAk@ 100258d0     libucrt:get_qualified_locale.obj
 0002:00006ff8       ??_C@_15EMKDOKLE@?$AAa?$AAr@ 10025ff8     libucrt:lcidtoname_downlevel.obj
 0002:00007000       ??_C@_15KNPADPLH@?$AAb?$AAg@ 10026000     libucrt:lcidtoname_downlevel.obj
 0002:00007008       ??_C@_15EDMHLDMO@?$AAc?$AAa@ 10026008     libucrt:lcidtoname_downlevel.obj
 0002:00007010       ??_C@_1O@BPEAJADD@?$AAz?$AAh?$AA?9?$AAC?$AAH?$AAS@ 10026010     libucrt:lcidtoname_downlevel.obj
 0002:00007020       ??_C@_15LJNHCMNK@?$AAc?$AAs@ 10026020     libucrt:lcidtoname_downlevel.obj
 0002:00007028       ??_C@_15FOMCIDHG@?$AAd?$AAa@ 10026028     libucrt:lcidtoname_downlevel.obj
 0002:00007030       ??_C@_15NBKABECB@?$AAd?$AAe@ 10026030     libucrt:lcidtoname_downlevel.obj
 0002:00007038       ??_C@_15GHPEIIAO@?$AAe?$AAl@ 10026038     libucrt:lcidtoname_downlevel.obj
 0002:00007040       ??_C@_15MNPNEAIF@?$AAe?$AAn@ 10026040     libucrt:lcidtoname_downlevel.obj
 0002:00007048       ??_C@_15GPIOMPMH@?$AAe?$AAs@ 10026048     libucrt:lcidtoname_downlevel.obj
 0002:00007050       ??_C@_15NGLOAKJC@?$AAf?$AAi@ 10026050     libucrt:lcidtoname_downlevel.obj
 0002:00007058       ??_C@_15FBKGNKAM@?$AAf?$AAr@ 10026058     libucrt:lcidtoname_downlevel.obj
 0002:00007060       ??_C@_15KGGCNEFK@?$AAh?$AAe@ 10026060     libucrt:lcidtoname_downlevel.obj
 0002:00007068       ??_C@_15PGHLIDMF@?$AAh?$AAu@ 10026068     libucrt:lcidtoname_downlevel.obj
 0002:00007070       ??_C@_15BIEMAPLM@?$AAi?$AAs@ 10026070     libucrt:lcidtoname_downlevel.obj
 0002:00007078       ??_C@_15IFJLDHAF@?$AAi?$AAt@ 10026078     libucrt:lcidtoname_downlevel.obj
 0002:00007080       ??_C@_15GEMIOCAG@?$AAj?$AAa@ 10026080     libucrt:lcidtoname_downlevel.obj
 0002:00007088       ??_C@_15EPELEGJA@?$AAk?$AAo@ 10026088     libucrt:lcidtoname_downlevel.obj
 0002:00007090       ??_C@_15NDDHIMN@?$AAn?$AAl@ 10026090     libucrt:lcidtoname_downlevel.obj
 0002:00007098       ??_C@_15BPIGNHCD@?$AAn?$AAo@ 10026098     libucrt:lcidtoname_downlevel.obj
 0002:000070a0       ??_C@_15DEOPBLCG@?$AAp?$AAl@ 100260a0     libucrt:lcidtoname_downlevel.obj
 0002:000070a8       ??_C@_15KBECGEFG@?$AAp?$AAt@ 100260a8     libucrt:lcidtoname_downlevel.obj
 0002:000070b0       ??_C@_15GLJCBFMD@?$AAr?$AAo@ 100260b0     libucrt:lcidtoname_downlevel.obj
 0002:000070b8       ??_C@_15FEDGKCDI@?$AAr?$AAu@ 100260b8     libucrt:lcidtoname_downlevel.obj
 0002:000070c0       ??_C@_15GLKMLLHM@?$AAh?$AAr@ 100260c0     libucrt:lcidtoname_downlevel.obj
 0002:000070c8       ??_C@_15CPKMFBDB@?$AAs?$AAk@ 100260c8     libucrt:lcidtoname_downlevel.obj
 0002:000070d0       ??_C@_15BAAIOGMK@?$AAs?$AAq@ 100260d0     libucrt:lcidtoname_downlevel.obj
 0002:000070d8       ??_C@_15INNPNOHD@?$AAs?$AAv@ 100260d8     libucrt:lcidtoname_downlevel.obj
 0002:000070e0       ??_C@_15CABMMOGH@?$AAt?$AAh@ 100260e0     libucrt:lcidtoname_downlevel.obj
 0002:000070e8       ??_C@_15BPLIHJJM@?$AAt?$AAr@ 100260e8     libucrt:lcidtoname_downlevel.obj
 0002:000070f0       ??_C@_15NEOEKKDJ@?$AAu?$AAr@ 100260f0     libucrt:lcidtoname_downlevel.obj
 0002:000070f8       ??_C@_15NFICGAJK@?$AAi?$AAd@ 100260f8     libucrt:lcidtoname_downlevel.obj
 0002:00007100       ??_C@_15HPJPHDM@?$AAb?$AAe@ 10026100     libucrt:lcidtoname_downlevel.obj
 0002:00007108       ??_C@_15LCHLGJII@?$AAs?$AAl@ 10026108     libucrt:lcidtoname_downlevel.obj
 0002:00007110       ??_C@_15PCFJPHHO@?$AAe?$AAt@ 10026110     libucrt:lcidtoname_downlevel.obj
 0002:00007118       ??_C@_15HPFPGODN@?$AAl?$AAv@ 10026118     libucrt:lcidtoname_downlevel.obj
 0002:00007120       ??_C@_15NFFGKGLG@?$AAl?$AAt@ 10026120     libucrt:lcidtoname_downlevel.obj
 0002:00007128       ??_C@_15BDAKCCHN@?$AAf?$AAa@ 10026128     libucrt:lcidtoname_downlevel.obj
 0002:00007130       ??_C@_15NFGIAIAJ@?$AAv?$AAi@ 10026130     libucrt:lcidtoname_downlevel.obj
 0002:00007138       ??_C@_15LMKNDMHN@?$AAh?$AAy@ 10026138     libucrt:lcidtoname_downlevel.obj
 0002:00007140       ??_C@_15IJBHMCFL@?$AAa?$AAz@ 10026140     libucrt:lcidtoname_downlevel.obj
 0002:00007148       ??_C@_15EKOFJABL@?$AAe?$AAu@ 10026148     libucrt:lcidtoname_downlevel.obj
 0002:00007150       ??_C@_15BGHADCNK@?$AAm?$AAk@ 10026150     libucrt:lcidtoname_downlevel.obj
 0002:00007158       ??_C@_15JDNICKHM@?$AAa?$AAf@ 10026158     libucrt:lcidtoname_downlevel.obj
 0002:00007160       ??_C@_15KPJEDBKD@?$AAk?$AAa@ 10026160     libucrt:lcidtoname_downlevel.obj
 0002:00007168       ??_C@_15PDNFFFEO@?$AAf?$AAo@ 10026168     libucrt:lcidtoname_downlevel.obj
 0002:00007170       ??_C@_15OMLEGLOC@?$AAh?$AAi@ 10026170     libucrt:lcidtoname_downlevel.obj
 0002:00007178       ??_C@_15IDNNENKK@?$AAm?$AAs@ 10026178     libucrt:lcidtoname_downlevel.obj
 0002:00007180       ??_C@_15MACJNBMH@?$AAk?$AAk@ 10026180     libucrt:lcidtoname_downlevel.obj
 0002:00007188       ??_C@_15DKDJEOND@?$AAk?$AAy@ 10026188     libucrt:lcidtoname_downlevel.obj
 0002:00007190       ??_C@_15DFGDLJBG@?$AAs?$AAw@ 10026190     libucrt:lcidtoname_downlevel.obj
 0002:00007198       ??_C@_15BBFAICNG@?$AAu?$AAz@ 10026198     libucrt:lcidtoname_downlevel.obj
 0002:000071a0       ??_C@_15DKNDCGEA@?$AAt?$AAt@ 100261a0     libucrt:lcidtoname_downlevel.obj
 0002:000071a8       ??_C@_15MGIFMDPL@?$AAp?$AAa@ 100261a8     libucrt:lcidtoname_downlevel.obj
 0002:000071b0       ??_C@_15HCNDBBA@?$AAg?$AAu@ 100261b0     libucrt:lcidtoname_downlevel.obj
 0002:000071b8       ??_C@_15FNBEIBON@?$AAt?$AAa@ 100261b8     libucrt:lcidtoname_downlevel.obj
 0002:000071c0       ??_C@_15NCHGBGLK@?$AAt?$AAe@ 100261c0     libucrt:lcidtoname_downlevel.obj
 0002:000071c8       ??_C@_15PHPHCBPF@?$AAk?$AAn@ 100261c8     libucrt:lcidtoname_downlevel.obj
 0002:000071d0       ??_C@_15DLGBCKMP@?$AAm?$AAr@ 100261d0     libucrt:lcidtoname_downlevel.obj
 0002:000071d8       ??_C@_15EABBLBFF@?$AAs?$AAa@ 100261d8     libucrt:lcidtoname_downlevel.obj
 0002:000071e0       ??_C@_15CBKOMCOI@?$AAm?$AAn@ 100261e0     libucrt:lcidtoname_downlevel.obj
 0002:000071e8       ??_C@_15CKDMCJAF@?$AAg?$AAl@ 100261e8     libucrt:lcidtoname_downlevel.obj
 0002:000071f0       ??_C@_17CNJFBPG@?$AAk?$AAo?$AAk@ 100261f0     libucrt:lcidtoname_downlevel.obj
 0002:000071f8       ??_C@_17FFBJICPL@?$AAs?$AAy?$AAr@ 100261f8     libucrt:lcidtoname_downlevel.obj
 0002:00007200       ??_C@_17KPNDCPAF@?$AAd?$AAi?$AAv@ 10026200     libucrt:lcidtoname_downlevel.obj
 0002:00007208       ??_C@_11LOCGONAA@@         10026208     libucrt:lcidtoname_downlevel.obj
 0002:0000720c       ??_C@_1M@OKAHONE@?$AAa?$AAr?$AA?9?$AAS?$AAA@ 1002620c     libucrt:lcidtoname_downlevel.obj
 0002:00007218       ??_C@_1M@FFFIGIGK@?$AAb?$AAg?$AA?9?$AAB?$AAG@ 10026218     libucrt:lcidtoname_downlevel.obj
 0002:00007224       ??_C@_1M@BJNKEDC@?$AAc?$AAa?$AA?9?$AAE?$AAS@ 10026224     libucrt:lcidtoname_downlevel.obj
 0002:00007230       ??_C@_1M@IJJHFJHA@?$AAc?$AAs?$AA?9?$AAC?$AAZ@ 10026230     libucrt:lcidtoname_downlevel.obj
 0002:0000723c       ??_C@_1M@CLPEOBGI@?$AAd?$AAa?$AA?9?$AAD?$AAK@ 1002623c     libucrt:lcidtoname_downlevel.obj
 0002:00007248       ??_C@_1M@MCMADGCB@?$AAd?$AAe?$AA?9?$AAD?$AAE@ 10026248     libucrt:lcidtoname_downlevel.obj
 0002:00007254       ??_C@_1M@OOCKEMAM@?$AAe?$AAl?$AA?9?$AAG?$AAR@ 10026254     libucrt:lcidtoname_downlevel.obj
 0002:00007260       ??_C@_1M@DDNJFGID@?$AAf?$AAi?$AA?9?$AAF?$AAI@ 10026260     libucrt:lcidtoname_downlevel.obj
 0002:0000726c       ??_C@_1M@GLIPPMAC@?$AAf?$AAr?$AA?9?$AAF?$AAR@ 1002626c     libucrt:lcidtoname_downlevel.obj
 0002:00007278       ??_C@_1M@GFMCHPE@?$AAh?$AAe?$AA?9?$AAI?$AAL@ 10026278     libucrt:lcidtoname_downlevel.obj
 0002:00007284       ??_C@_1M@MHLPGNKM@?$AAh?$AAu?$AA?9?$AAH?$AAU@ 10026284     libucrt:lcidtoname_downlevel.obj
 0002:00007290       ??_C@_1M@LPDDNNPN@?$AAi?$AAs?$AA?9?$AAI?$AAS@ 10026290     libucrt:lcidtoname_downlevel.obj
 0002:0000729c       ??_C@_1M@MADIPODN@?$AAi?$AAt?$AA?9?$AAI?$AAT@ 1002629c     libucrt:lcidtoname_downlevel.obj
 0002:000072a8       ??_C@_1M@IHBJJGG@?$AAn?$AAl?$AA?9?$AAN?$AAL@ 100262a8     libucrt:lcidtoname_downlevel.obj
 0002:000072b4       ??_C@_1M@EANAGDL@?$AAn?$AAb?$AA?9?$AAN?$AAO@ 100262b4     libucrt:lcidtoname_downlevel.obj
 0002:000072c0       ??_C@_1M@NEIEMEGP@?$AAp?$AAl?$AA?9?$AAP?$AAL@ 100262c0     libucrt:lcidtoname_downlevel.obj
 0002:000072cc       ??_C@_1M@BOCFIGEP@?$AAp?$AAt?$AA?9?$AAB?$AAR@ 100262cc     libucrt:lcidtoname_downlevel.obj
 0002:000072d8       ??_C@_1M@IMPFOPBG@?$AAr?$AAo?$AA?9?$AAR?$AAO@ 100262d8     libucrt:lcidtoname_downlevel.obj
 0002:000072e4       ??_C@_1M@IDNNEJMM@?$AAr?$AAu?$AA?9?$AAR?$AAU@ 100262e4     libucrt:lcidtoname_downlevel.obj
 0002:000072f0       ??_C@_1M@LILEEOGM@?$AAh?$AAr?$AA?9?$AAH?$AAR@ 100262f0     libucrt:lcidtoname_downlevel.obj
 0002:000072fc       ??_C@_1M@FKIFEHPB@?$AAs?$AAk?$AA?9?$AAS?$AAK@ 100262fc     libucrt:lcidtoname_downlevel.obj
 0002:00007308       ??_C@_1M@LJMAMNPJ@?$AAs?$AAq?$AA?9?$AAA?$AAL@ 10026308     libucrt:lcidtoname_downlevel.obj
 0002:00007314       ??_C@_1M@GIAKDKJK@?$AAs?$AAv?$AA?9?$AAS?$AAE@ 10026314     libucrt:lcidtoname_downlevel.obj
 0002:00007320       ??_C@_1M@MKJKIKCL@?$AAt?$AAh?$AA?9?$AAT?$AAH@ 10026320     libucrt:lcidtoname_downlevel.obj
 0002:0000732c       ??_C@_1M@MFLCCMPB@?$AAt?$AAr?$AA?9?$AAT?$AAR@ 1002632c     libucrt:lcidtoname_downlevel.obj
 0002:00007338       ??_C@_1M@OIJHDKJN@?$AAu?$AAr?$AA?9?$AAP?$AAK@ 10026338     libucrt:lcidtoname_downlevel.obj
 0002:00007344       ??_C@_1M@LHIPCIEK@?$AAi?$AAd?$AA?9?$AAI?$AAD@ 10026344     libucrt:lcidtoname_downlevel.obj
 0002:00007350       ??_C@_1M@MFMOBGI@?$AAu?$AAk?$AA?9?$AAU?$AAA@ 10026350     libucrt:lcidtoname_downlevel.obj
 0002:0000735c       ??_C@_1M@OBGLJIPL@?$AAb?$AAe?$AA?9?$AAB?$AAY@ 1002635c     libucrt:lcidtoname_downlevel.obj
 0002:00007368       ??_C@_1M@BCFAJEAD@?$AAs?$AAl?$AA?9?$AAS?$AAI@ 10026368     libucrt:lcidtoname_downlevel.obj
 0002:00007374       ??_C@_1M@FKFFEDDN@?$AAe?$AAt?$AA?9?$AAE?$AAE@ 10026374     libucrt:lcidtoname_downlevel.obj
 0002:00007380       ??_C@_1M@KGKKAACI@?$AAl?$AAv?$AA?9?$AAL?$AAV@ 10026380     libucrt:lcidtoname_downlevel.obj
 0002:0000738c       ??_C@_1M@IFGBIJO@?$AAl?$AAt?$AA?9?$AAL?$AAT@ 1002638c     libucrt:lcidtoname_downlevel.obj
 0002:00007398       ??_C@_1M@FGEAHEDM@?$AAf?$AAa?$AA?9?$AAI?$AAR@ 10026398     libucrt:lcidtoname_downlevel.obj
 0002:000073a4       ??_C@_1M@KBMAIBFN@?$AAv?$AAi?$AA?9?$AAV?$AAN@ 100263a4     libucrt:lcidtoname_downlevel.obj
 0002:000073b0       ??_C@_1M@GPCBKDJK@?$AAh?$AAy?$AA?9?$AAA?$AAM@ 100263b0     libucrt:lcidtoname_downlevel.obj
 0002:000073bc       ??_C@_1BG@BECMDDJB@?$AAa?$AAz?$AA?9?$AAA?$AAZ?$AA?9?$AAL?$AAa?$AAt?$AAn@ 100263bc     libucrt:lcidtoname_downlevel.obj
 0002:000073d4       ??_C@_1M@MAOFCAEA@?$AAe?$AAu?$AA?9?$AAE?$AAS@ 100263d4     libucrt:lcidtoname_downlevel.obj
 0002:000073e0       ??_C@_1M@IGHABKPI@?$AAm?$AAk?$AA?9?$AAM?$AAK@ 100263e0     libucrt:lcidtoname_downlevel.obj
 0002:000073ec       ??_C@_1M@IAIGNEJG@?$AAt?$AAn?$AA?9?$AAZ?$AAA@ 100263ec     libucrt:lcidtoname_downlevel.obj
 0002:000073f8       ??_C@_1M@IIJCOJFA@?$AAx?$AAh?$AA?9?$AAZ?$AAA@ 100263f8     libucrt:lcidtoname_downlevel.obj
 0002:00007404       ??_C@_1M@LGPJHNJH@?$AAz?$AAu?$AA?9?$AAZ?$AAA@ 10026404     libucrt:lcidtoname_downlevel.obj
 0002:00007410       ??_C@_1M@HOKAOIO@?$AAa?$AAf?$AA?9?$AAZ?$AAA@ 10026410     libucrt:lcidtoname_downlevel.obj
 0002:0000741c       ??_C@_1M@DPCLHLIE@?$AAk?$AAa?$AA?9?$AAG?$AAE@ 1002641c     libucrt:lcidtoname_downlevel.obj
 0002:00007428       ??_C@_1M@BLKMHJBI@?$AAf?$AAo?$AA?9?$AAF?$AAO@ 10026428     libucrt:lcidtoname_downlevel.obj
 0002:00007434       ??_C@_1M@LGGJAPPB@?$AAh?$AAi?$AA?9?$AAI?$AAN@ 10026434     libucrt:lcidtoname_downlevel.obj
 0002:00007440       ??_C@_1M@FIKPIHFE@?$AAm?$AAt?$AA?9?$AAM?$AAT@ 10026440     libucrt:lcidtoname_downlevel.obj
 0002:0000744c       ??_C@_1M@HEGGPBFA@?$AAs?$AAe?$AA?9?$AAN?$AAO@ 1002644c     libucrt:lcidtoname_downlevel.obj
 0002:00007458       ??_C@_1M@EIBJEEPA@?$AAm?$AAs?$AA?9?$AAM?$AAY@ 10026458     libucrt:lcidtoname_downlevel.obj
 0002:00007464       ??_C@_1M@FHLBGMPP@?$AAk?$AAk?$AA?9?$AAK?$AAZ@ 10026464     libucrt:lcidtoname_downlevel.obj
 0002:00007470       ??_C@_1M@NGJJLCGI@?$AAk?$AAy?$AA?9?$AAK?$AAG@ 10026470     libucrt:lcidtoname_downlevel.obj
 0002:0000747c       ??_C@_1M@GIENNBFC@?$AAs?$AAw?$AA?9?$AAK?$AAE@ 1002647c     libucrt:lcidtoname_downlevel.obj
 0002:00007488       ??_C@_1BG@NDGMJIMJ@?$AAu?$AAz?$AA?9?$AAU?$AAZ?$AA?9?$AAL?$AAa?$AAt?$AAn@ 10026488     libucrt:lcidtoname_downlevel.obj
 0002:000074a0       ??_C@_1M@IDCCIHBC@?$AAt?$AAt?$AA?9?$AAR?$AAU@ 100264a0     libucrt:lcidtoname_downlevel.obj
 0002:000074ac       ??_C@_1M@LOICPMOJ@?$AAb?$AAn?$AA?9?$AAI?$AAN@ 100264ac     libucrt:lcidtoname_downlevel.obj
 0002:000074b8       ??_C@_1M@KPKKNEAH@?$AAp?$AAa?$AA?9?$AAI?$AAN@ 100264b8     libucrt:lcidtoname_downlevel.obj
 0002:000074c4       ??_C@_1M@PJGPPBOG@?$AAg?$AAu?$AA?9?$AAI?$AAN@ 100264c4     libucrt:lcidtoname_downlevel.obj
 0002:000074d0       ??_C@_1M@KMKMOPHI@?$AAt?$AAa?$AA?9?$AAI?$AAN@ 100264d0     libucrt:lcidtoname_downlevel.obj
 0002:000074dc       ??_C@_1M@KFEHEPAC@?$AAt?$AAe?$AA?9?$AAI?$AAN@ 100264dc     libucrt:lcidtoname_downlevel.obj
 0002:000074e8       ??_C@_1M@CDCLMGHI@?$AAk?$AAn?$AA?9?$AAI?$AAN@ 100264e8     libucrt:lcidtoname_downlevel.obj
 0002:000074f4       ??_C@_1M@MIODLDKF@?$AAm?$AAl?$AA?9?$AAI?$AAN@ 100264f4     libucrt:lcidtoname_downlevel.obj
 0002:00007500       ??_C@_1M@PBIEACPO@?$AAm?$AAr?$AA?9?$AAI?$AAN@ 10026500     libucrt:lcidtoname_downlevel.obj
 0002:0000750c       ??_C@_1M@NIDEAGPH@?$AAs?$AAa?$AA?9?$AAI?$AAN@ 1002650c     libucrt:lcidtoname_downlevel.obj
 0002:00007518       ??_C@_1M@FHIHCBIO@?$AAm?$AAn?$AA?9?$AAM?$AAN@ 10026518     libucrt:lcidtoname_downlevel.obj
 0002:00007524       ??_C@_1M@JAIJPENP@?$AAc?$AAy?$AA?9?$AAG?$AAB@ 10026524     libucrt:lcidtoname_downlevel.obj
 0002:00007530       ??_C@_1M@PHGFBEPN@?$AAg?$AAl?$AA?9?$AAE?$AAS@ 10026530     libucrt:lcidtoname_downlevel.obj
 0002:0000753c       ??_C@_1O@KPIPDNCP@?$AAk?$AAo?$AAk?$AA?9?$AAI?$AAN@ 1002653c     libucrt:lcidtoname_downlevel.obj
 0002:0000754c       ??_C@_1O@KNHJLDJA@?$AAs?$AAy?$AAr?$AA?9?$AAS?$AAY@ 1002654c     libucrt:lcidtoname_downlevel.obj
 0002:0000755c       ??_C@_1O@MKEKBLAH@?$AAd?$AAi?$AAv?$AA?9?$AAM?$AAV@ 1002655c     libucrt:lcidtoname_downlevel.obj
 0002:0000756c       ??_C@_1O@OHDCKDDF@?$AAq?$AAu?$AAz?$AA?9?$AAB?$AAO@ 1002656c     libucrt:lcidtoname_downlevel.obj
 0002:0000757c       ??_C@_1M@LEPJNLFD@?$AAn?$AAs?$AA?9?$AAZ?$AAA@ 1002657c     libucrt:lcidtoname_downlevel.obj
 0002:00007588       ??_C@_1M@OMLEIIJB@?$AAm?$AAi?$AA?9?$AAN?$AAZ@ 10026588     libucrt:lcidtoname_downlevel.obj
 0002:00007594       ??_C@_1M@PMPEAILG@?$AAa?$AAr?$AA?9?$AAI?$AAQ@ 10026594     libucrt:lcidtoname_downlevel.obj
 0002:000075a0       ??_C@_1M@CNKPNOEE@?$AAd?$AAe?$AA?9?$AAC?$AAH@ 100265a0     libucrt:lcidtoname_downlevel.obj
 0002:000075ac       ??_C@_1M@LKMGMLKO@?$AAe?$AAn?$AA?9?$AAG?$AAB@ 100265ac     libucrt:lcidtoname_downlevel.obj
 0002:000075b8       ??_C@_1M@PGKJFFGL@?$AAe?$AAs?$AA?9?$AAM?$AAX@ 100265b8     libucrt:lcidtoname_downlevel.obj
 0002:000075c4       ??_C@_1M@DNNANBDC@?$AAf?$AAr?$AA?9?$AAB?$AAE@ 100265c4     libucrt:lcidtoname_downlevel.obj
 0002:000075d0       ??_C@_1M@HLGMDFHM@?$AAi?$AAt?$AA?9?$AAC?$AAH@ 100265d0     libucrt:lcidtoname_downlevel.obj
 0002:000075dc       ??_C@_1M@CLLBGJH@?$AAn?$AAl?$AA?9?$AAB?$AAE@ 100265dc     libucrt:lcidtoname_downlevel.obj
 0002:000075e8       ??_C@_1M@BODBOGLF@?$AAn?$AAn?$AA?9?$AAN?$AAO@ 100265e8     libucrt:lcidtoname_downlevel.obj
 0002:000075f4       ??_C@_1M@HFFAHKAD@?$AAp?$AAt?$AA?9?$AAP?$AAT@ 100265f4     libucrt:lcidtoname_downlevel.obj
 0002:00007600       ??_C@_1BG@LNOAKHIE@?$AAs?$AAr?$AA?9?$AAS?$AAP?$AA?9?$AAL?$AAa?$AAt?$AAn@ 10026600     libucrt:lcidtoname_downlevel.obj
 0002:00007618       ??_C@_1M@HBMHBGAK@?$AAs?$AAv?$AA?9?$AAF?$AAI@ 10026618     libucrt:lcidtoname_downlevel.obj
 0002:00007624       ??_C@_1BG@DGCJGJBE@?$AAa?$AAz?$AA?9?$AAA?$AAZ?$AA?9?$AAC?$AAy?$AAr?$AAl@ 10026624     libucrt:lcidtoname_downlevel.obj
 0002:0000763c       ??_C@_1M@KEJDAAHB@?$AAs?$AAe?$AA?9?$AAS?$AAE@ 1002663c     libucrt:lcidtoname_downlevel.obj
 0002:00007648       ??_C@_1M@HEIBJJAD@?$AAm?$AAs?$AA?9?$AAB?$AAN@ 10026648     libucrt:lcidtoname_downlevel.obj
 0002:00007654       ??_C@_1BG@PBGJMCEM@?$AAu?$AAz?$AA?9?$AAU?$AAZ?$AA?9?$AAC?$AAy?$AAr?$AAl@ 10026654     libucrt:lcidtoname_downlevel.obj
 0002:0000766c       ??_C@_1O@LAOBCMDF@?$AAq?$AAu?$AAz?$AA?9?$AAE?$AAC@ 1002666c     libucrt:lcidtoname_downlevel.obj
 0002:0000767c       ??_C@_1M@POEEMAIO@?$AAa?$AAr?$AA?9?$AAE?$AAG@ 1002667c     libucrt:lcidtoname_downlevel.obj
 0002:00007688       ??_C@_1M@EFAKDEDL@?$AAz?$AAh?$AA?9?$AAH?$AAK@ 10026688     libucrt:lcidtoname_downlevel.obj
 0002:00007694       ??_C@_1M@HKKIJHGI@?$AAd?$AAe?$AA?9?$AAA?$AAT@ 10026694     libucrt:lcidtoname_downlevel.obj
 0002:000076a0       ??_C@_1M@KBFBEHJF@?$AAe?$AAn?$AA?9?$AAA?$AAU@ 100266a0     libucrt:lcidtoname_downlevel.obj
 0002:000076ac       ??_C@_1M@MNPLFAAH@?$AAe?$AAs?$AA?9?$AAE?$AAS@ 100266ac     libucrt:lcidtoname_downlevel.obj
 0002:000076b8       ??_C@_1M@HJOOJFMA@?$AAf?$AAr?$AA?9?$AAC?$AAA@ 100266b8     libucrt:lcidtoname_downlevel.obj
 0002:000076c4       ??_C@_1BG@JPOFPNAB@?$AAs?$AAr?$AA?9?$AAS?$AAP?$AA?9?$AAC?$AAy?$AAr?$AAl@ 100266c4     libucrt:lcidtoname_downlevel.obj
 0002:000076dc       ??_C@_1M@LNFOCMOB@?$AAs?$AAe?$AA?9?$AAF?$AAI@ 100266dc     libucrt:lcidtoname_downlevel.obj
 0002:000076e8       ??_C@_1O@MGJBOAMB@?$AAq?$AAu?$AAz?$AA?9?$AAP?$AAE@ 100266e8     libucrt:lcidtoname_downlevel.obj
 0002:000076f8       ??_C@_1M@GJINLBOK@?$AAa?$AAr?$AA?9?$AAL?$AAY@ 100266f8     libucrt:lcidtoname_downlevel.obj
 0002:00007704       ??_C@_1M@GGMNHJNL@?$AAz?$AAh?$AA?9?$AAS?$AAG@ 10026704     libucrt:lcidtoname_downlevel.obj
 0002:00007710       ??_C@_1M@HOIKODND@?$AAd?$AAe?$AA?9?$AAL?$AAU@ 10026710     libucrt:lcidtoname_downlevel.obj
 0002:0000771c       ??_C@_1M@DDOCCGFG@?$AAe?$AAn?$AA?9?$AAC?$AAA@ 1002671c     libucrt:lcidtoname_downlevel.obj
 0002:00007728       ??_C@_1M@BNOEMJLF@?$AAe?$AAs?$AA?9?$AAG?$AAT@ 10026728     libucrt:lcidtoname_downlevel.obj
 0002:00007734       ??_C@_1M@EOGNKEK@?$AAf?$AAr?$AA?9?$AAC?$AAH@ 10026734     libucrt:lcidtoname_downlevel.obj
 0002:00007740       ??_C@_1M@FLIDJFHL@?$AAh?$AAr?$AA?9?$AAB?$AAA@ 10026740     libucrt:lcidtoname_downlevel.obj
 0002:0000774c       ??_C@_1O@FMCELNAJ@?$AAs?$AAm?$AAj?$AA?9?$AAN?$AAO@ 1002674c     libucrt:lcidtoname_downlevel.obj
 0002:0000775c       ??_C@_1M@JHGLJMGJ@?$AAa?$AAr?$AA?9?$AAD?$AAZ@ 1002675c     libucrt:lcidtoname_downlevel.obj
 0002:00007768       ??_C@_1M@JKKFDCNP@?$AAz?$AAh?$AA?9?$AAM?$AAO@ 10026768     libucrt:lcidtoname_downlevel.obj
 0002:00007774       ??_C@_1M@GEEFALPE@?$AAd?$AAe?$AA?9?$AAL?$AAI@ 10026774     libucrt:lcidtoname_downlevel.obj
 0002:00007780       ??_C@_1M@IGEOFBG@?$AAe?$AAn?$AA?9?$AAN?$AAZ@ 10026780     libucrt:lcidtoname_downlevel.obj
 0002:0000778c       ??_C@_1M@KDBONEHP@?$AAe?$AAs?$AA?9?$AAC?$AAR@ 1002678c     libucrt:lcidtoname_downlevel.obj
 0002:00007798       ??_C@_1M@FHMDOHNN@?$AAf?$AAr?$AA?9?$AAL?$AAU@ 10026798     libucrt:lcidtoname_downlevel.obj
 0002:000077a4       ??_C@_1BG@NFKKMAFG@?$AAb?$AAs?$AA?9?$AAB?$AAA?$AA?9?$AAL?$AAa?$AAt?$AAn@ 100267a4     libucrt:lcidtoname_downlevel.obj
 0002:000077bc       ??_C@_1O@IMNBEMCI@?$AAs?$AAm?$AAj?$AA?9?$AAS?$AAE@ 100267bc     libucrt:lcidtoname_downlevel.obj
 0002:000077cc       ??_C@_1M@DHHMBNDP@?$AAa?$AAr?$AA?9?$AAM?$AAA@ 100267cc     libucrt:lcidtoname_downlevel.obj
 0002:000077d8       ??_C@_1M@BNBLJCGH@?$AAe?$AAn?$AA?9?$AAI?$AAE@ 100267d8     libucrt:lcidtoname_downlevel.obj
 0002:000077e4       ??_C@_1M@GEPAFMDL@?$AAe?$AAs?$AA?9?$AAP?$AAA@ 100267e4     libucrt:lcidtoname_downlevel.obj
 0002:000077f0       ??_C@_1M@OJONDMDL@?$AAf?$AAr?$AA?9?$AAM?$AAC@ 100267f0     libucrt:lcidtoname_downlevel.obj
 0002:000077fc       ??_C@_1BG@OBCNFJB@?$AAs?$AAr?$AA?9?$AAB?$AAA?$AA?9?$AAL?$AAa?$AAt?$AAn@ 100267fc     libucrt:lcidtoname_downlevel.obj
 0002:00007814       ??_C@_1O@KEMEEGPO@?$AAs?$AAm?$AAa?$AA?9?$AAN?$AAO@ 10026814     libucrt:lcidtoname_downlevel.obj
 0002:00007824       ??_C@_1M@ELMGFODK@?$AAa?$AAr?$AA?9?$AAT?$AAN@ 10026824     libucrt:lcidtoname_downlevel.obj
 0002:00007830       ??_C@_1M@BHDLHFAF@?$AAe?$AAn?$AA?9?$AAZ?$AAA@ 10026830     libucrt:lcidtoname_downlevel.obj
 0002:0000783c       ??_C@_1M@BMGIGLIF@?$AAe?$AAs?$AA?9?$AAD?$AAO@ 1002683c     libucrt:lcidtoname_downlevel.obj
 0002:00007848       ??_C@_1BG@CMBHIPBE@?$AAs?$AAr?$AA?9?$AAB?$AAA?$AA?9?$AAC?$AAy?$AAr?$AAl@ 10026848     libucrt:lcidtoname_downlevel.obj
 0002:00007860       ??_C@_1O@HEDBLHNP@?$AAs?$AAm?$AAa?$AA?9?$AAS?$AAE@ 10026860     libucrt:lcidtoname_downlevel.obj
 0002:00007870       ??_C@_1M@DAGCADIM@?$AAa?$AAr?$AA?9?$AAO?$AAM@ 10026870     libucrt:lcidtoname_downlevel.obj
 0002:0000787c       ??_C@_1M@FODLMICG@?$AAe?$AAn?$AA?9?$AAJ?$AAM@ 1002687c     libucrt:lcidtoname_downlevel.obj
 0002:00007888       ??_C@_1M@DNMLCIHB@?$AAe?$AAs?$AA?9?$AAV?$AAE@ 10026888     libucrt:lcidtoname_downlevel.obj
 0002:00007894       ??_C@_1O@EOKHMKJK@?$AAs?$AAm?$AAs?$AA?9?$AAF?$AAI@ 10026894     libucrt:lcidtoname_downlevel.obj
 0002:000078a4       ??_C@_1M@CAFJMKOF@?$AAa?$AAr?$AA?9?$AAY?$AAE@ 100268a4     libucrt:lcidtoname_downlevel.obj
 0002:000078b0       ??_C@_1M@CBFHIJLI@?$AAe?$AAn?$AA?9?$AAC?$AAB@ 100268b0     libucrt:lcidtoname_downlevel.obj
 0002:000078bc       ??_C@_1M@BGNFLDN@?$AAe?$AAs?$AA?9?$AAC?$AAO@ 100268bc     libucrt:lcidtoname_downlevel.obj
 0002:000078c8       ??_C@_1O@JMPHMAMC@?$AAs?$AAm?$AAn?$AA?9?$AAF?$AAI@ 100268c8     libucrt:lcidtoname_downlevel.obj
 0002:000078d8       ??_C@_1M@JLANABKE@?$AAa?$AAr?$AA?9?$AAS?$AAY@ 100268d8     libucrt:lcidtoname_downlevel.obj
 0002:000078e4       ??_C@_1M@HPKGCFGN@?$AAe?$AAn?$AA?9?$AAB?$AAZ@ 100268e4     libucrt:lcidtoname_downlevel.obj
 0002:000078f0       ??_C@_1M@OLJCMLGM@?$AAe?$AAs?$AA?9?$AAP?$AAE@ 100268f0     libucrt:lcidtoname_downlevel.obj
 0002:000078fc       ??_C@_1M@MKKGFKLE@?$AAa?$AAr?$AA?9?$AAJ?$AAO@ 100268fc     libucrt:lcidtoname_downlevel.obj
 0002:00007908       ??_C@_1M@EKPGLDNI@?$AAe?$AAn?$AA?9?$AAT?$AAT@ 10026908     libucrt:lcidtoname_downlevel.obj
 0002:00007914       ??_C@_1M@OONGHFHE@?$AAe?$AAs?$AA?9?$AAA?$AAR@ 10026914     libucrt:lcidtoname_downlevel.obj
 0002:00007920       ??_C@_1M@OOJFGBHE@?$AAa?$AAr?$AA?9?$AAL?$AAB@ 10026920     libucrt:lcidtoname_downlevel.obj
 0002:0000792c       ??_C@_1M@GCEJHNEG@?$AAe?$AAn?$AA?9?$AAZ?$AAW@ 1002692c     libucrt:lcidtoname_downlevel.obj
 0002:00007938       ??_C@_1M@JNOCAHJI@?$AAe?$AAs?$AA?9?$AAE?$AAC@ 10026938     libucrt:lcidtoname_downlevel.obj
 0002:00007944       ??_C@_1M@JEFHPGGB@?$AAa?$AAr?$AA?9?$AAK?$AAW@ 10026944     libucrt:lcidtoname_downlevel.obj
 0002:00007950       ??_C@_1M@MLKIBJOJ@?$AAe?$AAn?$AA?9?$AAP?$AAH@ 10026950     libucrt:lcidtoname_downlevel.obj
 0002:0000795c       ??_C@_1M@BDNIPEND@?$AAe?$AAs?$AA?9?$AAC?$AAL@ 1002695c     libucrt:lcidtoname_downlevel.obj
 0002:00007968       ??_C@_1M@MPNMEKBD@?$AAa?$AAr?$AA?9?$AAA?$AAE@ 10026968     libucrt:lcidtoname_downlevel.obj
 0002:00007974       ??_C@_1M@KBJALCPI@?$AAe?$AAs?$AA?9?$AAU?$AAY@ 10026974     libucrt:lcidtoname_downlevel.obj
 0002:00007980       ??_C@_1M@LLCCOAGA@?$AAa?$AAr?$AA?9?$AAB?$AAH@ 10026980     libucrt:lcidtoname_downlevel.obj
 0002:0000798c       ??_C@_1M@PBFNCDEL@?$AAe?$AAs?$AA?9?$AAP?$AAY@ 1002698c     libucrt:lcidtoname_downlevel.obj
 0002:00007998       ??_C@_1M@EDGINPNP@?$AAa?$AAr?$AA?9?$AAQ?$AAA@ 10026998     libucrt:lcidtoname_downlevel.obj
 0002:000079a4       ??_C@_1M@MKDBIIJI@?$AAe?$AAs?$AA?9?$AAB?$AAO@ 100269a4     libucrt:lcidtoname_downlevel.obj
 0002:000079b0       ??_C@_1M@CPKKEBLD@?$AAe?$AAs?$AA?9?$AAS?$AAV@ 100269b0     libucrt:lcidtoname_downlevel.obj
 0002:000079bc       ??_C@_1M@NDBGMMJL@?$AAe?$AAs?$AA?9?$AAH?$AAN@ 100269bc     libucrt:lcidtoname_downlevel.obj
 0002:000079c8       ??_C@_1M@JIJIBHDP@?$AAe?$AAs?$AA?9?$AAN?$AAI@ 100269c8     libucrt:lcidtoname_downlevel.obj
 0002:000079d4       ??_C@_1M@CGFMKEEK@?$AAe?$AAs?$AA?9?$AAP?$AAR@ 100269d4     libucrt:lcidtoname_downlevel.obj
 0002:000079e0       ??_C@_1O@ICJHKIIK@?$AAz?$AAh?$AA?9?$AAC?$AAH?$AAT@ 100269e0     libucrt:lcidtoname_downlevel.obj
 0002:000079f0       ??_C@_15CLNEJCE@?$AAs?$AAr@ 100269f0     libucrt:lcidtoname_downlevel.obj
 0002:00008118       ??_C@_1M@KAHEKEIG@?$AAa?$AAf?$AA?9?$AAz?$AAa@ 10027118     libucrt:lcidtoname_downlevel.obj
 0002:00008124       ??_C@_1M@GIECOABL@?$AAa?$AAr?$AA?9?$AAa?$AAe@ 10027124     libucrt:lcidtoname_downlevel.obj
 0002:00008130       ??_C@_1M@BMLMEKGI@?$AAa?$AAr?$AA?9?$AAb?$AAh@ 10027130     libucrt:lcidtoname_downlevel.obj
 0002:0000813c       ??_C@_1M@DAPFDGGB@?$AAa?$AAr?$AA?9?$AAd?$AAz@ 1002713c     libucrt:lcidtoname_downlevel.obj
 0002:00008148       ??_C@_1M@FJNKGKIG@?$AAa?$AAr?$AA?9?$AAe?$AAg@ 10027148     libucrt:lcidtoname_downlevel.obj
 0002:00008154       ??_C@_1M@FLGKKCLO@?$AAa?$AAr?$AA?9?$AAi?$AAq@ 10027154     libucrt:lcidtoname_downlevel.obj
 0002:00008160       ??_C@_1M@GNDIPALM@?$AAa?$AAr?$AA?9?$AAj?$AAo@ 10027160     libucrt:lcidtoname_downlevel.obj
 0002:0000816c       ??_C@_1M@DDMJFMGJ@?$AAa?$AAr?$AA?9?$AAk?$AAw@ 1002716c     libucrt:lcidtoname_downlevel.obj
 0002:00008178       ??_C@_1M@EJALMLHM@?$AAa?$AAr?$AA?9?$AAl?$AAb@ 10027178     libucrt:lcidtoname_downlevel.obj
 0002:00008184       ??_C@_1M@MOBDBLOC@?$AAa?$AAr?$AA?9?$AAl?$AAy@ 10027184     libucrt:lcidtoname_downlevel.obj
 0002:00008190       ??_C@_1M@JAOCLHDH@?$AAa?$AAr?$AA?9?$AAm?$AAa@ 10027190     libucrt:lcidtoname_downlevel.obj
 0002:0000819c       ??_C@_1M@JHPMKJIE@?$AAa?$AAr?$AA?9?$AAo?$AAm@ 1002719c     libucrt:lcidtoname_downlevel.obj
 0002:000081a8       ??_C@_1M@OEPGHFNH@?$AAa?$AAr?$AA?9?$AAq?$AAa@ 100271a8     libucrt:lcidtoname_downlevel.obj
 0002:000081b4       ??_C@_1M@KJDONENM@?$AAa?$AAr?$AA?9?$AAs?$AAa@ 100271b4     libucrt:lcidtoname_downlevel.obj
 0002:000081c0       ??_C@_1M@DMJDKLKM@?$AAa?$AAr?$AA?9?$AAs?$AAy@ 100271c0     libucrt:lcidtoname_downlevel.obj
 0002:000081cc       ??_C@_1M@OMFIPEDC@?$AAa?$AAr?$AA?9?$AAt?$AAn@ 100271cc     libucrt:lcidtoname_downlevel.obj
 0002:000081d8       ??_C@_1M@IHMHGAON@?$AAa?$AAr?$AA?9?$AAy?$AAe@ 100271d8     libucrt:lcidtoname_downlevel.obj
 0002:000081e4       ??_C@_1BG@KDCPGJGB@?$AAa?$AAz?$AA?9?$AAa?$AAz?$AA?9?$AAc?$AAy?$AAr?$AAl@ 100271e4     libucrt:lcidtoname_downlevel.obj
 0002:000081fc       ??_C@_1BG@IBCKDDOE@?$AAa?$AAz?$AA?9?$AAa?$AAz?$AA?9?$AAl?$AAa?$AAt?$AAn@ 100271fc     libucrt:lcidtoname_downlevel.obj
 0002:00008214       ??_C@_1M@EGPFDCPD@?$AAb?$AAe?$AA?9?$AAb?$AAy@ 10027214     libucrt:lcidtoname_downlevel.obj
 0002:00008220       ??_C@_1M@PCMGMCGC@?$AAb?$AAg?$AA?9?$AAb?$AAg@ 10027220     libucrt:lcidtoname_downlevel.obj
 0002:0000822c       ??_C@_1M@BJBMFGOB@?$AAb?$AAn?$AA?9?$AAi?$AAn@ 1002722c     libucrt:lcidtoname_downlevel.obj
 0002:00008238       ??_C@_1BG@EAKMMACD@?$AAb?$AAs?$AA?9?$AAb?$AAa?$AA?9?$AAl?$AAa?$AAt?$AAn@ 10027238     libucrt:lcidtoname_downlevel.obj
 0002:00008250       ??_C@_1M@KGADAODK@?$AAc?$AAa?$AA?9?$AAe?$AAs@ 10027250     libucrt:lcidtoname_downlevel.obj
 0002:0000825c       ??_C@_1M@COAJPDHI@?$AAc?$AAs?$AA?9?$AAc?$AAz@ 1002725c     libucrt:lcidtoname_downlevel.obj
 0002:00008268       ??_C@_1M@DHBHFONH@?$AAc?$AAy?$AA?9?$AAg?$AAb@ 10027268     libucrt:lcidtoname_downlevel.obj
 0002:00008274       ??_C@_1M@IMGKELGA@?$AAd?$AAa?$AA?9?$AAd?$AAk@ 10027274     libucrt:lcidtoname_downlevel.obj
 0002:00008280       ??_C@_1M@NNDGDNGA@?$AAd?$AAe?$AA?9?$AAa?$AAt@ 10027280     libucrt:lcidtoname_downlevel.obj
 0002:0000828c       ??_C@_1M@IKDBHEEM@?$AAd?$AAe?$AA?9?$AAc?$AAh@ 1002728c     libucrt:lcidtoname_downlevel.obj
 0002:00008298       ??_C@_1M@GFFOJMCJ@?$AAd?$AAe?$AA?9?$AAd?$AAe@ 10027298     libucrt:lcidtoname_downlevel.obj
 0002:000082a4       ??_C@_1M@MDNLKBPM@?$AAd?$AAe?$AA?9?$AAl?$AAi@ 100272a4     libucrt:lcidtoname_downlevel.obj
 0002:000082b0       ??_C@_1M@NJBEEJNL@?$AAd?$AAe?$AA?9?$AAl?$AAu@ 100272b0     libucrt:lcidtoname_downlevel.obj
 0002:000082bc       ??_C@_1O@GNNELBAP@?$AAd?$AAi?$AAv?$AA?9?$AAm?$AAv@ 100272bc     libucrt:lcidtoname_downlevel.obj
 0002:000082cc       ??_C@_1M@EJLEOGAE@?$AAe?$AAl?$AA?9?$AAg?$AAr@ 100272cc     libucrt:lcidtoname_downlevel.obj
 0002:000082d8       ??_C@_1M@GMPONJN@?$AAe?$AAn?$AA?9?$AAa?$AAu@ 100272d8     libucrt:lcidtoname_downlevel.obj
 0002:000082e4       ??_C@_1M@NIDIIPGF@?$AAe?$AAn?$AA?9?$AAb?$AAz@ 100272e4     libucrt:lcidtoname_downlevel.obj
 0002:000082f0       ??_C@_1M@JEHMIMFO@?$AAe?$AAn?$AA?9?$AAc?$AAa@ 100272f0     libucrt:lcidtoname_downlevel.obj
 0002:000082fc       ??_C@_1M@IGMJCDLA@?$AAe?$AAn?$AA?9?$AAc?$AAb@ 100272fc     libucrt:lcidtoname_downlevel.obj
 0002:00008308       ??_C@_1M@BNFIGBKG@?$AAe?$AAn?$AA?9?$AAg?$AAb@ 10027308     libucrt:lcidtoname_downlevel.obj
 0002:00008314       ??_C@_1M@LKIFDIGP@?$AAe?$AAn?$AA?9?$AAi?$AAe@ 10027314     libucrt:lcidtoname_downlevel.obj
 0002:00008320       ??_C@_1M@PJKFGCCO@?$AAe?$AAn?$AA?9?$AAj?$AAm@ 10027320     libucrt:lcidtoname_downlevel.obj
 0002:0000832c       ??_C@_1M@KPPKEPBO@?$AAe?$AAn?$AA?9?$AAn?$AAz@ 1002732c     libucrt:lcidtoname_downlevel.obj
 0002:00008338       ??_C@_1M@GMDGLDOB@?$AAe?$AAn?$AA?9?$AAp?$AAh@ 10027338     libucrt:lcidtoname_downlevel.obj
 0002:00008344       ??_C@_1M@ONGIBJNA@?$AAe?$AAn?$AA?9?$AAt?$AAt@ 10027344     libucrt:lcidtoname_downlevel.obj
 0002:00008350       ??_C@_1M@LLODPCMM@?$AAe?$AAn?$AA?9?$AAu?$AAs@ 10027350     libucrt:lcidtoname_downlevel.obj
 0002:0000835c       ??_C@_1M@LAKFNPAN@?$AAe?$AAn?$AA?9?$AAz?$AAa@ 1002735c     libucrt:lcidtoname_downlevel.obj
 0002:00008368       ??_C@_1M@MFNHNHEO@?$AAe?$AAn?$AA?9?$AAz?$AAw@ 10027368     libucrt:lcidtoname_downlevel.obj
 0002:00008374       ??_C@_1M@EJEINPHM@?$AAe?$AAs?$AA?9?$AAa?$AAr@ 10027374     libucrt:lcidtoname_downlevel.obj
 0002:00008380       ??_C@_1M@GNKPCCJA@?$AAe?$AAs?$AA?9?$AAb?$AAo@ 10027380     libucrt:lcidtoname_downlevel.obj
 0002:0000838c       ??_C@_1M@LEEGFONL@?$AAe?$AAs?$AA?9?$AAc?$AAl@ 1002738c     libucrt:lcidtoname_downlevel.obj
 0002:00008398       ??_C@_1M@KGPDPBDF@?$AAe?$AAs?$AA?9?$AAc?$AAo@ 10027398     libucrt:lcidtoname_downlevel.obj
 0002:000083a4       ??_C@_1M@EIAHOHH@?$AAe?$AAs?$AA?9?$AAc?$AAr@ 100273a4     libucrt:lcidtoname_downlevel.obj
 0002:000083b0       ??_C@_1M@LLPGMBIN@?$AAe?$AAs?$AA?9?$AAd?$AAo@ 100273b0     libucrt:lcidtoname_downlevel.obj
 0002:000083bc       ??_C@_1M@DKHMKNJA@?$AAe?$AAs?$AA?9?$AAe?$AAc@ 100273bc     libucrt:lcidtoname_downlevel.obj
 0002:000083c8       ??_C@_1M@GKGFPKAP@?$AAe?$AAs?$AA?9?$AAe?$AAs@ 100273c8     libucrt:lcidtoname_downlevel.obj
 0002:000083d4       ??_C@_1M@LKHKGDLN@?$AAe?$AAs?$AA?9?$AAg?$AAt@ 100273d4     libucrt:lcidtoname_downlevel.obj
 0002:000083e0       ??_C@_1M@HEIIGGJD@?$AAe?$AAs?$AA?9?$AAh?$AAn@ 100273e0     libucrt:lcidtoname_downlevel.obj
 0002:000083ec       ??_C@_1M@FBDHPPGD@?$AAe?$AAs?$AA?9?$AAm?$AAx@ 100273ec     libucrt:lcidtoname_downlevel.obj
 0002:000083f8       ??_C@_1M@DPAGLNDH@?$AAe?$AAs?$AA?9?$AAn?$AAi@ 100273f8     libucrt:lcidtoname_downlevel.obj
 0002:00008404       ??_C@_1M@MDGOPGDD@?$AAe?$AAs?$AA?9?$AAp?$AAa@ 10027404     libucrt:lcidtoname_downlevel.obj
 0002:00008410       ??_C@_1M@EMAMGBGE@?$AAe?$AAs?$AA?9?$AAp?$AAe@ 10027410     libucrt:lcidtoname_downlevel.obj
 0002:0000841c       ??_C@_1M@IBMCAOEC@?$AAe?$AAs?$AA?9?$AAp?$AAr@ 1002741c     libucrt:lcidtoname_downlevel.obj
 0002:00008428       ??_C@_1M@FGMDIJED@?$AAe?$AAs?$AA?9?$AAp?$AAy@ 10027428     libucrt:lcidtoname_downlevel.obj
 0002:00008434       ??_C@_1M@IIDEOLLL@?$AAe?$AAs?$AA?9?$AAs?$AAv@ 10027434     libucrt:lcidtoname_downlevel.obj
 0002:00008440       ??_C@_1M@GAOBIPA@?$AAe?$AAs?$AA?9?$AAu?$AAy@ 10027440     libucrt:lcidtoname_downlevel.obj
 0002:0000844c       ??_C@_1M@JKFFICHJ@?$AAe?$AAs?$AA?9?$AAv?$AAe@ 1002744c     libucrt:lcidtoname_downlevel.obj
 0002:00008458       ??_C@_1M@PNMLOJDF@?$AAe?$AAt?$AA?9?$AAe?$AAe@ 10027458     libucrt:lcidtoname_downlevel.obj
 0002:00008464       ??_C@_1M@GHHLIKEI@?$AAe?$AAu?$AA?9?$AAe?$AAs@ 10027464     libucrt:lcidtoname_downlevel.obj
 0002:00008470       ??_C@_1M@PBNONODE@?$AAf?$AAa?$AA?9?$AAi?$AAr@ 10027470     libucrt:lcidtoname_downlevel.obj
 0002:0000847c       ??_C@_1M@JEEHPMIL@?$AAf?$AAi?$AA?9?$AAf?$AAi@ 1002747c     libucrt:lcidtoname_downlevel.obj
 0002:00008488       ??_C@_1M@LMDCNDBA@?$AAf?$AAo?$AA?9?$AAf?$AAo@ 10027488     libucrt:lcidtoname_downlevel.obj
 0002:00008494       ??_C@_1M@JKEOHLDK@?$AAf?$AAr?$AA?9?$AAb?$AAe@ 10027494     libucrt:lcidtoname_downlevel.obj
 0002:000084a0       ??_C@_1M@NOHADPMI@?$AAf?$AAr?$AA?9?$AAc?$AAa@ 100274a0     libucrt:lcidtoname_downlevel.obj
 0002:000084ac       ??_C@_1M@KDHIHAEC@?$AAf?$AAr?$AA?9?$AAc?$AAh@ 100274ac     libucrt:lcidtoname_downlevel.obj
 0002:000084b8       ??_C@_1M@MMBBFGAK@?$AAf?$AAr?$AA?9?$AAf?$AAr@ 100274b8     libucrt:lcidtoname_downlevel.obj
 0002:000084c4       ??_C@_1M@PAFNENNF@?$AAf?$AAr?$AA?9?$AAl?$AAu@ 100274c4     libucrt:lcidtoname_downlevel.obj
 0002:000084d0       ??_C@_1M@EOHDJGDD@?$AAf?$AAr?$AA?9?$AAm?$AAc@ 100274d0     libucrt:lcidtoname_downlevel.obj
 0002:000084dc       ??_C@_1M@FAPLLOPF@?$AAg?$AAl?$AA?9?$AAe?$AAs@ 100274dc     libucrt:lcidtoname_downlevel.obj
 0002:000084e8       ??_C@_1M@FOPBFLOO@?$AAg?$AAu?$AA?9?$AAi?$AAn@ 100274e8     libucrt:lcidtoname_downlevel.obj
 0002:000084f4       ??_C@_1M@KBMCINPM@?$AAh?$AAe?$AA?9?$AAi?$AAl@ 100274f4     libucrt:lcidtoname_downlevel.obj
 0002:00008500       ??_C@_1M@BBPHKFPJ@?$AAh?$AAi?$AA?9?$AAi?$AAn@ 10027500     libucrt:lcidtoname_downlevel.obj
 0002:0000850c       ??_C@_1M@PMBNDPHD@?$AAh?$AAr?$AA?9?$AAb?$AAa@ 1002750c     libucrt:lcidtoname_downlevel.obj
 0002:00008518       ??_C@_1M@BPCKOEGE@?$AAh?$AAr?$AA?9?$AAh?$AAr@ 10027518     libucrt:lcidtoname_downlevel.obj
 0002:00008524       ??_C@_1M@GACBMHKE@?$AAh?$AAu?$AA?9?$AAh?$AAu@ 10027524     libucrt:lcidtoname_downlevel.obj
 0002:00008530       ??_C@_1M@MILPAJJC@?$AAh?$AAy?$AA?9?$AAa?$AAm@ 10027530     libucrt:lcidtoname_downlevel.obj
 0002:0000853c       ??_C@_1M@BABBICEC@?$AAi?$AAd?$AA?9?$AAi?$AAd@ 1002753c     libucrt:lcidtoname_downlevel.obj
 0002:00008548       ??_C@_1M@BIKNHHPF@?$AAi?$AAs?$AA?9?$AAi?$AAs@ 10027548     libucrt:lcidtoname_downlevel.obj
 0002:00008554       ??_C@_1M@NMPCJPHE@?$AAi?$AAt?$AA?9?$AAc?$AAh@ 10027554     libucrt:lcidtoname_downlevel.obj
 0002:00008560       ??_C@_1M@GHKGFEDF@?$AAi?$AAt?$AA?9?$AAi?$AAt@ 10027560     libucrt:lcidtoname_downlevel.obj
 0002:0000856c       ??_C@_1M@NIEJCJJA@?$AAj?$AAa?$AA?9?$AAj?$AAp@ 1002756c     libucrt:lcidtoname_downlevel.obj
 0002:00008578       ??_C@_1M@JILFNBIM@?$AAk?$AAa?$AA?9?$AAg?$AAe@ 10027578     libucrt:lcidtoname_downlevel.obj
 0002:00008584       ??_C@_1M@PACPMGPH@?$AAk?$AAk?$AA?9?$AAk?$AAz@ 10027584     libucrt:lcidtoname_downlevel.obj
 0002:00008590       ??_C@_1M@IELFGMHA@?$AAk?$AAn?$AA?9?$AAi?$AAn@ 10027590     libucrt:lcidtoname_downlevel.obj
 0002:0000859c       ??_C@_1O@IBBJHCH@?$AAk?$AAo?$AAk?$AA?9?$AAi?$AAn@ 1002759c     libucrt:lcidtoname_downlevel.obj
 0002:000085ac       ??_C@_1M@DMHAEOGC@?$AAk?$AAo?$AA?9?$AAk?$AAr@ 100275ac     libucrt:lcidtoname_downlevel.obj
 0002:000085b8       ??_C@_1M@HBAHBIGA@?$AAk?$AAy?$AA?9?$AAk?$AAg@ 100275b8     libucrt:lcidtoname_downlevel.obj
 0002:000085c4       ??_C@_1M@KPMILCJG@?$AAl?$AAt?$AA?9?$AAl?$AAt@ 100275c4     libucrt:lcidtoname_downlevel.obj
 0002:000085d0       ??_C@_1M@BDEKKCA@?$AAl?$AAv?$AA?9?$AAl?$AAv@ 100275d0     libucrt:lcidtoname_downlevel.obj
 0002:000085dc       ??_C@_1M@ELCKCCJJ@?$AAm?$AAi?$AA?9?$AAn?$AAz@ 100275dc     libucrt:lcidtoname_downlevel.obj
 0002:000085e8       ??_C@_1M@CBOOLAPA@?$AAm?$AAk?$AA?9?$AAm?$AAk@ 100275e8     libucrt:lcidtoname_downlevel.obj
 0002:000085f4       ??_C@_1M@GPHNBJKN@?$AAm?$AAl?$AA?9?$AAi?$AAn@ 100275f4     libucrt:lcidtoname_downlevel.obj
 0002:00008600       ??_C@_1M@PABJILIG@?$AAm?$AAn?$AA?9?$AAm?$AAn@ 10027600     libucrt:lcidtoname_downlevel.obj
 0002:0000860c       ??_C@_1M@FGBKKIPG@?$AAm?$AAr?$AA?9?$AAi?$AAn@ 1002760c     libucrt:lcidtoname_downlevel.obj
 0002:00008618       ??_C@_1M@NDBPDDAL@?$AAm?$AAs?$AA?9?$AAb?$AAn@ 10027618     libucrt:lcidtoname_downlevel.obj
 0002:00008624       ??_C@_1M@OPIHOOPI@?$AAm?$AAs?$AA?9?$AAm?$AAy@ 10027624     libucrt:lcidtoname_downlevel.obj
 0002:00008630       ??_C@_1M@PPDBCNFM@?$AAm?$AAt?$AA?9?$AAm?$AAt@ 10027630     libucrt:lcidtoname_downlevel.obj
 0002:0000863c       ??_C@_1M@KDJDKMDD@?$AAn?$AAb?$AA?9?$AAn?$AAo@ 1002763c     libucrt:lcidtoname_downlevel.obj
 0002:00008648       ??_C@_1M@KFCFLMJP@?$AAn?$AAl?$AA?9?$AAb?$AAe@ 10027648     libucrt:lcidtoname_downlevel.obj
 0002:00008654       ??_C@_1M@KPOPDDGO@?$AAn?$AAl?$AA?9?$AAn?$AAl@ 10027654     libucrt:lcidtoname_downlevel.obj
 0002:00008660       ??_C@_1M@LJKPEMLN@?$AAn?$AAn?$AA?9?$AAn?$AAo@ 10027660     libucrt:lcidtoname_downlevel.obj
 0002:0000866c       ??_C@_1M@BDGHHBFL@?$AAn?$AAs?$AA?9?$AAz?$AAa@ 1002766c     libucrt:lcidtoname_downlevel.obj
 0002:00008678       ??_C@_1M@IDEHOAP@?$AAp?$AAa?$AA?9?$AAi?$AAn@ 10027678     libucrt:lcidtoname_downlevel.obj
 0002:00008684       ??_C@_1M@HDBKGOGH@?$AAp?$AAl?$AA?9?$AAp?$AAl@ 10027684     libucrt:lcidtoname_downlevel.obj
 0002:00008690       ??_C@_1M@LJLLCMEH@?$AAp?$AAt?$AA?9?$AAb?$AAr@ 10027690     libucrt:lcidtoname_downlevel.obj
 0002:0000869c       ??_C@_1M@NCMONAAL@?$AAp?$AAt?$AA?9?$AAp?$AAt@ 1002769c     libucrt:lcidtoname_downlevel.obj
 0002:000086a8       ??_C@_1O@EAKMAJDN@?$AAq?$AAu?$AAz?$AA?9?$AAb?$AAo@ 100276a8     libucrt:lcidtoname_downlevel.obj
 0002:000086b8       ??_C@_1O@BHHPIGDN@?$AAq?$AAu?$AAz?$AA?9?$AAe?$AAc@ 100276b8     libucrt:lcidtoname_downlevel.obj
 0002:000086c8       ??_C@_1O@GBAPEKMJ@?$AAq?$AAu?$AAz?$AA?9?$AAp?$AAe@ 100276c8     libucrt:lcidtoname_downlevel.obj
 0002:000086d8       ??_C@_1M@CLGLEFBO@?$AAr?$AAo?$AA?9?$AAr?$AAo@ 100276d8     libucrt:lcidtoname_downlevel.obj
 0002:000086e4       ??_C@_1M@CEEDODME@?$AAr?$AAu?$AA?9?$AAr?$AAu@ 100276e4     libucrt:lcidtoname_downlevel.obj
 0002:000086f0       ??_C@_1M@HPKKKMPP@?$AAs?$AAa?$AA?9?$AAi?$AAn@ 100276f0     libucrt:lcidtoname_downlevel.obj
 0002:000086fc       ??_C@_1M@BKMAIGOJ@?$AAs?$AAe?$AA?9?$AAf?$AAi@ 100276fc     libucrt:lcidtoname_downlevel.obj
 0002:00008708       ??_C@_1M@NDPIFLFI@?$AAs?$AAe?$AA?9?$AAn?$AAo@ 10027708     libucrt:lcidtoname_downlevel.obj
 0002:00008714       ??_C@_1M@DANKKHJ@?$AAs?$AAe?$AA?9?$AAs?$AAe@ 10027714     libucrt:lcidtoname_downlevel.obj
 0002:00008720       ??_C@_1M@PNBLONPJ@?$AAs?$AAk?$AA?9?$AAs?$AAk@ 10027720     libucrt:lcidtoname_downlevel.obj
 0002:0000872c       ??_C@_1M@LFMODOAL@?$AAs?$AAl?$AA?9?$AAs?$AAi@ 1002772c     libucrt:lcidtoname_downlevel.obj
 0002:00008738       ??_C@_1O@DFKOMPG@?$AAs?$AAm?$AAa?$AA?9?$AAn?$AAo@ 10027738     libucrt:lcidtoname_downlevel.obj
 0002:00008748       ??_C@_1O@NDKPBNNH@?$AAs?$AAm?$AAa?$AA?9?$AAs?$AAe@ 10027748     libucrt:lcidtoname_downlevel.obj
 0002:00008758       ??_C@_1O@PLLKBHAB@?$AAs?$AAm?$AAj?$AA?9?$AAn?$AAo@ 10027758     libucrt:lcidtoname_downlevel.obj
 0002:00008768       ??_C@_1O@CLEPOGCA@?$AAs?$AAm?$AAj?$AA?9?$AAs?$AAe@ 10027768     libucrt:lcidtoname_downlevel.obj
 0002:00008778       ??_C@_1O@DLGJGKMK@?$AAs?$AAm?$AAn?$AA?9?$AAf?$AAi@ 10027778     libucrt:lcidtoname_downlevel.obj
 0002:00008788       ??_C@_1O@OJDJGAJC@?$AAs?$AAm?$AAs?$AA?9?$AAf?$AAi@ 10027788     libucrt:lcidtoname_downlevel.obj
 0002:00008798       ??_C@_1M@BOFOGHPB@?$AAs?$AAq?$AA?9?$AAa?$AAl@ 10027798     libucrt:lcidtoname_downlevel.obj
 0002:000087a4       ??_C@_1BG@LJBBIPGB@?$AAs?$AAr?$AA?9?$AAb?$AAa?$AA?9?$AAc?$AAy?$AAr?$AAl@ 100277a4     libucrt:lcidtoname_downlevel.obj
 0002:000087bc       ??_C@_1BG@JLBENFOE@?$AAs?$AAr?$AA?9?$AAb?$AAa?$AA?9?$AAl?$AAa?$AAt?$AAn@ 100277bc     libucrt:lcidtoname_downlevel.obj
 0002:000087d4       ??_C@_1BG@KODPNHE@?$AAs?$AAr?$AA?9?$AAs?$AAp?$AA?9?$AAc?$AAy?$AAr?$AAl@ 100277d4     libucrt:lcidtoname_downlevel.obj
 0002:000087ec       ??_C@_1BG@CIOGKHPB@?$AAs?$AAr?$AA?9?$AAs?$AAp?$AA?9?$AAl?$AAa?$AAt?$AAn@ 100277ec     libucrt:lcidtoname_downlevel.obj
 0002:00008804       ??_C@_1M@NGFJLMAC@?$AAs?$AAv?$AA?9?$AAf?$AAi@ 10027804     libucrt:lcidtoname_downlevel.obj
 0002:00008810       ??_C@_1M@MPJEJAJC@?$AAs?$AAv?$AA?9?$AAs?$AAe@ 10027810     libucrt:lcidtoname_downlevel.obj
 0002:0000881c       ??_C@_1M@MPNDHLFK@?$AAs?$AAw?$AA?9?$AAk?$AAe@ 1002781c     libucrt:lcidtoname_downlevel.obj
 0002:00008828       ??_C@_1O@KOHBJJI@?$AAs?$AAy?$AAr?$AA?9?$AAs?$AAy@ 10027828     libucrt:lcidtoname_downlevel.obj
 0002:00008838       ??_C@_1M@LDCEFHA@?$AAt?$AAa?$AA?9?$AAi?$AAn@ 10027838     libucrt:lcidtoname_downlevel.obj
 0002:00008844       ??_C@_1M@CNJOFAK@?$AAt?$AAe?$AA?9?$AAi?$AAn@ 10027844     libucrt:lcidtoname_downlevel.obj
 0002:00008850       ??_C@_1M@GNAECACD@?$AAt?$AAh?$AA?9?$AAt?$AAh@ 10027850     libucrt:lcidtoname_downlevel.obj
 0002:0000885c       ??_C@_1M@CHBIHOJO@?$AAt?$AAn?$AA?9?$AAz?$AAa@ 1002785c     libucrt:lcidtoname_downlevel.obj
 0002:00008868       ??_C@_1M@GCCMIGPJ@?$AAt?$AAr?$AA?9?$AAt?$AAr@ 10027868     libucrt:lcidtoname_downlevel.obj
 0002:00008874       ??_C@_1M@CELMCNBK@?$AAt?$AAt?$AA?9?$AAr?$AAu@ 10027874     libucrt:lcidtoname_downlevel.obj
 0002:00008880       ??_C@_1M@KLMCELGA@?$AAu?$AAk?$AA?9?$AAu?$AAa@ 10027880     libucrt:lcidtoname_downlevel.obj
 0002:0000888c       ??_C@_1M@EPAJJAJF@?$AAu?$AAr?$AA?9?$AAp?$AAk@ 1002788c     libucrt:lcidtoname_downlevel.obj
 0002:00008898       ??_C@_1BG@GEGPMCDJ@?$AAu?$AAz?$AA?9?$AAu?$AAz?$AA?9?$AAc?$AAy?$AAr?$AAl@ 10027898     libucrt:lcidtoname_downlevel.obj
 0002:000088b0       ??_C@_1BG@EGGKJILM@?$AAu?$AAz?$AA?9?$AAu?$AAz?$AA?9?$AAl?$AAa?$AAt?$AAn@ 100278b0     libucrt:lcidtoname_downlevel.obj
 0002:000088c8       ??_C@_1M@GFOCLFF@?$AAv?$AAi?$AA?9?$AAv?$AAn@ 100278c8     libucrt:lcidtoname_downlevel.obj
 0002:000088d4       ??_C@_1M@CPAMEDFI@?$AAx?$AAh?$AA?9?$AAz?$AAa@ 100278d4     libucrt:lcidtoname_downlevel.obj
 0002:000088e0       ??_C@_1O@EBKIFIGN@?$AAz?$AAh?$AA?9?$AAc?$AAh?$AAs@ 100278e0     libucrt:lcidtoname_downlevel.obj
 0002:000088f0       ??_C@_1O@NMHPGANE@?$AAz?$AAh?$AA?9?$AAc?$AAh?$AAt@ 100278f0     libucrt:lcidtoname_downlevel.obj
 0002:00008900       ??_C@_1M@LPINJOMC@?$AAz?$AAh?$AA?9?$AAc?$AAn@ 10027900     libucrt:lcidtoname_downlevel.obj
 0002:0000890c       ??_C@_1M@OCJEJODD@?$AAz?$AAh?$AA?9?$AAh?$AAk@ 1002790c     libucrt:lcidtoname_downlevel.obj
 0002:00008918       ??_C@_1M@DNDLJINH@?$AAz?$AAh?$AA?9?$AAm?$AAo@ 10027918     libucrt:lcidtoname_downlevel.obj
 0002:00008924       ??_C@_1M@MBFDNDND@?$AAz?$AAh?$AA?9?$AAs?$AAg@ 10027924     libucrt:lcidtoname_downlevel.obj
 0002:00008930       ??_C@_1M@IMEPLEPE@?$AAz?$AAh?$AA?9?$AAt?$AAw@ 10027930     libucrt:lcidtoname_downlevel.obj
 0002:0000893c       ??_C@_1M@BBGHNHJP@?$AAz?$AAu?$AA?9?$AAz?$AAa@ 1002793c     libucrt:lcidtoname_downlevel.obj
 0002:00008948       ?large_power_data@?1??multiply_by_power_of_ten@__crt_strtox@@YA_NAAUbig_integer@2@I@Z@4QBIB 10027948     libucrt:cfout.obj
 0002:00009250       ?large_power_indices@?1??multiply_by_power_of_ten@__crt_strtox@@YA_NAAUbig_integer@2@I@Z@4QBUunpack_index@?1??12@YA_N0I@Z@B 10028250     libucrt:cfout.obj
 0002:000092e8       ?small_powers_of_ten@?1??multiply_by_power_of_ten@__crt_strtox@@YA_NAAUbig_integer@2@I@Z@4QBIB 100282e8     libucrt:cfout.obj
 0002:0000930c       ??_C@_05DNEBIAHO@1?$CDINF@ 1002830c     libucrt:cfout.obj
 0002:00009314       ??_C@_06IMKFLFPG@1?$CDQNAN@ 10028314     libucrt:cfout.obj
 0002:0000931c       ??_C@_06PGGFOGJG@1?$CDSNAN@ 1002831c     libucrt:cfout.obj
 0002:00009324       ??_C@_05PHHOCPM@1?$CDIND@  10028324     libucrt:cfout.obj
 0002:00009388       ??_C@_1BA@BALFACEM@?$AAC?$AAO?$AAN?$AAO?$AAU?$AAT?$AA$@ 10028388     libucrt:initcon.obj
 0002:000094a0       __infinity                 100284a0     libucrt:87tran.obj
 0002:000094aa       __minfinity                100284aa     libucrt:87tran.obj
 0002:000094b4       __logemax                  100284b4     libucrt:87tran.obj
 0002:000094da       __OP_EXPjmptab             100284da     libucrt:87tran.obj
 0002:00009500       __indefinite               10028500     libucrt:87disp.obj
 0002:0000950a       __piby2                    1002850a     libucrt:87disp.obj
 0002:00009514       __piby4                    10028514     libucrt:87disp.obj
 0002:00009548       __DEFAULT_CW_in_mem        10028548     libucrt:common.obj
 0002:0000954a       __pi_by_2_to_61            1002854a     libucrt:common.obj
 0002:00009584       ??_C@_03MGHMBJCF@log@      10028584     libucrt:libm_error.obj
 0002:00009588       ??_C@_05HGHHAHAP@log10@    10028588     libucrt:libm_error.obj
 0002:00009590       ??_C@_03KHJOGHMM@exp@      10028590     libucrt:libm_error.obj
 0002:00009594       ??_C@_03JGHBODFD@pow@      10028594     libucrt:libm_error.obj
 0002:00009598       ??_C@_04FIHNOPOL@asin@     10028598     libucrt:libm_error.obj
 0002:000095a0       ??_C@_04PDIFKINK@acos@     100285a0     libucrt:libm_error.obj
 0002:000095a8       ??_C@_04EIAKFFMI@sqrt@     100285a8     libucrt:libm_error.obj
 0002:000095b0       __real@3ff0000000000000    100285b0     libucrt:libm_error.obj
 0002:000095d0       ___acrt_log10_table_t      100285d0     libucrt:log10_tables.obj
 0002:000099e0       ___acrt_log10_table_cb     100289e0     libucrt:log10_tables.obj
 0002:00009df0       __real@3fe0000000000000    10028df0     libucrt:powhlp.obj
 0002:00009ee0       ??_C@_04COOMCNPB@sinh@     10028ee0     libucrt:fpexcept.obj
 0002:00009ee8       ??_C@_04HPJJNFIM@cosh@     10028ee8     libucrt:fpexcept.obj
 0002:00009ef0       ??_C@_04FJHINJAO@tanh@     10028ef0     libucrt:fpexcept.obj
 0002:00009ef8       ??_C@_04MLLJIGOK@atan@     10028ef8     libucrt:fpexcept.obj
 0002:00009f00       ??_C@_05KNGEOGJB@atan2@    10028f00     libucrt:fpexcept.obj
 0002:00009f08       ??_C@_03BLEJJJBH@sin@      10028f08     libucrt:fpexcept.obj
 0002:00009f0c       ??_C@_03LALBNOCG@cos@      10028f0c     libucrt:fpexcept.obj
 0002:00009f10       ??_C@_03IIINPABG@tan@      10028f10     libucrt:fpexcept.obj
 0002:00009f14       ??_C@_04GFPJNGEK@ceil@     10028f14     libucrt:fpexcept.obj
 0002:00009f1c       ??_C@_05PBJFFIGL@floor@    10028f1c     libucrt:fpexcept.obj
 0002:00009f24       ??_C@_04ODHECPBC@fabs@     10028f24     libucrt:fpexcept.obj
 0002:00009f2c       ??_C@_04EHEDPDJG@modf@     10028f2c     libucrt:fpexcept.obj
 0002:00009f34       ??_C@_05CEJMAHNP@ldexp@    10028f34     libucrt:fpexcept.obj
 0002:00009f3c       ??_C@_05KBKMEMPO@_cabs@    10028f3c     libucrt:fpexcept.obj
 0002:00009f44       ??_C@_06MEIMCGCF@_hypot@   10028f44     libucrt:fpexcept.obj
 0002:00009f4c       ??_C@_04KEPJIHGP@fmod@     10028f4c     libucrt:fpexcept.obj
 0002:00009f54       ??_C@_05GKKHEGJL@frexp@    10028f54     libucrt:fpexcept.obj
 0002:00009f5c       ??_C@_03MJLDFKDL@_y0@      10028f5c     libucrt:fpexcept.obj
 0002:00009f60       ??_C@_03NAKIGLHK@_y1@      10028f60     libucrt:fpexcept.obj
 0002:00009f64       ??_C@_03ONILCKOB@_yn@      10028f64     libucrt:fpexcept.obj
 0002:00009f68       ??_C@_05JGDBENOH@_logb@    10028f68     libucrt:fpexcept.obj
 0002:00009f70       ??_C@_0L@KDOEJCKC@_nextafter@ 10028f70     libucrt:fpexcept.obj
 0002:00009f80       __d_inf                    10028f80     libucrt:util.obj
 0002:00009f88       __d_max                    10028f88     libucrt:util.obj
 0002:00009f90       __d_mzero                  10028f90     libucrt:util.obj
 0002:00009f9c       ??_7type_info@@6B@         10028f9c     LIBCMT:std_type_info_static.obj
 0002:00009fb0       __load_config_used         10028fb0     LIBCMT:loadcfg.obj
 0002:0000a100       ??_R4exception@std@@6B@    10029100     libvcruntime:frame.obj
 0002:0000a114       ??_R3exception@std@@8      10029114     libvcruntime:frame.obj
 0002:0000a124       ??_R2exception@std@@8      10029124     libvcruntime:frame.obj
 0002:0000a12c       ??_R1A@?0A@EA@exception@std@@8 1002912c     libvcruntime:frame.obj
 0002:0000a148       ??_R4bad_exception@std@@6B@ 10029148     libvcruntime:frame.obj
 0002:0000a15c       ??_R3bad_exception@std@@8  1002915c     libvcruntime:frame.obj
 0002:0000a16c       ??_R2bad_exception@std@@8  1002916c     libvcruntime:frame.obj
 0002:0000a178       ??_R1A@?0A@EA@bad_exception@std@@8 10029178     libvcruntime:frame.obj
 0002:0000a194       ??_R4type_info@@6B@        10029194     LIBCMT:std_type_info_static.obj
 0002:0000a1a8       ??_R3type_info@@8          100291a8     LIBCMT:std_type_info_static.obj
 0002:0000a1b8       ??_R2type_info@@8          100291b8     LIBCMT:std_type_info_static.obj
 0002:0000a1c0       ??_R1A@?0A@EA@type_info@@8 100291c0     LIBCMT:std_type_info_static.obj
 0002:0000a1dc       ___safe_se_handler_table   100291dc     <linker-defined>
 0002:0000a204       ___volatile_metadata       10029204     <linker-defined>
 0002:0000a754       ___rtc_iaa                 10029754     LIBCMT:initsect.obj
 0002:0000a758       ___rtc_izz                 10029758     LIBCMT:initsect.obj
 0002:0000a75c       ___rtc_taa                 1002975c     LIBCMT:initsect.obj
 0002:0000a760       ___rtc_tzz                 10029760     LIBCMT:initsect.obj
 0002:0000a8f4       __TI2?AVbad_exception@std@@ 100298f4     libvcruntime:frame.obj
 0002:0000a904       __CTA2?AVbad_exception@std@@ 10029904     libvcruntime:frame.obj
 0002:0000a910       __CT??_R0?AVbad_exception@std@@@8??0bad_exception@std@@QAE@ABV01@@Z12 10029910     libvcruntime:frame.obj
 0002:0000a92c       __CT??_R0?AVexception@std@@@8??0exception@std@@QAE@ABV01@@Z12 1002992c     libvcruntime:frame.obj
 0002:0000b168       __IMPORT_DESCRIPTOR_KERNEL32 1002a168     kernel32:KERNEL32.dll
 0002:0000b17c       __NULL_IMPORT_DESCRIPTOR   1002a17c     kernel32:KERNEL32.dll
 0003:00000004       ___security_cookie_complement 1002b004     LIBCMT:gs_cookie.obj
 0003:00000008       ___security_cookie         1002b008     LIBCMT:gs_cookie.obj
 0003:00000010       ___scrt_native_dllmain_reason 1002b010     LIBCMT:utility.obj
 0003:00000020       ___isa_enabled             1002b020     LIBCMT:cpu_disp.obj
 0003:00000040       __NLG_Destination          1002b040     libvcruntime:exsup.obj
 0003:00000050       __iob                      1002b050     libucrt:_file.obj
 0003:00000110       __lookuptrailbytes         1002b110     libucrt:read.obj
 0003:00000210       ___abort_behavior          1002b210     libucrt:abort.obj
 0003:00000228       ___acrt_initial_locale_data 1002b228     libucrt:nlsdata.obj
 0003:000002e0       ___acrt_initial_locale_pointers 1002b2e0     libucrt:nlsdata.obj
 0003:000002e8       ___acrt_wide_c_locale_string 1002b2e8     libucrt:nlsdata.obj
 0003:000002f0       ___badioinfo               1002b2f0     libucrt:ioinit.obj
 0003:00000328       ___acrt_initial_multibyte_data 1002b328     libucrt:mbctype.obj
 0003:00000848       ___globallocalestatus      1002b848     libucrt:glstatus.obj
 0003:00000850       ___acrt_lconv_c            1002b850     libucrt:localeconv.obj
 0003:000008a0       ___acrt_lconv_static_decimal 1002b8a0     libucrt:localeconv.obj
 0003:000008a4       ___acrt_lconv_static_W_decimal 1002b8a4     libucrt:localeconv.obj
 0003:000008d0       __fltused                  1002b8d0     LIBCMT:fltused.obj
 0003:000008e0       ??_R0?AVbad_exception@std@@@8 1002b8e0     libvcruntime:frame.obj
 0003:00000900       ??_R0?AVexception@std@@@8  1002b900     libvcruntime:frame.obj
 0003:0000091c       ??_R0?AVtype_info@@@8      1002b91c     LIBCMT:std_type_info_static.obj
 0003:00000c90       ?__type_info_root_node@@3U__type_info_node@@A 1002bc90     LIBCMT:tncleanup.obj
 0003:00000c98       ?_OptionsStorage@?1??__local_stdio_scanf_options@@9@4_KA 1002bc98     LIBCMT:default_local_stdio_options.obj
 0003:00000ca0       ___scrt_current_native_startup_state 1002bca0     LIBCMT:utility.obj
 0003:00000ca4       ___scrt_native_startup_lock 1002bca4     LIBCMT:utility.obj
 0003:00000cc4       ___scrt_debugger_hook_flag 1002bcc4     LIBCMT:utility_desktop.obj
 0003:00000cc8       ___isa_available           1002bcc8     LIBCMT:cpu_disp.obj
 0003:00000ccc       ___favor                   1002bccc     LIBCMT:cpu_disp.obj
 0003:00000cd0       ?__WinRTOutOfMemoryExceptionCallback@@3P6GPAXXZA 1002bcd0     libvcruntime:ehhelpers.obj
 0003:00000cd4       ?pArgList@UnDecorator@@0PAVReplicator@@A 1002bcd4     libvcruntime:undname.obj
 0003:00000cd8       ?pZNameList@UnDecorator@@0PAVReplicator@@A 1002bcd8     libvcruntime:undname.obj
 0003:00000cdc       ?pTemplateArgList@UnDecorator@@0PAVReplicator@@A 1002bcdc     libvcruntime:undname.obj
 0003:00000ce0       ?gName@UnDecorator@@0PBDB  1002bce0     libvcruntime:undname.obj
 0003:00000ce4       ?name@UnDecorator@@0PBDB   1002bce4     libvcruntime:undname.obj
 0003:00000ce8       ?disableFlags@UnDecorator@@0KA 1002bce8     libvcruntime:undname.obj
 0003:00000cec       ?fExplicitTemplateParams@UnDecorator@@0_NA 1002bcec     libvcruntime:undname.obj
 0003:00000ced       ?fGetTemplateArgumentList@UnDecorator@@0_NA 1002bced     libvcruntime:undname.obj
 0003:00000cf0       ?m_pGetParameter@UnDecorator@@0P6APADJ@ZA 1002bcf0     libvcruntime:undname.obj
 0003:00000cf4       ?m_CHPENameOffset@UnDecorator@@0KA 1002bcf4     libvcruntime:undname.obj
 0003:00000cf8       ?m_recursionLevel@UnDecorator@@0KA 1002bcf8     libvcruntime:undname.obj
 0003:00000d74       ___pPurecall               1002bd74     libvcruntime:purevirt_data.obj
 0003:00000d78       __nstream                  1002bd78     libucrt:_file.obj
 0003:00000d7c       ___piob                    1002bd7c     libucrt:_file.obj
 0003:00000d80       __cflush                   1002bd80     libucrt:_file.obj
 0003:00000e98       __environ_table            1002be98     libucrt:environment_initialization.obj
 0003:00000e9c       __wenviron_table           1002be9c     libucrt:environment_initialization.obj
 0003:00000ea0       ___dcrt_initial_wide_environment 1002bea0     libucrt:environment_initialization.obj
 0003:00000ea4       ___dcrt_initial_narrow_environment 1002bea4     libucrt:environment_initialization.obj
 0003:00000ea8       ___acrt_atexit_table       1002bea8     libucrt:onexit.obj
 0003:00000eb4       ___acrt_at_quick_exit_table 1002beb4     libucrt:onexit.obj
 0003:00000ec4       ___acrt_locale_changed_data 1002bec4     libucrt:wsetlocale.obj
 0003:00000ec8       ___acrt_current_locale_data 1002bec8     libucrt:nlsdata.obj
 0003:00000fb8       ___pioinfo                 1002bfb8     libucrt:ioinit.obj
 0003:000011b8       __nhandle                  1002c1b8     libucrt:ioinit.obj
 0003:000011c8       ___acrt_stdout_buffer      1002c1c8     libucrt:_sftbuf.obj
 0003:000011cc       ___acrt_stderr_buffer      1002c1cc     libucrt:_sftbuf.obj
 0003:00001324       __mbctype                  1002c324     libucrt:mbctype.obj
 0003:00001328       __mbcasemap                1002c328     libucrt:mbctype.obj
 0003:0000132c       ___acrt_current_multibyte_data 1002c32c     libucrt:mbctype.obj
 0003:00001338       __pgmptr                   1002c338     libucrt:argv_data.obj
 0003:0000133c       ___argc                    1002c33c     libucrt:argv_data.obj
 0003:00001340       ___argv                    1002c340     libucrt:argv_data.obj
 0003:00001344       ___wargv                   1002c344     libucrt:argv_data.obj
 0003:00001348       __acmdln                   1002c348     libucrt:argv_data.obj
 0003:0000134c       __wcmdln                   1002c34c     libucrt:argv_data.obj
 0003:00001350       ___acrt_heap               1002c350     libucrt:heap_handle.obj
 0003:0000136c       __umaskval                 1002c36c     libucrt:umask.obj
 0003:00001374       ___acrt_lconv_static_null  1002c374     libucrt:localeconv.obj
 0003:00001378       ___acrt_lconv_static_W_null 1002c378     libucrt:localeconv.obj
 0003:00001380       __fmode                    1002c380     libucrt:txtmode.obj
 0003:0000138c       ___fastflag                1002c38c     libucrt:fp_flags.obj
 0003:00001398       ?_OptionsStorage@?1??__local_stdio_printf_options@@9@9 1002c398     <common>
 0003:000013a0       ___scrt_ucrt_dll_is_in_use 1002c3a0     <common>
 0003:000013a4       ___dyn_tls_init_callback   1002c3a4     <common>
 0003:000013a8       __pmatherr                 1002c3a8     <common>
 0003:000013ac       ___use_sse2_mathfcns       1002c3ac     <common>

 entry point at        0001:000079bc

 Static symbols

 0000:fffd0000       .debug$S                   10000000     instrument.exp
 0000:fffd0000       .debug$S                   10000000     kernel32:KERNEL32.dll
 0000:fffd0000       .debug$S                   10000000     kernel32:KERNEL32.dll
 0000:fffd0000       .debug$S                   10000000     kernel32:KERNEL32.dll
 0000:fffd0000       .debug$S                   10000000     kernel32:KERNEL32.dll
 0000:fffd0000       .debug$S                   10000000     kernel32:KERNEL32.dll
 0000:fffd0000       .debug$S                   10000000     kernel32:KERNEL32.dll
 0000:fffd0000       .debug$S                   10000000     kernel32:KERNEL32.dll
 0000:fffd0000       .debug$S                   10000000     kernel32:KERNEL32.dll
 0000:fffd0000       .debug$S                   10000000     kernel32:KERNEL32.dll
 0000:fffd0000       .debug$S                   10000000     kernel32:KERNEL32.dll
 0000:fffd0000       .debug$S                   10000000     kernel32:KERNEL32.dll
 0000:fffd0000       .debug$S                   10000000     kernel32:KERNEL32.dll
 0000:fffd0000       .debug$S                   10000000     kernel32:KERNEL32.dll
 0000:fffd0000       .debug$S                   10000000     kernel32:KERNEL32.dll
 0000:fffd0000       .debug$S                   10000000     kernel32:KERNEL32.dll
 0000:fffd0000       .debug$S                   10000000     kernel32:KERNEL32.dll
 0000:fffd0000       .debug$S                   10000000     kernel32:KERNEL32.dll
 0000:fffd0000       .debug$S                   10000000     kernel32:KERNEL32.dll
 0000:fffd0000       .debug$S                   10000000     kernel32:KERNEL32.dll
 0000:fffd0000       .debug$S                   10000000     kernel32:KERNEL32.dll
 0000:fffd0000       .debug$S                   10000000     kernel32:KERNEL32.dll
 0000:fffd0000       .debug$S                   10000000     kernel32:KERNEL32.dll
 0000:fffd0000       .debug$S                   10000000     kernel32:KERNEL32.dll
 0000:fffd0000       .debug$S                   10000000     kernel32:KERNEL32.dll
 0000:fffd0000       .debug$S                   10000000     kernel32:KERNEL32.dll
 0000:fffd0000       .debug$S                   10000000     kernel32:KERNEL32.dll
 0000:fffd0000       .debug$S                   10000000     kernel32:KERNEL32.dll
 0000:fffd0000       .debug$S                   10000000     kernel32:KERNEL32.dll
 0000:fffd0000       .debug$S                   10000000     kernel32:KERNEL32.dll
 0000:fffd0000       .debug$S                   10000000     kernel32:KERNEL32.dll
 0000:fffd0000       .debug$S                   10000000     kernel32:KERNEL32.dll
 0000:fffd0000       .debug$S                   10000000     kernel32:KERNEL32.dll
 0000:fffd0000       .debug$S                   10000000     kernel32:KERNEL32.dll
 0000:fffd0000       .debug$S                   10000000     kernel32:KERNEL32.dll
 0000:fffd0000       .debug$S                   10000000     kernel32:KERNEL32.dll
 0000:fffd0000       .debug$S                   10000000     kernel32:KERNEL32.dll
 0000:fffd0000       .debug$S                   10000000     kernel32:KERNEL32.dll
 0000:fffd0000       .debug$S                   10000000     kernel32:KERNEL32.dll
 0000:fffd0000       .debug$S                   10000000     kernel32:KERNEL32.dll
 0000:fffd0000       .debug$S                   10000000     kernel32:KERNEL32.dll
 0000:fffd0000       .debug$S                   10000000     kernel32:KERNEL32.dll
 0000:fffd0000       .debug$S                   10000000     kernel32:KERNEL32.dll
 0000:fffd0000       .debug$S                   10000000     kernel32:KERNEL32.dll
 0000:fffd0000       .debug$S                   10000000     kernel32:KERNEL32.dll
 0000:fffd0000       .debug$S                   10000000     kernel32:KERNEL32.dll
 0000:fffd0000       .debug$S                   10000000     kernel32:KERNEL32.dll
 0000:fffd0000       .debug$S                   10000000     kernel32:KERNEL32.dll
 0000:fffd0000       .debug$S                   10000000     kernel32:KERNEL32.dll
 0000:fffd0000       .debug$S                   10000000     kernel32:KERNEL32.dll
 0000:fffd0000       .debug$S                   10000000     kernel32:KERNEL32.dll
 0000:fffd0000       .debug$S                   10000000     kernel32:KERNEL32.dll
 0000:fffd0000       .debug$S                   10000000     kernel32:KERNEL32.dll
 0000:fffd0000       .debug$S                   10000000     kernel32:KERNEL32.dll
 0000:fffd0000       .debug$S                   10000000     kernel32:KERNEL32.dll
 0000:fffd0000       .debug$S                   10000000     kernel32:KERNEL32.dll
 0000:fffd0000       .debug$S                   10000000     kernel32:KERNEL32.dll
 0000:fffd0000       .debug$S                   10000000     kernel32:KERNEL32.dll
 0000:fffd0000       .debug$S                   10000000     kernel32:KERNEL32.dll
 0000:fffd0000       .debug$S                   10000000     kernel32:KERNEL32.dll
 0000:fffd0000       .debug$S                   10000000     kernel32:KERNEL32.dll
 0000:fffd0000       .debug$S                   10000000     kernel32:KERNEL32.dll
 0000:fffd0000       .debug$S                   10000000     kernel32:KERNEL32.dll
 0000:fffd0000       .debug$S                   10000000     kernel32:KERNEL32.dll
 0000:fffd0000       .debug$S                   10000000     kernel32:KERNEL32.dll
 0000:fffd0000       .debug$S                   10000000     kernel32:KERNEL32.dll
 0000:fffd0000       .debug$S                   10000000     kernel32:KERNEL32.dll
 0000:fffd0000       .debug$S                   10000000     kernel32:KERNEL32.dll
 0000:fffd0000       .debug$S                   10000000     kernel32:KERNEL32.dll
 0000:fffd0000       .debug$S                   10000000     kernel32:KERNEL32.dll
 0000:fffd0000       .debug$S                   10000000     kernel32:KERNEL32.dll
 0000:fffd0000       .debug$S                   10000000     kernel32:KERNEL32.dll
 0000:fffd0000       .debug$S                   10000000     kernel32:KERNEL32.dll
 0000:fffd0000       .debug$S                   10000000     kernel32:KERNEL32.dll
 0000:fffd0000       .debug$S                   10000000     kernel32:KERNEL32.dll
 0000:fffd0000       .debug$S                   10000000     kernel32:KERNEL32.dll
 0000:fffd0000       .debug$S                   10000000     kernel32:KERNEL32.dll
 0000:fffd0000       .debug$S                   10000000     kernel32:KERNEL32.dll
 0000:fffd0000       .debug$S                   10000000     kernel32:KERNEL32.dll
 0000:fffd0000       .debug$S                   10000000     kernel32:KERNEL32.dll
 0000:fffd0000       .debug$S                   10000000     kernel32:KERNEL32.dll
 0000:fffd0000       .debug$S                   10000000     kernel32:KERNEL32.dll
 0000:fffd0000       .debug$S                   10000000     kernel32:KERNEL32.dll
 0000:fffd0000       .debug$S                   10000000     kernel32:KERNEL32.dll
 0000:fffd0000       .debug$S                   10000000     kernel32:KERNEL32.dll
 0000:fffd0000       .debug$S                   10000000     kernel32:KERNEL32.dll
 0000:fffd0000       .debug$S                   10000000     kernel32:KERNEL32.dll
 0000:fffd0000       .debug$S                   10000000     kernel32:KERNEL32.dll
 0000:fffd0000       .debug$S                   10000000     kernel32:KERNEL32.dll
 0000:fffd0000       .debug$S                   10000000     kernel32:KERNEL32.dll
 0000:fffd0000       .debug$S                   10000000     kernel32:KERNEL32.dll
 0001:0000043f       _isSlash                   1000143f f   FileSystemSupport_md.obj
 0001:000004be       _normalizePath             100014be f   FileSystemSupport_md.obj
 0001:000005c0       _normalizePrefix           100015c0 f   FileSystemSupport_md.obj
 0001:00000da2       _appendBootClassPath       10001da2 f   InvocationAdapter.obj
 0001:000010b7       _appendClassPath           100020b7 f   InvocationAdapter.obj
 0001:000011e5       _decodeNibble              100021e5 f   InvocationAdapter.obj
 0001:00001217       _decodePath                10002217 f   InvocationAdapter.obj
 0001:000013e2       _parseArgumentTail         100023e2 f   InvocationAdapter.obj
 0001:00001477       _splitPathList             10002477 f   InvocationAdapter.obj
 0001:00003291       _doAttribute               10004291 f   JarFacade.obj
 0001:00003a4a       _highMask                  10004a4a f   PathCharsValidator.obj
 0001:00003ab0       _highMaskRange             10004ab0 f   PathCharsValidator.obj
 0001:00003b28       _initialize                10004b28 f   PathCharsValidator.obj
 0001:00003c4f       _lowMask                   10004c4f f   PathCharsValidator.obj
 0001:00003cad       _match                     10004cad f   PathCharsValidator.obj
 0001:00004399       _cp                        10005399 f   canonicalize_md.obj
 0001:0000442a       _nextsep                   1000542a f   canonicalize_md.obj
 0001:00004513       _compute_cen               10005513 f   jli_static:parse_manifest.obj
 0001:000048ca       _find_end                  100058ca f   jli_static:parse_manifest.obj
 0001:00004a8f       _find_end64                10005a8f f   jli_static:parse_manifest.obj
 0001:00004b09       _find_file                 10005b09 f   jli_static:parse_manifest.obj
 0001:00004e4c       _haveZIP64                 10005e4c f   jli_static:parse_manifest.obj
 0001:00004ebc       _inflate_file              10005ebc f   jli_static:parse_manifest.obj
 0001:00004ff0       _parse_nv_pair             10005ff0 f   jli_static:parse_manifest.obj
 0001:00006561       $LN761                     10007561     jli_static:inflate.obj
 0001:000067df       _inflateStateCheck         100077df f   jli_static:inflate.obj
 0001:00006812       _updatewindow              10007812 f   jli_static:inflate.obj
 0001:00006df7       _crc_word                  10007df7 f   jli_static:zcrc32.obj
 0001:0000767c       ?dllmain_crt_dispatch@@YGHQAUHINSTANCE__@@KQAX@Z 1000867c f   LIBCMT:dll_dllmain.obj
 0001:000076cf       ?dllmain_crt_process_attach@@YAHQAUHINSTANCE__@@QAX@Z 100086cf f   LIBCMT:dll_dllmain.obj
 0001:000077d6       ?dllmain_crt_process_detach@@YAH_N@Z 100087d6 f   LIBCMT:dll_dllmain.obj
 0001:00007886       ?dllmain_dispatch@@YAHQAUHINSTANCE__@@KQAX@Z 10008886 f   LIBCMT:dll_dllmain.obj
 0001:00007991       ?dllmain_raw@@YGHQAUHINSTANCE__@@KQAX@Z 10008991 f   LIBCMT:dll_dllmain.obj
 0001:000079e0       $$000000                   100089e0     LIBCMT:llrem.obj
 0001:00007a00       L1                         10008a00     LIBCMT:llrem.obj
 0001:00007a1b       L2                         10008a1b     LIBCMT:llrem.obj
 0001:00007a3a       L3                         10008a3a     LIBCMT:llrem.obj
 0001:00007a48       L5                         10008a48     LIBCMT:llrem.obj
 0001:00007a73       L6                         10008a73     LIBCMT:llrem.obj
 0001:00007a7b       L7                         10008a7b     LIBCMT:llrem.obj
 0001:00007a86       L4                         10008a86     LIBCMT:llrem.obj
 0001:00007a8d       L8                         10008a8d     LIBCMT:llrem.obj
 0001:00007bb4       ___get_entropy             10008bb4 f   LIBCMT:gs_support.obj
 0001:00007c8d       ?find_pe_section@@YAPAU_IMAGE_SECTION_HEADER@@QAEI@Z 10008c8d f   LIBCMT:utility.obj
 0001:000080f0       $$000000                   100090f0     LIBCMT:sehprolg4.obj
 0001:00008320       $$000000                   10009320     libvcruntime:memcpy.obj
 0001:00008320       $$000000                   10009320     libvcruntime:memmove.obj
 0001:00008340       CopyUp                     10009340     libvcruntime:memcpy.obj
 0001:00008340       CopyUp                     10009340     libvcruntime:memmove.obj
 0001:00008364       CopyUpLargeMov             10009364     libvcruntime:memcpy.obj
 0001:00008364       CopyUpLargeMov             10009364     libvcruntime:memmove.obj
 0001:00008377       CopyUpSSE2Check            10009377     libvcruntime:memcpy.obj
 0001:00008377       CopyUpSSE2Check            10009377     libvcruntime:memmove.obj
 0001:00008390       AtomChk                    10009390     libvcruntime:memcpy.obj
 0001:00008390       AtomChk                    10009390     libvcruntime:memmove.obj
 0001:000083b6       PalignHead4                100093b6     libvcruntime:memcpy.obj
 0001:000083b6       PalignHead4                100093b6     libvcruntime:memmove.obj
 0001:000083c9       PalignHead8                100093c9     libvcruntime:memcpy.obj
 0001:000083c9       PalignHead8                100093c9     libvcruntime:memmove.obj
 0001:000083e0       PalignLoop                 100093e0     libvcruntime:memcpy.obj
 0001:000083e0       PalignLoop                 100093e0     libvcruntime:memmove.obj
 0001:000083f2       MovPalign12                100093f2     libvcruntime:memcpy.obj
 0001:000083f2       MovPalign12                100093f2     libvcruntime:memmove.obj
 0001:000083fc       PalignLoop12               100093fc     libvcruntime:memcpy.obj
 0001:000083fc       PalignLoop12               100093fc     libvcruntime:memmove.obj
 0001:0000844d       MovPalign8                 1000944d     libvcruntime:memcpy.obj
 0001:0000844d       MovPalign8                 1000944d     libvcruntime:memmove.obj
 0001:00008458       PalignLoop8                10009458     libvcruntime:memcpy.obj
 0001:00008458       PalignLoop8                10009458     libvcruntime:memmove.obj
 0001:000084a6       MovPalign4                 100094a6     libvcruntime:memcpy.obj
 0001:000084a6       MovPalign4                 100094a6     libvcruntime:memmove.obj
 0001:000084b0       PalignLoop4                100094b0     libvcruntime:memcpy.obj
 0001:000084b0       PalignLoop4                100094b0     libvcruntime:memmove.obj
 0001:000084fc       PalignTail                 100094fc     libvcruntime:memcpy.obj
 0001:000084fc       PalignTail                 100094fc     libvcruntime:memmove.obj
 0001:00008514       PalignTail4                10009514     libvcruntime:memcpy.obj
 0001:00008514       PalignTail4                10009514     libvcruntime:memmove.obj
 0001:00008527       PalignTail8                10009527     libvcruntime:memcpy.obj
 0001:00008527       PalignTail8                10009527     libvcruntime:memmove.obj
 0001:0000853e       PalignTailLE3              1000953e     libvcruntime:memcpy.obj
 0001:0000853e       PalignTailLE3              1000953e     libvcruntime:memmove.obj
 0001:00008547       Dword_align                10009547     libvcruntime:memcpy.obj
 0001:00008547       Dword_align                10009547     libvcruntime:memmove.obj
 0001:0000854f       Dword_up_align_loop        1000954f     libvcruntime:memcpy.obj
 0001:0000854f       Dword_up_align_loop        1000954f     libvcruntime:memmove.obj
 0001:00008562       Dword_align_Ok             10009562     libvcruntime:memcpy.obj
 0001:00008562       Dword_align_Ok             10009562     libvcruntime:memmove.obj
 0001:0000857c       ByteCopyUp                 1000957c     libvcruntime:memcpy.obj
 0001:0000857c       ByteCopyUp                 1000957c     libvcruntime:memmove.obj
 0001:00008584       TrailingUpVec              10009584     libvcruntime:memcpy.obj
 0001:00008584       TrailingUpVec              10009584     libvcruntime:memmove.obj
 0001:00008594       TrailingUp0                10009594     libvcruntime:memcpy.obj
 0001:00008594       TrailingUp0                10009594     libvcruntime:memmove.obj
 0001:0000859c       TrailingUp1                1000959c     libvcruntime:memcpy.obj
 0001:0000859c       TrailingUp1                1000959c     libvcruntime:memmove.obj
 0001:000085a8       TrailingUp2                100095a8     libvcruntime:memcpy.obj
 0001:000085a8       TrailingUp2                100095a8     libvcruntime:memmove.obj
 0001:000085bc       TrailingUp3                100095bc     libvcruntime:memcpy.obj
 0001:000085bc       TrailingUp3                100095bc     libvcruntime:memmove.obj
 0001:000085d4       CopyDown                   100095d4     libvcruntime:memcpy.obj
 0001:000085d4       CopyDown                   100095d4     libvcruntime:memmove.obj
 0001:000085f9       CopyDownNotAligned         100095f9     libvcruntime:memcpy.obj
 0001:000085f9       CopyDownNotAligned         100095f9     libvcruntime:memmove.obj
 0001:00008600       CopyDownAlignLoop          10009600     libvcruntime:memcpy.obj
 0001:00008600       CopyDownAlignLoop          10009600     libvcruntime:memmove.obj
 0001:0000860d       CopyDownAligned            1000960d     libvcruntime:memcpy.obj
 0001:0000860d       CopyDownAligned            1000960d     libvcruntime:memmove.obj
 0001:00008630       TrailingDownVec            10009630     libvcruntime:memcpy.obj
 0001:00008630       TrailingDownVec            10009630     libvcruntime:memmove.obj
 0001:00008640       TrailingDown0              10009640     libvcruntime:memcpy.obj
 0001:00008640       TrailingDown0              10009640     libvcruntime:memmove.obj
 0001:00008648       TrailingDown1              10009648     libvcruntime:memcpy.obj
 0001:00008648       TrailingDown1              10009648     libvcruntime:memmove.obj
 0001:00008658       TrailingDown2              10009658     libvcruntime:memcpy.obj
 0001:00008658       TrailingDown2              10009658     libvcruntime:memmove.obj
 0001:0000866c       TrailingDown3              1000966c     libvcruntime:memcpy.obj
 0001:0000866c       TrailingDown3              1000966c     libvcruntime:memmove.obj
 0001:00008685       XmmMovLargeAlignTest       10009685     libvcruntime:memcpy.obj
 0001:00008685       XmmMovLargeAlignTest       10009685     libvcruntime:memmove.obj
 0001:0000868d       XmmMovAlignLoop            1000968d     libvcruntime:memcpy.obj
 0001:0000868d       XmmMovAlignLoop            1000968d     libvcruntime:memmove.obj
 0001:0000869c       XmmMovLargeLoop            1000969c     libvcruntime:memcpy.obj
 0001:0000869c       XmmMovLargeLoop            1000969c     libvcruntime:memmove.obj
 0001:0000870c       XmmMovSmallTest            1000970c     libvcruntime:memcpy.obj
 0001:0000870c       XmmMovSmallTest            1000970c     libvcruntime:memmove.obj
 0001:00008711       XmmMovSmallLoop            10009711     libvcruntime:memcpy.obj
 0001:00008711       XmmMovSmallLoop            10009711     libvcruntime:memmove.obj
 0001:00008734       CopyDownSmall              10009734     libvcruntime:memcpy.obj
 0001:00008734       CopyDownSmall              10009734     libvcruntime:memmove.obj
 0001:0000873c       CopyDownDwordLoop          1000973c     libvcruntime:memcpy.obj
 0001:0000873c       CopyDownDwordLoop          1000973c     libvcruntime:memmove.obj
 0001:00008751       CopyDownByteTest           10009751     libvcruntime:memcpy.obj
 0001:00008751       CopyDownByteTest           10009751     libvcruntime:memmove.obj
 0001:00008755       CopyDownByteLoop           10009755     libvcruntime:memcpy.obj
 0001:00008755       CopyDownByteLoop           10009755     libvcruntime:memmove.obj
 0001:00008764       CopyDownReturn             10009764     libvcruntime:memcpy.obj
 0001:00008764       CopyDownReturn             10009764     libvcruntime:memmove.obj
 0001:00008770       XmmCopy                    10009770     libvcruntime:memcpy.obj
 0001:00008770       XmmCopy                    10009770     libvcruntime:memmove.obj
 0001:0000877d       XmmCopyAligned             1000977d     libvcruntime:memcpy.obj
 0001:0000877d       XmmCopyAligned             1000977d     libvcruntime:memmove.obj
 0001:00008790       XmmCopyLargeLoop           10009790     libvcruntime:memcpy.obj
 0001:00008790       XmmCopyLargeLoop           10009790     libvcruntime:memmove.obj
 0001:000087ed       XmmCopySmallTest           100097ed     libvcruntime:memcpy.obj
 0001:000087ed       XmmCopySmallTest           100097ed     libvcruntime:memmove.obj
 0001:00008800       XmmCopySmallLoop           10009800     libvcruntime:memcpy.obj
 0001:00008800       XmmCopySmallLoop           10009800     libvcruntime:memmove.obj
 0001:0000881b       CopyUpDwordMov             1000981b     libvcruntime:memcpy.obj
 0001:0000881b       CopyUpDwordMov             1000981b     libvcruntime:memmove.obj
 0001:00008820       CopyUpDwordTest            10009820     libvcruntime:memcpy.obj
 0001:00008820       CopyUpDwordTest            10009820     libvcruntime:memmove.obj
 0001:00008827       CopyUpDwordLoop            10009827     libvcruntime:memcpy.obj
 0001:00008827       CopyUpDwordLoop            10009827     libvcruntime:memmove.obj
 0001:00008836       CopyUpByteTest             10009836     libvcruntime:memcpy.obj
 0001:00008836       CopyUpByteTest             10009836     libvcruntime:memmove.obj
 0001:0000883d       CopyUpByteLoop             1000983d     libvcruntime:memcpy.obj
 0001:0000883d       CopyUpByteLoop             1000983d     libvcruntime:memmove.obj
 0001:00008850       CopyUpReturn               10009850     libvcruntime:memcpy.obj
 0001:00008850       CopyUpReturn               10009850     libvcruntime:memmove.obj
 0001:00008860       XmmCopyUnaligned           10009860     libvcruntime:memcpy.obj
 0001:00008860       XmmCopyUnaligned           10009860     libvcruntime:memmove.obj
 0001:00008873       XmmAlignByte               10009873     libvcruntime:memcpy.obj
 0001:00008873       XmmAlignByte               10009873     libvcruntime:memmove.obj
 0001:0000887c       XmmAlignDwordTest          1000987c     libvcruntime:memcpy.obj
 0001:0000887c       XmmAlignDwordTest          1000987c     libvcruntime:memmove.obj
 0001:00008881       XmmAlignDwordLoop          10009881     libvcruntime:memcpy.obj
 0001:00008881       XmmAlignDwordLoop          10009881     libvcruntime:memmove.obj
 0001:0000888e       XmmAlignAdjustCnt          1000988e     libvcruntime:memcpy.obj
 0001:0000888e       XmmAlignAdjustCnt          1000988e     libvcruntime:memmove.obj
 0001:000088a0       $$000000                   100098a0     libvcruntime:strchr.obj
 0001:000088d3       strchr_sse_loop            100098d3     libvcruntime:strchr.obj
 0001:000088f7       strchr_sse_break           100098f7     libvcruntime:strchr.obj
 0001:00008908       strchr_no_sse2             10009908     libvcruntime:strchr.obj
 0001:00008920       str_misaligned             10009920     libvcruntime:strchr.obj
 0001:00008935       main_loop_start            10009935     libvcruntime:strchr.obj
 0001:00008940       main_loop                  10009940     libvcruntime:strchr.obj
 0001:0000897c       retnull                    1000997c     libvcruntime:strchr.obj
 0001:0000897e       retnull_bx                 1000997e     libvcruntime:strchr.obj
 0001:00008982       found_bx                   10009982     libvcruntime:strchr.obj
 0001:00008987       chr_is_found               10009987     libvcruntime:strchr.obj
 0001:000089af       byte_3                     100099af     libvcruntime:strchr.obj
 0001:000089b6       byte_2                     100099b6     libvcruntime:strchr.obj
 0001:000089bd       byte_1                     100099bd     libvcruntime:strchr.obj
 0001:000089c4       byte_0                     100099c4     libvcruntime:strchr.obj
 0001:000089d0       $$000000                   100099d0     libvcruntime:memset.obj
 0001:00008a15       XMMMov                     10009a15     libvcruntime:memset.obj
 0001:00008a50       LargeRangeBytes            10009a50     libvcruntime:memset.obj
 0001:00008a8d       XmmMovSmall                10009a8d     libvcruntime:memset.obj
 0001:00008aa0       XmmSmallLoop               10009aa0     libvcruntime:memset.obj
 0001:00008aa5       MidRangeBytes              10009aa5     libvcruntime:memset.obj
 0001:00008ac1       XMMTrailingBytes           10009ac1     libvcruntime:memset.obj
 0001:00008ad5       SmallMov                   10009ad5     libvcruntime:memset.obj
 0001:00008add       ByteLoop                   10009add     libvcruntime:memset.obj
 0001:00008aeb       DwordTest                  10009aeb     libvcruntime:memset.obj
 0001:00008afb       QwordTest                  10009afb     libvcruntime:memset.obj
 0001:00008b10       QwordLoop                  10009b10     libvcruntime:memset.obj
 0001:00008b23       toend                      10009b23     libvcruntime:memset.obj
 0001:0000a126       $LN1250                    1000b126     libvcruntime:memcmp.obj
 0001:0000a1b0       _ValidateLocalCookies      1000b1b0 f   libvcruntime:chandler4.obj
 0001:0000a4ac       ?_FilterSetCurrentException@@YAKPAU_EXCEPTION_POINTERS@@E@Z 1000b4ac f   libvcruntime:ehhelpers.obj
 0001:0000a5b0       $$000000                   1000b5b0     libvcruntime:exsup4.obj
 0001:0000a5e2       _lu_top                    1000b5e2     libvcruntime:exsup4.obj
 0001:0000a641       _lu_done                   1000b641     libvcruntime:exsup4.obj
 0001:0000a650       $$000000                   1000b650     libvcruntime:exsup4.obj
 0001:0000a650       __unwind_handler4          1000b650 f   libvcruntime:exsup4.obj
 0001:0000a6a0       $$000000                   1000b6a0     libvcruntime:exsup4.obj
 0001:0000a6c0       $$000000                   1000b6c0     libvcruntime:exsup4.obj
 0001:0000a6e0       $$000000                   1000b6e0     libvcruntime:exsup4.obj
 0001:0000a6f5       ReturnPoint                1000b6f5     libvcruntime:exsup4.obj
 0001:0000a700       $$000000                   1000b700     libvcruntime:exsup4.obj
 0001:0000a8f0       $$000000                   1000b8f0     libvcruntime:exsup.obj
 0001:0000a900       $$000000                   1000b900     libvcruntime:exsup.obj
 0001:0000a90b       __NLG_Go                   1000b90b     libvcruntime:exsup.obj
 0001:0000a920       $$000000                   1000b920     libvcruntime:exsup.obj
 0001:0000acd9       ?try_get_function@@YAPAXW4function_id@?A0x14174aea@@QBDQBW4module_id@2@2@Z 1000bcd9 f   libvcruntime:winapi_downlevel.obj
 0001:0000ad79       ?try_load_library_from_system_directory@@YAPAUHINSTANCE__@@QB_W@Z 1000bd79 f   libvcruntime:winapi_downlevel.obj
 0001:0000aefa       ??$BuildCatchObjectHelperInternal@V__FrameHandler3@@@@YAHPAUEHExceptionRecord@@PAXPBU_s_HandlerType@@PBU_s_CatchableType@@@Z 1000befa f   libvcruntime:frame.obj
 0001:0000b038       ??$BuildCatchObjectInternal@V__FrameHandler3@@@@YAXPAUEHExceptionRecord@@PAXPBU_s_HandlerType@@PBU_s_CatchableType@@@Z 1000c038 f   libvcruntime:frame.obj
 0001:0000b0d1       ??$CatchIt@V__FrameHandler3@@@@YAXPAUEHExceptionRecord@@PAUEHRegistrationNode@@PAU_CONTEXT@@PAXPBU_s_FuncInfo@@PBU_s_HandlerType@@PBU_s_CatchableType@@PBU_s_TryBlockMapEntry@@H1EE@Z 1000c0d1 f   libvcruntime:frame.obj
 0001:0000b151       ??$FindHandler@V__FrameHandler3@@@@YAXPAUEHExceptionRecord@@PAUEHRegistrationNode@@PAU_CONTEXT@@PAXPBU_s_FuncInfo@@EH1@Z 1000c151 f   libvcruntime:frame.obj
 0001:0000b4f6       ??$FindHandlerForForeignException@V__FrameHandler3@@@@YAXPAUEHExceptionRecord@@PAUEHRegistrationNode@@PAU_CONTEXT@@PAXPBU_s_FuncInfo@@HH1@Z 1000c4f6 f   libvcruntime:frame.obj
 0001:0000b881       ?CallCatchBlock@@YAPAXPAUEHExceptionRecord@@PAUEHRegistrationNode@@PAU_CONTEXT@@PBU_s_FuncInfo@@PAXHK@Z 1000c881 f   libvcruntime:frame.obj
 0001:0000ba50       ?CallUnexpected@@YAXPBU_s_ESTypeList@@@Z 1000ca50 f   libvcruntime:frame.obj
 0001:0000ba70       __catch$?CallUnexpected@@YAXPBU_s_ESTypeList@@@Z$0 1000ca70 f   libvcruntime:frame.obj
 0001:0000ba8f       ?ExFilterRethrow@@YAHPAU_EXCEPTION_POINTERS@@@Z 1000ca8f f   libvcruntime:frame.obj
 0001:0000bbd9       ?IsInExceptionSpec@@YAEPAUEHExceptionRecord@@PBU_s_ESTypeList@@@Z 1000cbd9 f   libvcruntime:frame.obj
 0001:0000bcb0       $$000000                   1000ccb0     libvcruntime:lowhelpr.obj
 0001:0000bcef       _NLG_Continue              1000ccef     libvcruntime:lowhelpr.obj
 0001:0000c4da       ??$?RV<lambda_62491a2101a2aba6cc4a769149c84f1f>@@AAV<lambda_826c27fce7726908515bbc79a5266961>@@V<lambda_4e64bbd54b50a7b070e3ea8d795375b6>@@@?$__crt_seh_guarded_call@H@@QAEH$$QAV<lambda_62491a2101a2aba6cc4a769149c84f1f>@@AAV<lambda_826c27fce7726908515bbc79a5266961>@@$$QAV<lambda_4e64bbd54b50a7b070e3ea8d795375b6>@@@Z 1000d4da f   libucrt:output.obj
 0001:0000d088       ??R<lambda_826c27fce7726908515bbc79a5266961>@@QBEHXZ 1000e088 f   libucrt:output.obj
 0001:0000d523       $LN121                     1000e523     libucrt:output.obj
 0001:0000da12       $LN18                      1000ea12     libucrt:output.obj
 0001:0000da26       $LN17                      1000ea26     libucrt:output.obj
 0001:0000e050       $$000000                   1000f050     libucrt:strlen.obj
 0001:0000e0e0       $$000000                   1000f0e0     libucrt:strcat.obj
 0001:0000e1f0       $$000000                   1000f1f0     libucrt:strncpy.obj
 0001:0000e8e3       ??$common_fullpath@D@@YAPADQADQBDIH1H@Z 1000f8e3 f   libucrt:fullpath.obj
 0001:0000ebfb       _memcpy_s                  1000fbfb f   libucrt:cfout.obj
 0001:0000ebfb       _memcpy_s                  1000fbfb f   libucrt:fullpath.obj
 0001:0000ebfb       _memcpy_s                  1000fbfb f   libucrt:mbctype.obj
 0001:0000f150       $$000000                   10010150     libucrt:strpbrk.obj
 0001:0000f190       ??$common_lseek@_J@@YA_JH_JHAAV__crt_cached_ptd_host@@@Z 10010190 f   libucrt:lseek.obj
 0001:0000f2b5       ??$common_lseek_nolock@_J@@YA_JH_JHAAV__crt_cached_ptd_host@@@Z 100102b5 f   libucrt:lseek.obj
 0001:0000f595       ??$?RV<lambda_03b1d95aef87969028cfba75ccab2455>@@AAV<lambda_6e4b09c48022b2350581041d5f6b0c4c>@@V<lambda_22bdf7517842c4b3e53723af5aa32b9e>@@@?$__crt_seh_guarded_call@X@@QAEX$$QAV<lambda_03b1d95aef87969028cfba75ccab2455>@@AAV<lambda_6e4b09c48022b2350581041d5f6b0c4c>@@$$QAV<lambda_22bdf7517842c4b3e53723af5aa32b9e>@@@Z 10010595 f   libucrt:exit.obj
 0001:0000f5fd       ??R<lambda_6e4b09c48022b2350581041d5f6b0c4c>@@QBE@XZ 100105fd f   libucrt:exit.obj
 0001:0000f6e5       ?common_exit@@YAXHW4_crt_exit_cleanup_mode@@W4_crt_exit_return_mode@@@Z 100106e5 f   libucrt:exit.obj
 0001:0000f77c       ?exit_or_terminate_process@@YAXI@Z 1001077c f   libucrt:exit.obj
 0001:0000f7ad       ?is_managed_app@@YA_NXZ    100107ad f   libucrt:exit.obj
 0001:0000f7ef       ?should_call_terminate_process@@YA_NXZ 100107ef f   libucrt:exit.obj
 0001:0000f808       ?try_cor_exit_process@@YAXI@Z 10010808 f   libucrt:exit.obj
 0001:0000f8c5       ??$common_configure_argv@D@@YAHW4_crt_argv_mode@@@Z 100108c5 f   libucrt:argv_parsing.obj
 0001:0000fa02       ??$parse_command_line@D@@YAXPADPAPAD0PAI2@Z 10010a02 f   libucrt:argv_parsing.obj
 0001:0000fbd0       ??$common_initialize_environment_nolock@D@@YAHXZ 10010bd0 f   libucrt:environment_initialization.obj
 0001:0000fc2a       ??$create_environment@D@@YAQAPADQAD@Z 10010c2a f   libucrt:environment_initialization.obj
 0001:0000fd0c       ??$free_environment@D@@YAXQAPAD@Z 10010d0c f   libucrt:environment_initialization.obj
 0001:0000fd0c       ??$free_environment@_W@@YAXQAPA_W@Z 10010d0c f   libucrt:environment_initialization.obj
 0001:0000fd3b       ??$uninitialize_environment_internal@D@@YAXAAPAPAD@Z 10010d3b f   libucrt:environment_initialization.obj
 0001:0000fd56       ??$uninitialize_environment_internal@_W@@YAXAAPAPA_W@Z 10010d56 f   libucrt:environment_initialization.obj
 0001:0000fdc7       ??$?RV<lambda_69a2805e680e0e292e8ba93315fe43a8>@@AAV<lambda_f03950bc5685219e0bcd2087efbe011e>@@V<lambda_03fcd07e894ec930e3f35da366ca99d6>@@@?$__crt_seh_guarded_call@H@@QAEH$$QAV<lambda_69a2805e680e0e292e8ba93315fe43a8>@@AAV<lambda_f03950bc5685219e0bcd2087efbe011e>@@$$QAV<lambda_03fcd07e894ec930e3f35da366ca99d6>@@@Z 10010dc7 f   libucrt:onexit.obj
 0001:0000fe22       ??R<lambda_f03950bc5685219e0bcd2087efbe011e>@@QBE@XZ 10010e22 f   libucrt:onexit.obj
 0001:0000ff63       _initialize_global_variables 10010f63 f   libucrt:initialization.obj
 0001:0000ff70       _initialize_c              10010f70 f   libucrt:initialization.obj
 0001:0000ff8a       _initialize_environment    10010f8a f   libucrt:initialization.obj
 0001:0000ff8a       _initialize_global_state_isolation 10010f8a f   libucrt:initialization.obj
 0001:0000ff8a       _report_memory_leaks       10010f8a f   libucrt:initialization.obj
 0001:0000ff8a       _uninitialize_c            10010f8a f   libucrt:initialization.obj
 0001:0000ff8a       _uninitialize_global_state_isolation 10010f8a f   libucrt:initialization.obj
 0001:0000ff8d       _uninitialize_environment  10010f8d f   libucrt:initialization.obj
 0001:0000ff95       _initialize_pointers       10010f95 f   libucrt:initialization.obj
 0001:0000ffc3       _uninitialize_vcruntime    10010fc3 f   libucrt:initialization.obj
 0001:0000ffcc       _uninitialize_allocated_memory 10010fcc f   libucrt:initialization.obj
 0001:0000ffe3       _uninitialize_allocated_io_buffers 10010fe3 f   libucrt:initialization.obj
 0001:00010052       ??R<lambda_af42a3ee9806e9a7305d451646e05244>@@QBE@AAPAU__crt_multibyte_data@@@Z 10011052 f   libucrt:initialization.obj
 0001:00010289       ??$?RV<lambda_d422a76eb4c3bf3ad751449ab71a6ea4>@@AAV<lambda_c9ba49e555ba839a7b07aa3fbecb7617>@@V<lambda_9476263c8ee91a25d21c55370bdb50de>@@@?$__crt_seh_guarded_call@H@@QAEH$$QAV<lambda_d422a76eb4c3bf3ad751449ab71a6ea4>@@AAV<lambda_c9ba49e555ba839a7b07aa3fbecb7617>@@$$QAV<lambda_9476263c8ee91a25d21c55370bdb50de>@@@Z 10011289 f   libucrt:close.obj
 0001:000104bd       ??$common_open@D@@YAHQBDHH@Z 100114bd f   libucrt:open.obj
 0001:0001058e       ?configure_text_mode@@YAHHUfile_options@?A0xa9d50aae@@HAAW4__crt_lowio_text_mode@@@Z 1001158e f   libucrt:open.obj
 0001:000107e4       ?create_file@@YAPAXQB_WQAU_SECURITY_ATTRIBUTES@@Ufile_options@?A0xa9d50aae@@@Z 100117e4 f   libucrt:open.obj
 0001:00010809       ?decode_open_create_flags@@YAKH@Z 10011809 f   libucrt:open.obj
 0001:00010879       ?decode_options@@YA?AUfile_options@?A0xa9d50aae@@HHH@Z 10011879 f   libucrt:open.obj
 0001:000109f3       ?truncate_ctrl_z_if_present@@YAHH@Z 100119f3 f   libucrt:open.obj
 0001:00010e4d       ??$translate_text_mode_nolock@D@@YAHHQADI@Z 10011e4d f   libucrt:read.obj
 0001:00010f9a       ??$translate_text_mode_nolock@_W@@YAHHQA_WI@Z 10011f9a f   libucrt:read.obj
 0001:00011154       ?translate_ansi_or_utf8_nolock@@YAHHQADIQA_WI@Z 10012154 f   libucrt:read.obj
 0001:000112ab       ?translate_utf16_from_console_nolock@@YAHHQA_WI@Z 100122ab f   libucrt:read.obj
 0001:00011870       $$000000                   10012870     libucrt:strncmp.obj
 0001:00011d84       ??$?RV<lambda_15ade71b0218206bbe3333a0c9b79046>@@AAV<lambda_da44e0f8b0f19ba52fefafb335991732>@@V<lambda_207f2d024fc103971653565357d6cd41>@@@?$__crt_seh_guarded_call@X@@QAEX$$QAV<lambda_15ade71b0218206bbe3333a0c9b79046>@@AAV<lambda_da44e0f8b0f19ba52fefafb335991732>@@$$QAV<lambda_207f2d024fc103971653565357d6cd41>@@@Z 10012d84 f   libucrt:per_thread_data.obj
 0001:00011dd6       ??$?RV<lambda_38edbb1296d33220d7e4dd0ed76b244a>@@AAV<lambda_5ce1d447e08cb34b2473517608e21441>@@V<lambda_fb385d3da700c9147fc39e65dd577a8c>@@@?$__crt_seh_guarded_call@X@@QAEX$$QAV<lambda_38edbb1296d33220d7e4dd0ed76b244a>@@AAV<lambda_5ce1d447e08cb34b2473517608e21441>@@$$QAV<lambda_fb385d3da700c9147fc39e65dd577a8c>@@@Z 10012dd6 f   libucrt:per_thread_data.obj
 0001:00011e41       ??$?RV<lambda_6affb1475c98b40b75cdec977db92e3c>@@AAV<lambda_b8d4b9c228a6ecc3f80208dbb4b4a104>@@V<lambda_608742c3c92a14382c1684fc64f96c88>@@@?$__crt_seh_guarded_call@X@@QAEX$$QAV<lambda_6affb1475c98b40b75cdec977db92e3c>@@AAV<lambda_b8d4b9c228a6ecc3f80208dbb4b4a104>@@$$QAV<lambda_608742c3c92a14382c1684fc64f96c88>@@@Z 10012e41 f   libucrt:per_thread_data.obj
 0001:00011e96       ??$?RV<lambda_a7e850c220f1c8d1e6efeecdedd162c6>@@AAV<lambda_46720907175c18b6c9d2717bc0d2d362>@@V<lambda_9048902d66e8d99359bc9897bbb930a8>@@@?$__crt_seh_guarded_call@X@@QAEX$$QAV<lambda_a7e850c220f1c8d1e6efeecdedd162c6>@@AAV<lambda_46720907175c18b6c9d2717bc0d2d362>@@$$QAV<lambda_9048902d66e8d99359bc9897bbb930a8>@@@Z 10012e96 f   libucrt:per_thread_data.obj
 0001:00011ef0       ?construct_ptd@@YAXQAU__acrt_ptd@@QAPAU__crt_locale_data@@@Z 10012ef0 f   libucrt:per_thread_data.obj
 0001:00011f89       ?destroy_fls@@YGXPAX@Z     10012f89 f   libucrt:per_thread_data.obj
 0001:00011faa       ?destroy_ptd@@YAXQAU__acrt_ptd@@@Z 10012faa f   libucrt:per_thread_data.obj
 0001:00012077       ?replace_current_thread_locale_nolock@@YAXQAU__acrt_ptd@@QAU__crt_locale_data@@@Z 10013077 f   libucrt:per_thread_data.obj
 0001:000123d9       ??$?RV<lambda_e5124f882df8998aaf41531e079ba474>@@AAV<lambda_3e16ef9562a7dcce91392c22ab16ea36>@@V<lambda_e25ca0880e6ef98be67edffd8c599615>@@@?$__crt_seh_guarded_call@X@@QAEX$$QAV<lambda_e5124f882df8998aaf41531e079ba474>@@AAV<lambda_3e16ef9562a7dcce91392c22ab16ea36>@@$$QAV<lambda_e25ca0880e6ef98be67edffd8c599615>@@@Z 100133d9 f   libucrt:wsetlocale.obj
 0001:000124d6       ?try_get_AreFileApisANSI@@YAP6GHXZXZ 100134d6 f   libucrt:winapi_thunks.obj
 0001:000124f0       ?try_get_LCMapStringEx@@YAP6GHPB_WK0HPA_WHPAU_nlsversioninfo@@PAXJ@ZXZ 100134f0 f   libucrt:winapi_thunks.obj
 0001:0001250a       ?try_get_LocaleNameToLCID@@YAP6GKPB_WK@ZXZ 1001350a f   libucrt:winapi_thunks.obj
 0001:00012524       ?try_get_first_available_module@@YAPAUHINSTANCE__@@QBW4module_id@?A0x391cf84c@@0@Z 10013524 f   libucrt:winapi_thunks.obj
 0001:000125ef       ?try_get_function@@YAPAXW4function_id@?A0x391cf84c@@QBDQBW4module_id@2@2@Z 100135ef f   libucrt:winapi_thunks.obj
 0001:000129a0       ??$?RV<lambda_2866be3712abc81a800a822484c830d8>@@AAV<lambda_39ca0ed439415581b5b15c265174cece>@@V<lambda_2b24c74d71094a6cd0cb82e44167d71b>@@@?$__crt_seh_guarded_call@X@@QAEX$$QAV<lambda_2866be3712abc81a800a822484c830d8>@@AAV<lambda_39ca0ed439415581b5b15c265174cece>@@$$QAV<lambda_2b24c74d71094a6cd0cb82e44167d71b>@@@Z 100139a0 f   libucrt:fflush.obj
 0001:00012a2c       ??$?RV<lambda_2cc53f568c5a2bb6f192f930a45d44ea>@@AAV<lambda_ab61a845afdef5b7c387490eaf3616ee>@@V<lambda_c2ffc0b7726aa6be21d5f0026187e748>@@@?$__crt_seh_guarded_call@X@@QAEX$$QAV<lambda_2cc53f568c5a2bb6f192f930a45d44ea>@@AAV<lambda_ab61a845afdef5b7c387490eaf3616ee>@@$$QAV<lambda_c2ffc0b7726aa6be21d5f0026187e748>@@@Z 10013a2c f   libucrt:fflush.obj
 0001:00012ad8       ?common_flush_all@@YAH_N@Z 10013ad8 f   libucrt:fflush.obj
 0001:00012b25       ?common_flush_all_should_try_to_flush_stream@@YA_NV__crt_stdio_stream@@QAH@Z 10013b25 f   libucrt:fflush.obj
 0001:00012b56       ?is_stream_flushable_or_commitable@@YA_NJ@Z 10013b56 f   libucrt:fflush.obj
 0001:00012c90       ?initialize_inherited_file_handles_nolock@@YAXXZ 10013c90 f   libucrt:ioinit.obj
 0001:00012d46       ?initialize_stdio_handles_nolock@@YAXXZ 10013d46 f   libucrt:ioinit.obj
 0001:00012ee4       ?fe_to_nearest@@YA_NQBN_KF@Z 10013ee4 f   libucrt:cvt.obj
 0001:00012f87       ?fp_format_a@@YAHQBNPADIQADIH_NIW4__acrt_rounding_mode@@AAV__crt_cached_ptd_host@@@Z 10013f87 f   libucrt:cvt.obj
 0001:000132b4       ?fp_format_e@@YAHQBNQADI1IH_NIW4__acrt_rounding_mode@@AAV__crt_cached_ptd_host@@@Z 100142b4 f   libucrt:cvt.obj
 0001:00013358       ?fp_format_e_internal@@YAHQADIH_NIQAU_strflt@@1AAV__crt_cached_ptd_host@@@Z 10014358 f   libucrt:cvt.obj
 0001:000134ab       ?fp_format_f@@YAHQBNQADI1IHW4__acrt_rounding_mode@@AAV__crt_cached_ptd_host@@@Z 100144ab f   libucrt:cvt.obj
 0001:00013541       ?fp_format_f_internal@@YAHQADIHQAU_strflt@@_NAAV__crt_cached_ptd_host@@@Z 10014541 f   libucrt:cvt.obj
 0001:0001362f       ?fp_format_g@@YAHQBNQADI1IH_NIW4__acrt_rounding_mode@@AAV__crt_cached_ptd_host@@@Z 1001462f f   libucrt:cvt.obj
 0001:000136fe       ?fp_format_nan_or_infinity@@YAHW4__acrt_fp_class@@_NPADI1@Z 100146fe f   libucrt:cvt.obj
 0001:00013793       ?shift_bytes@@YAXQADI0H@Z  10014793 f   libucrt:cvt.obj
 0001:000137c7       ?should_round_up@@YA_NQBN_KFW4__acrt_rounding_mode@@@Z 100147c7 f   libucrt:cvt.obj
 0001:00013e71       ??$common_getdcwd@D@@YAPADHPADHHQBDH@Z 10014e71 f   libucrt:getcwd.obj
 0001:00013f9f       ?is_valid_drive@@YAHI@Z    10014f9f f   libucrt:getcwd.obj
 0001:0001403a       ?filter_mbtowcs_flags@@YAKIK@Z 1001503a f   libucrt:multibytetowidechar.obj
 0001:000140fc       ?filter_wcstomb_flags@@YAKIK@Z 100150fc f   libucrt:widechartomultibyte.obj
 0001:000141f8       ?__acrt_LCMapStringA_stat@@YAHPAU__crt_locale_pointers@@PB_WKPBDHPADHHH@Z 100151f8 f   libucrt:lcmapstringa.obj
 0001:00014970       ?<lambda_invoker_cdecl>@<lambda_838c7f62c73c983481e27c09e84b0b5d>@@CAHPBX0@Z 10015970 f   libucrt:argv_wildcards.obj
 0001:00014a4e       ??$common_expand_argv_wildcards@D@@YAHQAPADQAPAPAD@Z 10015a4e f   libucrt:argv_wildcards.obj
 0001:00014bcb       ??$copy_and_add_argument_to_buffer@D@@YAHQBD0IAAV?$argument_list@D@?A0x5f5c8891@@@Z 10015bcb f   libucrt:argv_wildcards.obj
 0001:00014c7c       ??$expand_argument_wildcards@D@@YAHQAD0AAV?$argument_list@D@?A0x5f5c8891@@@Z 10015c7c f   libucrt:argv_wildcards.obj
 0001:00014f01       ??1?$argument_list@D@?A0x5f5c8891@@QAE@XZ 10015f01 f   libucrt:argv_wildcards.obj
 0001:00014f62       ?expand_if_necessary@?$argument_list@D@?A0x5f5c8891@@AAEHXZ 10015f62 f   libucrt:argv_wildcards.obj
 0001:00015095       ??$?RV<lambda_ceb1ee4838e85a9d631eb091e2fbe199>@@AAV<lambda_ae742caa10f662c28703da3d2ea5e57e>@@V<lambda_cd08b5d6af4937fe54fc07d0c9bf6b37>@@@?$__crt_seh_guarded_call@X@@QAEX$$QAV<lambda_ceb1ee4838e85a9d631eb091e2fbe199>@@AAV<lambda_ae742caa10f662c28703da3d2ea5e57e>@@$$QAV<lambda_cd08b5d6af4937fe54fc07d0c9bf6b37>@@@Z 10016095 f   libucrt:mbctype.obj
 0001:000150e2       ??R<lambda_ae742caa10f662c28703da3d2ea5e57e>@@QBE@XZ 100160e2 f   libucrt:mbctype.obj
 0001:00015165       ?CPtoLocaleName@@YAPB_WH@Z 10016165 f   libucrt:mbctype.obj
 0001:000151a3       ?getSystemCP@@YAHH@Z       100161a3 f   libucrt:mbctype.obj
 0001:00015214       ?setSBCS@@YAXPAU__crt_multibyte_data@@@Z 10016214 f   libucrt:mbctype.obj
 0001:00015277       ?setSBUpLow@@YAXPAU__crt_multibyte_data@@@Z 10016277 f   libucrt:mbctype.obj
 0001:0001541c       ?setmbcp_internal@@YAHH_NQAU__acrt_ptd@@QAPAU__crt_multibyte_data@@@Z 1001641c f   libucrt:mbctype.obj
 0001:00015571       ?update_thread_multibyte_data_internal@@YAPAU__crt_multibyte_data@@QAU__acrt_ptd@@QAPAU1@@Z 10016571 f   libucrt:mbctype.obj
 0001:00015871       ?x_ismbbtype_l@@YAHPAU__crt_locale_pointers@@IHH@Z 10016871 f   libucrt:ismbbyte.obj
 0001:000158f2       ?find_end_of_double_null_terminated_sequence@@YAPB_WQB_W@Z 100168f2 f   libucrt:get_environment_from_os.obj
 0001:00015b7c       ??$?RV<lambda_cbab9ec6f41b0180b23cc171c22676b0>@@AAV<lambda_44731a7d0e6d81c3e6aa82d741081786>@@V<lambda_4b292cb8dd18144e164572427af410ab>@@@?$__crt_seh_guarded_call@P6AXH@Z@@QAEP6AXH@Z$$QAV<lambda_cbab9ec6f41b0180b23cc171c22676b0>@@AAV<lambda_44731a7d0e6d81c3e6aa82d741081786>@@$$QAV<lambda_4b292cb8dd18144e164572427af410ab>@@@Z 10016b7c f   libucrt:signal.obj
 0001:00015be4       ?get_global_action_nolock@@YAPAP6AXH@ZH@Z 10016be4 f   libucrt:signal.obj
 0001:00015c26       ?siglookup@@YAPAU__crt_signal_action_t@@HQAU1@@Z 10016c26 f   libucrt:signal.obj
 0001:00015ee7       ?write_double_translated_ansi_nolock@@YA?AUwrite_result@?A0x17268360@@HQBDIAAV__crt_cached_ptd_host@@@Z 10016ee7 f   libucrt:write.obj
 0001:000162ae       ?write_double_translated_unicode_nolock@@YA?AUwrite_result@?A0x17268360@@QBDI@Z 100172ae f   libucrt:write.obj
 0001:00016316       ?write_requires_double_translation_nolock@@YA_NHAAV__crt_cached_ptd_host@@@Z 10017316 f   libucrt:write.obj
 0001:00016393       ?write_text_ansi_nolock@@YA?AUwrite_result@?A0x17268360@@HQBDI@Z 10017393 f   libucrt:write.obj
 0001:0001646e       ?write_text_utf16le_nolock@@YA?AUwrite_result@?A0x17268360@@HQBDI@Z 1001746e f   libucrt:write.obj
 0001:00016557       ?write_text_utf8_nolock@@YA?AUwrite_result@?A0x17268360@@HQBDI@Z 10017557 f   libucrt:write.obj
 0001:00017363       ?free_crt_array_internal@@YAXQAPBXI@Z 10018363 f   libucrt:inittime.obj
 0001:0001746c       ?GetTableIndexFromLocaleName@@YAHPB_W@Z 1001846c f   libucrt:lcidtoname_downlevel.obj
 0001:000174e8       ?_fclose_internal@@YAHQAU_iobuf@@AAV__crt_cached_ptd_host@@@Z 100184e8 f   libucrt:fclose.obj
 0001:0001757f       ?_fclose_nolock_internal@@YAHQAU_iobuf@@AAV__crt_cached_ptd_host@@@Z 1001857f f   libucrt:fclose.obj
 0001:0001763d       ??$?RV<lambda_9e9de3de5fa147e2223d7db92bc10aa6>@@AAV<lambda_38ce7e780aa69e748d6df282ebc68efe>@@V<lambda_8ca6da459f0f6780f1cff60fdc3d00e5>@@@?$__crt_seh_guarded_call@H@@QAEH$$QAV<lambda_9e9de3de5fa147e2223d7db92bc10aa6>@@AAV<lambda_38ce7e780aa69e748d6df282ebc68efe>@@$$QAV<lambda_8ca6da459f0f6780f1cff60fdc3d00e5>@@@Z 1001863d f   libucrt:commit.obj
 0001:0001775c       ?check_trailing@@YA_NPBDW4__acrt_has_trailing_digits@@@Z 1001875c f   libucrt:_fptostr.obj
 0001:0001777f       ?should_round_up@@YA_NQBD0HW4__acrt_has_trailing_digits@@W4__acrt_rounding_mode@@@Z 1001877f f   libucrt:_fptostr.obj
 0001:00019460       ??R<lambda_e96123212306c92459f955e8e4eac55d>@@QBEIPBD@Z 1001a460 f   libucrt:mbrtowc.obj
 0001:000195d7       ??$common_flush_and_write_nolock@D@@YAHHV__crt_stdio_stream@@AAV__crt_cached_ptd_host@@@Z 1001a5d7 f   libucrt:_flsbuf.obj
 0001:000196cd       ??$write_buffer_nolock@D@@YA_NDV__crt_stdio_stream@@AAV__crt_cached_ptd_host@@@Z 1001a6cd f   libucrt:_flsbuf.obj
 0001:0001979f       ?stream_is_at_end_of_file_nolock@@YA_NV__crt_stdio_stream@@@Z 1001a79f f   libucrt:_flsbuf.obj
 0001:0001982f       ?get_drive_number_from_path@@YAHQB_W@Z 1001a82f f   libucrt:drive.obj
 0001:00019e0e       ??$common_tcsncpy_s@D@@YAHQADIQBDI@Z 1001ae0e f   libucrt:strncpy_s.obj
 0001:00019f74       ?initialize_multibyte@@YAHXZ 1001af74 f   libucrt:multibyte_initializer.obj
 0001:0001a1a0       $$000000                   1001b1a0     libucrt:log10_impl.obj
 0001:0001a2b0       $$000000                   1001b2b0     libucrt:ceil_pentium4.obj
 0001:0001a3cd       ?to_abstract_control@@YA?AW4__acrt_fenv_abstract_control@@W4__acrt_fenv_machine_sse_control@@@Z 1001b3cd f   libucrt:_fenvutils.obj
 0001:0001a47d       ?to_abstract_control@@YA?AW4__acrt_fenv_abstract_control@@W4__acrt_fenv_machine_x87_control@@@Z 1001b47d f   libucrt:_fenvutils.obj
 0001:0001a52a       ?to_machine_sse_control@@YA?AW4__acrt_fenv_machine_sse_control@@W4__acrt_fenv_abstract_control@@@Z 1001b52a f   libucrt:_fenvutils.obj
 0001:0001a5e0       ?to_machine_x87_control@@YA?AW4__acrt_fenv_machine_x87_control@@W4__acrt_fenv_abstract_control@@@Z 1001b5e0 f   libucrt:_fenvutils.obj
 0001:0001ab9c       ?__dcrt_lowio_initialize_console_output@@YAXXZ 1001bb9c f   libucrt:initcon.obj
 0001:0001ac46       ___hw_cw_sse2              1001bc46 f   libucrt:ieee87.obj
 0001:0001b0cc       __hw_cw                    1001c0cc f   libucrt:ieee87.obj
 0001:0001b180       $$000000                   1001c180     libucrt:log10_pentium4.obj
 0001:0001b410       $$000000                   1001c410     libucrt:87tran.obj
 0001:0001b620       $$000000                   1001c620     libucrt:87disp.obj
 0001:0001b880       $$000000                   1001c880     libucrt:common.obj
 0001:0001ba10       $$000000                   1001ca10     libucrt:genexcep.obj
 0001:0001bd20       $$000000                   1001cd20     libucrt:_strnicm.obj
 0001:0001ccd0       $$000000                   1001dcd0     LIBCMT:llmul.obj
 0001:0001cce9       hard                       1001dce9     LIBCMT:llmul.obj
 0001:0001cd10       $$000000                   1001dd10     LIBCMT:ulldiv.obj
 0001:0001cd32       L1                         1001dd32     LIBCMT:ulldiv.obj
 0001:0001cd40       L3                         1001dd40     LIBCMT:ulldiv.obj
 0001:0001cd6e       L4                         1001dd6e     LIBCMT:ulldiv.obj
 0001:0001cd6f       L5                         1001dd6f     LIBCMT:ulldiv.obj
 0001:0001cd73       L2                         1001dd73     LIBCMT:ulldiv.obj
 0001:0001cd80       $$000000                   1001dd80     LIBCMT:ullrem.obj
 0001:0001cda1       L1                         1001dda1     LIBCMT:ullrem.obj
 0001:0001cdaf       L3                         1001ddaf     LIBCMT:ullrem.obj
 0001:0001cdda       L4                         1001ddda     LIBCMT:ullrem.obj
 0001:0001cde2       L5                         1001dde2     LIBCMT:ullrem.obj
 0001:0001cdf1       L2                         1001ddf1     LIBCMT:ullrem.obj
 0001:0001ce00       $$000000                   1001de00     LIBCMT:lldiv.obj
 0001:0001ce21       L1                         1001de21     LIBCMT:lldiv.obj
 0001:0001ce3d       L2                         1001de3d     LIBCMT:lldiv.obj
 0001:0001ce59       L3                         1001de59     LIBCMT:lldiv.obj
 0001:0001ce67       L5                         1001de67     LIBCMT:lldiv.obj
 0001:0001ce95       L6                         1001de95     LIBCMT:lldiv.obj
 0001:0001ce96       L7                         1001de96     LIBCMT:lldiv.obj
 0001:0001ce9a       L4                         1001de9a     LIBCMT:lldiv.obj
 0001:0001cea4       L8                         1001dea4     LIBCMT:lldiv.obj
 0001:0001ceb0       $$000000                   1001deb0     LIBCMT:llshl.obj
 0001:0001cec0       MORE32                     1001dec0     LIBCMT:llshl.obj
 0001:0001ceca       RETZERO                    1001deca     LIBCMT:llshl.obj
 0001:0001ced0       $$000000                   1001ded0     LIBCMT:ullshr.obj
 0001:0001cee0       MORE32                     1001dee0     LIBCMT:ullshr.obj
 0001:0001ceea       RETZERO                    1001deea     LIBCMT:ullshr.obj
 0001:0001cef0       $$000000                   1001def0     LIBCMT:alloca16.obj
 0001:0001cf06       alloca_8                   1001df06     LIBCMT:alloca16.obj
 0001:0001cf20       $$000000                   1001df20     LIBCMT:chkstk.obj
 0001:0001cf34       cs10                       1001df34     LIBCMT:chkstk.obj
 0001:0001cf42       cs20                       1001df42     LIBCMT:chkstk.obj
 0001:0001cf50       $$000000                   1001df50     LIBCMT:ftol2.obj
 0001:0001cf60       $$000000                   1001df60     LIBCMT:ftol2.obj
 0001:0001cf71       L3B                        1001df71     LIBCMT:ftol2.obj
 0001:0001cfb4       L3F                        1001dfb4     LIBCMT:ftol2.obj
 0001:0001cfbc       L40                        1001dfbc     LIBCMT:ftol2.obj
 0001:0001cfcf       L41                        1001dfcf     LIBCMT:ftol2.obj
 0001:0001cff0       $$000000                   1001dff0     libvcruntime:strrchr.obj
 0001:0001d02d       strrchr_sse_loop           1001e02d     libvcruntime:strrchr.obj
 0001:0001d05d       strrchr_sse_break          1001e05d     libvcruntime:strrchr.obj
 0001:0001d07d       strrchr_sttni              1001e07d     libvcruntime:strrchr.obj
 0001:0001d08f       strrchr_sttni_chars        1001e08f     libvcruntime:strrchr.obj
 0001:0001d0a4       strrchr_sttni_aligned      1001e0a4     libvcruntime:strrchr.obj
 0001:0001d0a8       strrchr_sttni_xmm          1001e0a8     libvcruntime:strrchr.obj
 0001:0001d0bb       exit                       1001e0bb     libvcruntime:strrchr.obj
 0001:0001d0be       strrchr_zero               1001e0be     libvcruntime:strrchr.obj
 0001:0001d0e3       strchr_zero_loop           1001e0e3     libvcruntime:strrchr.obj
 0001:0001d0f7       strchr_zero_result         1001e0f7     libvcruntime:strrchr.obj
 0001:0001d0fe       strrchr_no_sse             1001e0fe     libvcruntime:strrchr.obj
 0001:0001d121       returndi                   1001e121     libvcruntime:strrchr.obj
 0001:0001d123       toend                      1001e123     libvcruntime:strrchr.obj
 0001:0001d19f       __ehhandler$?CallUnexpected@@YAXPBU_s_ESTypeList@@@Z 1001e19f f   libvcruntime:frame.obj
 0001:0001d1bc       __ehhandler$?common_exit@@YAXHW4_crt_exit_cleanup_mode@@W4_crt_exit_return_mode@@@Z 1001e1bc f   libucrt:exit.obj
 0001:0001d1d9       __ehhandler$?try_cor_exit_process@@YAXI@Z 1001e1d9 f   libucrt:exit.obj
 0001:0001d1f6       __ehhandler$___dcrt_uninitialize_environments_nolock 1001e1f6 f   libucrt:environment_initialization.obj
 0001:0001d213       __ehhandler$__execute_onexit_table 1001e213 f   libucrt:onexit.obj
 0001:0001d230       __ehhandler$?write_double_translated_ansi_nolock@@YA?AUwrite_result@?A0x17268360@@HQBDIAAV__crt_cached_ptd_host@@@Z 1001e230 f   libucrt:write.obj
 0002:000013d8       ?lenfix@?1??fixedtables@@9@9 100203d8     jli_static:inflate.obj
 0002:00001bd8       ?distfix@?1??fixedtables@@9@9 10020bd8     jli_static:inflate.obj
 0002:00001c58       ?order@?1??inflate@@9@9    10020c58     jli_static:inflate.obj
 0002:00001e68       _crc_table                 10020e68     jli_static:zcrc32.obj
 0002:00002268       _crc_big_table             10021268     jli_static:zcrc32.obj
 0002:00002668       _crc_braid_table           10021668     jli_static:zcrc32.obj
 0002:00003668       _crc_braid_big_table       10022668     jli_static:zcrc32.obj
 0002:00004668       _x2n_table                 10023668     jli_static:zcrc32.obj
 0002:000047c0       ?lbase@?1??inflate_table@@9@9 100237c0     jli_static:inftrees.obj
 0002:00004800       ?lext@?1??inflate_table@@9@9 10023800     jli_static:inftrees.obj
 0002:00004840       ?dbase@?1??inflate_table@@9@9 10023840     jli_static:inftrees.obj
 0002:00004880       ?dext@?1??inflate_table@@9@9 10023880     jli_static:inftrees.obj
 0002:000048c4       _GS_ExceptionPointers      100238c4     LIBCMT:gs_report.obj
 0002:000048d0       ?tokenTable@@3QBUStringLiteral@@B 100238d0     libvcruntime:undname.obj
 0002:00004958       ?nameTable@@3QBUStringLiteral@@B 10023958     libvcruntime:undname.obj
 0002:00004bf0       ?rttiTable@@3QBUStringLiteral@@B 10023bf0     libvcruntime:undname.obj
 0002:00004c18       ?IndirectionName@@3QBUStringLiteral@@B 10023c18     libvcruntime:undname.obj
 0002:00004c48       ?PrefixName@@3QBUStringLiteral@@B 10023c48     libvcruntime:undname.obj
 0002:00005284       ?module_names@?A0x14174aea@@3QBQB_WB 10024284     libvcruntime:winapi_downlevel.obj
 0002:0000532c       ?candidate_modules@?1??try_get_FlsAlloc@@YAP6GKP6GXPAX@Z@ZXZ@4QBW4module_id@?A0x14174aea@@B 1002432c     libvcruntime:winapi_downlevel.obj
 0002:00005340       ?candidate_modules@?1??try_get_FlsFree@@YAP6GHK@ZXZ@4QBW4module_id@?A0x14174aea@@B 10024340     libvcruntime:winapi_downlevel.obj
 0002:00005350       ?candidate_modules@?1??try_get_FlsGetValue@@YAP6GPAXK@ZXZ@4QBW4module_id@?A0x14174aea@@B 10024350     libvcruntime:winapi_downlevel.obj
 0002:00005364       ?candidate_modules@?1??try_get_FlsSetValue@@YAP6GHKPAX@ZXZ@4QBW4module_id@?A0x14174aea@@B 10024364     libvcruntime:winapi_downlevel.obj
 0002:00005378       ?candidate_modules@?1??try_get_InitializeCriticalSectionEx@@YAP6GHPAU_RTL_CRITICAL_SECTION@@KK@ZXZ@4QBW4module_id@?A0x14174aea@@B 10024378     libvcruntime:winapi_downlevel.obj
 0002:000054f0       ?errtable@@3QBUerrentry@?A0x31fdb9ec@@B 100244f0     libucrt:errno.obj
 0002:00005720       ___acrt_initializers       10024720     libucrt:initialization.obj
 0002:00006260       ?module_names@?A0x391cf84c@@3QBQB_WB 10025260     libucrt:winapi_thunks.obj
 0002:0000676c       ?candidate_modules@?1??try_get_AreFileApisANSI@@YAP6GHXZXZ@4QBW4module_id@?A0x391cf84c@@B 1002576c     libucrt:winapi_thunks.obj
 0002:00006780       ?candidate_modules@?1??try_get_InitializeCriticalSectionEx@@YAP6GHPAU_RTL_CRITICAL_SECTION@@KK@ZXZ@4QBW4module_id@?A0x391cf84c@@B 10025780     libucrt:winapi_thunks.obj
 0002:00006788       ?candidate_modules@?1??try_get_LCMapStringEx@@YAP6GHPB_WK0HPA_WHPAU_nlsversioninfo@@PAXJ@ZXZ@4QBW4module_id@?A0x391cf84c@@B 10025788     libucrt:winapi_thunks.obj
 0002:000067a0       ?candidate_modules@?1??try_get_LocaleNameToLCID@@YAP6GKPB_WK@ZXZ@4QBW4module_id@?A0x391cf84c@@B 100257a0     libucrt:winapi_thunks.obj
 0002:000067bc       ?candidate_modules@?1??try_get_AppPolicyGetProcessTerminationMethod@@YAP6GJPAXPAW4AppPolicyProcessTerminationMethod@@@ZXZ@4QBW4module_id@?A0x391cf84c@@B 100257bc     libucrt:winapi_thunks.obj
 0002:000067e8       ?candidate_modules@?1??try_get_FlsAlloc@@YAP6GKP6GXPAX@Z@ZXZ@4QBW4module_id@?A0x391cf84c@@B 100257e8     libucrt:winapi_thunks.obj
 0002:000067f0       ?candidate_modules@?1??try_get_FlsFree@@YAP6GHK@ZXZ@4QBW4module_id@?A0x391cf84c@@B 100257f0     libucrt:winapi_thunks.obj
 0002:000067f8       ?candidate_modules@?1??try_get_FlsGetValue@@YAP6GPAXK@ZXZ@4QBW4module_id@?A0x391cf84c@@B 100257f8     libucrt:winapi_thunks.obj
 0002:00006800       ?candidate_modules@?1??try_get_FlsSetValue@@YAP6GHKPAX@ZXZ@4QBW4module_id@?A0x391cf84c@@B 10025800     libucrt:winapi_thunks.obj
 0002:00006808       ?strings@?1??fp_format_nan_or_infinity@@YAHW4__acrt_fp_class@@_NPADI1@Z@4QAY03QBDA 10025808     libucrt:cvt.obj
 0002:00006890       ?_mb_locale_names@@3QBQB_WB 10025890     libucrt:mbctype.obj
 0002:000068d8       ?LcidToLocaleNameTable@?A0x881e4c05@@3QBULcidToLocaleName@1@B 100258d8     libucrt:lcidtoname_downlevel.obj
 0002:000079f8       ?LocaleNameToIndexTable@?A0x881e4c05@@3QBULocaleNameIndex@1@B 100269f8     libucrt:lcidtoname_downlevel.obj
 0002:00009330       LOG_name                   10028330     libucrt:log10_impl.obj
 0002:00009340       _One                       10028340     libucrt:ceil_pentium4.obj
 0002:00009350       _Bns                       10028350     libucrt:ceil_pentium4.obj
 0002:00009360       _Zero                      10028360     libucrt:ceil_pentium4.obj
 0002:00009370       _S                         10028370     libucrt:ceil_pentium4.obj
 0002:00009380       _NegZero                   10028380     libucrt:ceil_pentium4.obj
 0002:000093a0       emask                      100283a0     libucrt:log10_pentium4.obj
 0002:000093b0       CC                         100283b0     libucrt:log10_pentium4.obj
 0002:000093c0       Magic                      100283c0     libucrt:log10_pentium4.obj
 0002:000093d0       hi_mask                    100283d0     libucrt:log10_pentium4.obj
 0002:000093e0       LOG10_2                    100283e0     libucrt:log10_pentium4.obj
 0002:000093f0       place_L                    100283f0     libucrt:log10_pentium4.obj
 0002:00009410       One                        10028410     libucrt:log10_pentium4.obj
 0002:00009420       Zero                       10028420     libucrt:log10_pentium4.obj
 0002:00009430       Two52                      10028430     libucrt:log10_pentium4.obj
 0002:00009440       Infs                       10028440     libucrt:log10_pentium4.obj
 0002:00009450       NaN                        10028450     libucrt:log10_pentium4.obj
 0002:00009460       coeff                      10028460     libucrt:log10_pentium4.obj
 0002:000094be       _log2max                   100284be     libucrt:87tran.obj
 0002:000094c8       _smallarg                  100284c8     libucrt:87tran.obj
 0002:000094d2       _half                      100284d2     libucrt:87tran.obj
 0002:0000951e       One                        1002851e     libucrt:87disp.obj
 0002:00009526       Three                      10028526     libucrt:87disp.obj
 0002:0000952e       XAMtoTagTab                1002852e     libucrt:87disp.obj
 0002:00009540       One                        10028540     libucrt:common.obj
 0002:00009554       DblMax                     10028554     libucrt:common.obj
 0002:0000955c       DblMin                     1002855c     libucrt:common.obj
 0002:00009564       IeeeAdjO                   10028564     libucrt:common.obj
 0002:0000956c       IeeeAdjU                   1002856c     libucrt:common.obj
 0002:00009574       _infinity                  10028574     libucrt:common.obj
 0002:0000957c       _zero                      1002857c     libucrt:common.obj
 0002:000095b8       _over                      100285b8     libucrt:fpctrl.obj
 0002:000095c4       _under                     100285c4     libucrt:fpctrl.obj
 0002:00009df8       ?_names@?1??_get_fname@@9@4QBU<unnamed-type-_names>@?1??1@YAPADI@Z@B 10028df8     libucrt:fpexcept.obj
 0002:00009fa0       two32                      10028fa0     LIBCMT:ftol2.obj
 0002:00009fa4       two63                      10028fa4     LIBCMT:ftol2.obj
 0002:00009fa8       _NaN                       10028fa8     LIBCMT:ftol2.obj
 0002:0000a768       __sehtable$?dllmain_crt_process_attach@@YAHQAUHINSTANCE__@@QAX@Z 10029768     LIBCMT:dll_dllmain.obj
 0002:0000a788       __sehtable$?dllmain_crt_process_detach@@YAH_N@Z 10029788     LIBCMT:dll_dllmain.obj
 0002:0000a7b0       __sehtable$?dllmain_dispatch@@YAHQAUHINSTANCE__@@KQAX@Z 100297b0     LIBCMT:dll_dllmain.obj
 0002:0000a7d0       __sehtable$___scrt_is_nonwritable_in_current_image 100297d0     LIBCMT:utility.obj
 0002:0000a7f0       __sehtable$___DestructExceptionObject 100297f0     libvcruntime:ehhelpers.obj
 0002:0000a810       __sehtable$?FrameUnwindToState@__FrameHandler3@@SAXPAUEHRegistrationNode@@PAXPBU_s_FuncInfo@@H@Z 10029810     libvcruntime:frame.obj
 0002:0000a838       __sehtable$?CallCatchBlock@@YAPAXPAUEHExceptionRecord@@PAUEHRegistrationNode@@PAU_CONTEXT@@PBU_s_FuncInfo@@PAXHK@Z 10029838     libvcruntime:frame.obj
 0002:0000a860       __catchsym$?CallUnexpected@@YAXPBU_s_ESTypeList@@@Z$2 10029860     libvcruntime:frame.obj
 0002:0000a870       __unwindtable$?CallUnexpected@@YAXPBU_s_ESTypeList@@@Z 10029870     libvcruntime:frame.obj
 0002:0000a880       __tryblocktable$?CallUnexpected@@YAXPBU_s_ESTypeList@@@Z 10029880     libvcruntime:frame.obj
 0002:0000a894       __ehfuncinfo$?CallUnexpected@@YAXPBU_s_ESTypeList@@@Z 10029894     libvcruntime:frame.obj
 0002:0000a8b8       __sehtable$??$BuildCatchObjectHelperInternal@V__FrameHandler3@@@@YAHPAUEHExceptionRecord@@PAXPBU_s_HandlerType@@PBU_s_CatchableType@@@Z 100298b8     libvcruntime:frame.obj
 0002:0000a8d8       __sehtable$??$BuildCatchObjectInternal@V__FrameHandler3@@@@YAXPAUEHExceptionRecord@@PAXPBU_s_HandlerType@@PBU_s_CatchableType@@@Z 100298d8     libvcruntime:frame.obj
 0002:0000a948       __sehtable$??$?RV<lambda_62491a2101a2aba6cc4a769149c84f1f>@@AAV<lambda_826c27fce7726908515bbc79a5266961>@@V<lambda_4e64bbd54b50a7b070e3ea8d795375b6>@@@?$__crt_seh_guarded_call@H@@QAEH$$QAV<lambda_62491a2101a2aba6cc4a769149c84f1f>@@AAV<lambda_826c27fce7726908515bbc79a5266961>@@$$QAV<lambda_4e64bbd54b50a7b070e3ea8d795375b6>@@@Z 10029948     libucrt:output.obj
 0002:0000a968       __sehtable$??$common_lseek@_J@@YA_JH_JHAAV__crt_cached_ptd_host@@@Z 10029968     libucrt:lseek.obj
 0002:0000a984       __ehfuncinfo$?write_double_translated_ansi_nolock@@YA?AUwrite_result@?A0x17268360@@HQBDIAAV__crt_cached_ptd_host@@@Z 10029984     libucrt:write.obj
 0002:0000a984       __ehfuncinfo$?try_cor_exit_process@@YAXI@Z 10029984     libucrt:exit.obj
 0002:0000a9a8       __unwindtable$?common_exit@@YAXHW4_crt_exit_cleanup_mode@@W4_crt_exit_return_mode@@@Z 100299a8     libucrt:exit.obj
 0002:0000a9b0       __ehfuncinfo$?common_exit@@YAXHW4_crt_exit_cleanup_mode@@W4_crt_exit_return_mode@@@Z 100299b0     libucrt:exit.obj
 0002:0000a9d8       __sehtable$??R<lambda_6e4b09c48022b2350581041d5f6b0c4c>@@QBE@XZ 100299d8     libucrt:exit.obj
 0002:0000a9f8       __sehtable$??$?RV<lambda_03b1d95aef87969028cfba75ccab2455>@@AAV<lambda_6e4b09c48022b2350581041d5f6b0c4c>@@V<lambda_22bdf7517842c4b3e53723af5aa32b9e>@@@?$__crt_seh_guarded_call@X@@QAEX$$QAV<lambda_03b1d95aef87969028cfba75ccab2455>@@AAV<lambda_6e4b09c48022b2350581041d5f6b0c4c>@@$$QAV<lambda_22bdf7517842c4b3e53723af5aa32b9e>@@@Z 100299f8     libucrt:exit.obj
 0002:0000aa14       __unwindtable$___dcrt_uninitialize_environments_nolock 10029a14     libucrt:environment_initialization.obj
 0002:0000aa24       __ehfuncinfo$___dcrt_uninitialize_environments_nolock 10029a24     libucrt:environment_initialization.obj
 0002:0000aa48       __unwindtable$__execute_onexit_table 10029a48     libucrt:onexit.obj
 0002:0000aa50       __ehfuncinfo$__execute_onexit_table 10029a50     libucrt:onexit.obj
 0002:0000aa78       __sehtable$??$?RV<lambda_69a2805e680e0e292e8ba93315fe43a8>@@AAV<lambda_f03950bc5685219e0bcd2087efbe011e>@@V<lambda_03fcd07e894ec930e3f35da366ca99d6>@@@?$__crt_seh_guarded_call@H@@QAEH$$QAV<lambda_69a2805e680e0e292e8ba93315fe43a8>@@AAV<lambda_f03950bc5685219e0bcd2087efbe011e>@@$$QAV<lambda_03fcd07e894ec930e3f35da366ca99d6>@@@Z 10029a78     libucrt:onexit.obj
 0002:0000aa98       __sehtable$_terminate      10029a98     libucrt:terminate.obj
 0002:0000aab8       __sehtable$??$?RV<lambda_d422a76eb4c3bf3ad751449ab71a6ea4>@@AAV<lambda_c9ba49e555ba839a7b07aa3fbecb7617>@@V<lambda_9476263c8ee91a25d21c55370bdb50de>@@@?$__crt_seh_guarded_call@H@@QAEH$$QAV<lambda_d422a76eb4c3bf3ad751449ab71a6ea4>@@AAV<lambda_c9ba49e555ba839a7b07aa3fbecb7617>@@$$QAV<lambda_9476263c8ee91a25d21c55370bdb50de>@@@Z 10029ab8     libucrt:close.obj
 0002:0000aad8       __sehtable$??$common_open@D@@YAHQBDHH@Z 10029ad8     libucrt:open.obj
 0002:0000aaf8       __sehtable$__read          10029af8     libucrt:read.obj
 0002:0000ab18       __sehtable$??$?RV<lambda_15ade71b0218206bbe3333a0c9b79046>@@AAV<lambda_da44e0f8b0f19ba52fefafb335991732>@@V<lambda_207f2d024fc103971653565357d6cd41>@@@?$__crt_seh_guarded_call@X@@QAEX$$QAV<lambda_15ade71b0218206bbe3333a0c9b79046>@@AAV<lambda_da44e0f8b0f19ba52fefafb335991732>@@$$QAV<lambda_207f2d024fc103971653565357d6cd41>@@@Z 10029b18     libucrt:per_thread_data.obj
 0002:0000ab38       __sehtable$??$?RV<lambda_a7e850c220f1c8d1e6efeecdedd162c6>@@AAV<lambda_46720907175c18b6c9d2717bc0d2d362>@@V<lambda_9048902d66e8d99359bc9897bbb930a8>@@@?$__crt_seh_guarded_call@X@@QAEX$$QAV<lambda_a7e850c220f1c8d1e6efeecdedd162c6>@@AAV<lambda_46720907175c18b6c9d2717bc0d2d362>@@$$QAV<lambda_9048902d66e8d99359bc9897bbb930a8>@@@Z 10029b38     libucrt:per_thread_data.obj
 0002:0000ab58       __sehtable$??$?RV<lambda_38edbb1296d33220d7e4dd0ed76b244a>@@AAV<lambda_5ce1d447e08cb34b2473517608e21441>@@V<lambda_fb385d3da700c9147fc39e65dd577a8c>@@@?$__crt_seh_guarded_call@X@@QAEX$$QAV<lambda_38edbb1296d33220d7e4dd0ed76b244a>@@AAV<lambda_5ce1d447e08cb34b2473517608e21441>@@$$QAV<lambda_fb385d3da700c9147fc39e65dd577a8c>@@@Z 10029b58     libucrt:per_thread_data.obj
 0002:0000ab78       __sehtable$??$?RV<lambda_6affb1475c98b40b75cdec977db92e3c>@@AAV<lambda_b8d4b9c228a6ecc3f80208dbb4b4a104>@@V<lambda_608742c3c92a14382c1684fc64f96c88>@@@?$__crt_seh_guarded_call@X@@QAEX$$QAV<lambda_6affb1475c98b40b75cdec977db92e3c>@@AAV<lambda_b8d4b9c228a6ecc3f80208dbb4b4a104>@@$$QAV<lambda_608742c3c92a14382c1684fc64f96c88>@@@Z 10029b78     libucrt:per_thread_data.obj
 0002:0000ab98       __sehtable$??$?RV<lambda_e5124f882df8998aaf41531e079ba474>@@AAV<lambda_3e16ef9562a7dcce91392c22ab16ea36>@@V<lambda_e25ca0880e6ef98be67edffd8c599615>@@@?$__crt_seh_guarded_call@X@@QAEX$$QAV<lambda_e5124f882df8998aaf41531e079ba474>@@AAV<lambda_3e16ef9562a7dcce91392c22ab16ea36>@@$$QAV<lambda_e25ca0880e6ef98be67edffd8c599615>@@@Z 10029b98     libucrt:wsetlocale.obj
 0002:0000abb8       __sehtable$__fcloseall     10029bb8     libucrt:closeall.obj
 0002:0000abd8       __sehtable$??$?RV<lambda_2866be3712abc81a800a822484c830d8>@@AAV<lambda_39ca0ed439415581b5b15c265174cece>@@V<lambda_2b24c74d71094a6cd0cb82e44167d71b>@@@?$__crt_seh_guarded_call@X@@QAEX$$QAV<lambda_2866be3712abc81a800a822484c830d8>@@AAV<lambda_39ca0ed439415581b5b15c265174cece>@@$$QAV<lambda_2b24c74d71094a6cd0cb82e44167d71b>@@@Z 10029bd8     libucrt:fflush.obj
 0002:0000abf8       __sehtable$??$?RV<lambda_2cc53f568c5a2bb6f192f930a45d44ea>@@AAV<lambda_ab61a845afdef5b7c387490eaf3616ee>@@V<lambda_c2ffc0b7726aa6be21d5f0026187e748>@@@?$__crt_seh_guarded_call@X@@QAEX$$QAV<lambda_2cc53f568c5a2bb6f192f930a45d44ea>@@AAV<lambda_ab61a845afdef5b7c387490eaf3616ee>@@$$QAV<lambda_c2ffc0b7726aa6be21d5f0026187e748>@@@Z 10029bf8     libucrt:fflush.obj
 0002:0000ac18       __sehtable$___acrt_initialize_lowio 10029c18     libucrt:ioinit.obj
 0002:0000ac38       __sehtable$__alloc_osfhnd  10029c38     libucrt:osfinfo.obj
 0002:0000ac58       __sehtable$___acrt_lowio_ensure_fh_exists 10029c58     libucrt:osfinfo.obj
 0002:0000ac78       __sehtable$?update_thread_multibyte_data_internal@@YAPAU__crt_multibyte_data@@QAU__acrt_ptd@@QAPAU1@@Z 10029c78     libucrt:mbctype.obj
 0002:0000ac98       __sehtable$??$?RV<lambda_ceb1ee4838e85a9d631eb091e2fbe199>@@AAV<lambda_ae742caa10f662c28703da3d2ea5e57e>@@V<lambda_cd08b5d6af4937fe54fc07d0c9bf6b37>@@@?$__crt_seh_guarded_call@X@@QAEX$$QAV<lambda_ceb1ee4838e85a9d631eb091e2fbe199>@@AAV<lambda_ae742caa10f662c28703da3d2ea5e57e>@@$$QAV<lambda_cd08b5d6af4937fe54fc07d0c9bf6b37>@@@Z 10029c98     libucrt:mbctype.obj
 0002:0000acb8       __sehtable$__query_new_handler 10029cb8     libucrt:new_handler.obj
 0002:0000acd8       __sehtable$_raise          10029cd8     libucrt:signal.obj
 0002:0000acf8       __sehtable$??$?RV<lambda_cbab9ec6f41b0180b23cc171c22676b0>@@AAV<lambda_44731a7d0e6d81c3e6aa82d741081786>@@V<lambda_4b292cb8dd18144e164572427af410ab>@@@?$__crt_seh_guarded_call@P6AXH@Z@@QAEP6AXH@Z$$QAV<lambda_cbab9ec6f41b0180b23cc171c22676b0>@@AAV<lambda_44731a7d0e6d81c3e6aa82d741081786>@@$$QAV<lambda_4b292cb8dd18144e164572427af410ab>@@@Z 10029cf8     libucrt:signal.obj
 0002:0000ad18       __sehtable$__write_internal 10029d18     libucrt:write.obj
 0002:0000ad38       __sehtable$___acrt_update_thread_locale_data 10029d38     libucrt:locale_refcounting.obj
 0002:0000ad58       __sehtable$?_fclose_internal@@YAHQAU_iobuf@@AAV__crt_cached_ptd_host@@@Z 10029d58     libucrt:fclose.obj
 0002:0000ad78       __sehtable$??$?RV<lambda_9e9de3de5fa147e2223d7db92bc10aa6>@@AAV<lambda_38ce7e780aa69e748d6df282ebc68efe>@@V<lambda_8ca6da459f0f6780f1cff60fdc3d00e5>@@@?$__crt_seh_guarded_call@H@@QAEH$$QAV<lambda_9e9de3de5fa147e2223d7db92bc10aa6>@@AAV<lambda_38ce7e780aa69e748d6df282ebc68efe>@@$$QAV<lambda_8ca6da459f0f6780f1cff60fdc3d00e5>@@@Z 10029d78     libucrt:commit.obj
 0002:0000ad98       __sehtable$___set_fpsr_sse2 10029d98     libucrt:fpctrl.obj
 0002:0000adb8       __sehtable$__IsNonwritableInCurrentImage 10029db8     LIBCMT:pesect.obj
 0002:0000ade0       .edata                     10029de0     instrument.exp
 0002:0000ae08       rgpv                       10029e08     instrument.exp
 0002:0000ae3c       rgszName                   10029e3c     instrument.exp
 0002:0000ae70       rgwOrd                     10029e70     instrument.exp
 0002:0000ae8a       szName                     10029e8a     instrument.exp
 0002:0000ae99       $N00001                    10029e99     instrument.exp
 0002:0000aea8       $N00002                    10029ea8     instrument.exp
 0002:0000aeb9       $N00003                    10029eb9     instrument.exp
 0002:0000aecb       $N00004                    10029ecb     instrument.exp
 0002:0000af12       $N00005                    10029f12     instrument.exp
 0002:0000af53       $N00006                    10029f53     instrument.exp
 0002:0000af94       $N00007                    10029f94     instrument.exp
 0002:0000afcf       $N00008                    10029fcf     instrument.exp
 0002:0000b00e       $N00009                    1002a00e     instrument.exp
 0002:0000b059       $N00010                    1002a059     instrument.exp
 0002:0000b096       $N00011                    1002a096     instrument.exp
 0002:0000b0d6       $N00012                    1002a0d6     instrument.exp
 0002:0000b124       $N00013                    1002a124     instrument.exp
 0002:0000b490       .idata$6                   1002a490     kernel32:KERNEL32.dll
 0003:00000000       _manifest_name             1002b000     jli_static:parse_manifest.obj
 0003:00000030       ?__vcrt_flsindex@@3KA      1002b030     libvcruntime:per_thread_data.obj
 0003:00000100       ?errno_no_memory@@3HA      1002b100     libucrt:errno.obj
 0003:00000104       ?doserrno_no_memory@@3KA   1002b104     libucrt:errno.obj
 0003:00000220       ?__acrt_flsindex@@3KA      1002b220     libucrt:per_thread_data.obj
 0003:00000548       __mbctypes                 1002b548     libucrt:mbctype.obj
 0003:00000650       __mbcasemaps               1002b650     libucrt:mbctype.obj
 0003:00000750       ?__rgctypeflag@@3PADA      1002b750     libucrt:mbctype.obj
 0003:00000758       ?__rgcode_page_info@@3PAUcode_page_info@@A 1002b758     libucrt:mbctype.obj
 0003:000008b0       ?__dcrt_lowio_console_output_handle@@3PAXA 1002b8b0     libucrt:initcon.obj
 0003:000008c0       ?__DAZ_ENABLED@?1??__set_fpsr_sse2@@9@9 1002b8c0     libucrt:fpctrl.obj
 0003:00000938       _sFallbackInternalError    1002b938     JavaExceptions.obj
 0003:00000940       _L_HEX                     1002b940     PathCharsValidator.obj
 0003:00000948       _H_HEX                     1002b948     PathCharsValidator.obj
 0003:00000950       _L_PATH                    1002b950     PathCharsValidator.obj
 0003:00000958       _H_PATH                    1002b958     PathCharsValidator.obj
 0003:00000960       _manifest                  1002b960     jli_static:parse_manifest.obj
 0003:00000964       _zip64_present             1002b964     jli_static:parse_manifest.obj
 0003:00000968       ?__proc_attached@@3HA      1002b968     LIBCMT:dll_dllmain.obj
 0003:00000970       _GS_ExceptionRecord        1002b970     LIBCMT:gs_report.obj
 0003:000009c0       _GS_ContextRecord          1002b9c0     LIBCMT:gs_report.obj
 0003:00000ca8       ?is_initialized_as_dll@@3_NA 1002bca8     LIBCMT:utility.obj
 0003:00000ca9       ?module_local_atexit_table_initialized@@3_NA 1002bca9     LIBCMT:utility.obj
 0003:00000cac       ?module_local_atexit_table@@3U_onexit_table_t@@A 1002bcac     LIBCMT:utility.obj
 0003:00000cb8       ?module_local_at_quick_exit_table@@3U_onexit_table_t@@A 1002bcb8     LIBCMT:utility.obj
 0003:00000cfc       ?heap@@3V_HeapManager@@A   1002bcfc     libvcruntime:undname.obj
 0003:00000d10       ?__vcrt_startup_thread_ptd@@3U__vcrt_ptd@@A 1002bd10     libvcruntime:per_thread_data.obj
 0003:00000d38       ___vcrt_lock_table         1002bd38     libvcruntime:locks.obj
 0003:00000d50       ___vcrt_locks_initialized  1002bd50     libvcruntime:locks.obj
 0003:00000d54       ?module_handles@@3PAPAUHINSTANCE__@@A 1002bd54     libvcruntime:winapi_downlevel.obj
 0003:00000d60       ?function_pointers@@3PAPAXA 1002bd60     libvcruntime:winapi_downlevel.obj
 0003:00000d84       ?c_termination_complete@@3JA 1002bd84     libucrt:exit.obj
 0003:00000d88       ?thread_local_exit_callback_func@@3P6GXPAXK0@ZA 1002bd88     libucrt:exit.obj
 0003:00000d8c       ?c_exit_complete@?1???R<lambda_6e4b09c48022b2350581041d5f6b0c4c>@@QBE@XZ@4_NA 1002bd8c     libucrt:exit.obj
 0003:00000d90       ?program_name@?1???$common_configure_argv@D@@YAHW4_crt_argv_mode@@@Z@4PADA 1002bd90     libucrt:argv_parsing.obj
 0003:00000ec0       ?__acrt_invalid_parameter_handler@@3V?$dual_state_global@P6AXPB_W00II@Z@__crt_state_management@@A 1002bec0     libucrt:invalid_parameter.obj
 0003:00000ed0       ?module_handles@@3PAPAUHINSTANCE__@@A 1002bed0     libucrt:winapi_thunks.obj
 0003:00000f28       ?encoded_function_pointers@@3PAPAXA 1002bf28     libucrt:winapi_thunks.obj
 0003:000011bc       ?internal_state@?1??_mbtowc_internal@@9@4U_Mbstatet@@A 1002c1bc     libucrt:mbtowc.obj
 0003:000011c4       ?enable_percent_n@@3IA     1002c1c4     libucrt:printf_count_output.obj
 0003:000011d0       ?__acrt_lock_table@@3PAU_RTL_CRITICAL_SECTION@@A 1002c1d0     libucrt:locks.obj
 0003:00001320       ?__acrt_locks_initialized@@3IA 1002c320     libucrt:locks.obj
 0003:00001330       ?fSystemSet@@3HA           1002c330     libucrt:mbctype.obj
 0003:00001334       ?initialized@?1??__acrt_initialize_multibyte@@9@4_NA 1002c334     libucrt:mbctype.obj
 0003:00001354       ?__acrt_new_handler@@3V?$dual_state_global@P6AHI@Z@__crt_state_management@@A 1002c354     libucrt:new_handler.obj
 0003:00001358       ?ctrlc_action@@3V?$dual_state_global@P6AXH@Z@__crt_state_management@@A 1002c358     libucrt:signal.obj
 0003:0000135c       ?ctrlbreak_action@@3V?$dual_state_global@P6AXH@Z@__crt_state_management@@A 1002c35c     libucrt:signal.obj
 0003:00001360       ?abort_action@@3V?$dual_state_global@P6AXH@Z@__crt_state_management@@A 1002c360     libucrt:signal.obj
 0003:00001364       ?term_action@@3V?$dual_state_global@P6AXH@Z@__crt_state_management@@A 1002c364     libucrt:signal.obj
 0003:00001368       ?user_matherr@@3V?$dual_state_global@P6AHPAU_exception@@@Z@__crt_state_management@@A 1002c368     libucrt:matherr.obj
 0003:00001370       ?__acrt_global_new_mode@@3V?$dual_state_global@J@__crt_state_management@@A 1002c370     libucrt:new_mode.obj
 0003:0000137c       ?__acrt_app_type@@3W4_crt_app_type@@A 1002c37c     libucrt:report_runtime_error.obj
 0003:00001384       ?internal_pst@?1??__mbrtoc32_utf8@__crt_mbstring@@YAIPA_UPBDIPAU_Mbstatet@@AAV__crt_cached_ptd_host@@@Z@4U3@A 1002c384     libucrt:mbrtoc32.obj
 0003:00001390       __pmatherr_set             1002c390     libucrt:libm_error.obj
 0004:00000060       $R000000                   1002d060     instrument.dll.res
